:040000006F80F021FC
:100004000000000000000000E0760000E27600003E
:10001400000000001C8A0000000000000000000036
:100024001C8A00001C8A0000000000000000000080
:100034001C8A0000000000001C8A00000000000070
:100044001C8A00001C8A00001C8A00001C8A000014
:100054001C8A00001C8A00001C8A00001C8A000004
:100064001C8A00001C8A00001C8A00001C8A0000F4
:100074001C8A00001C8A00001C8A00001C8A0000E4
:100084001C8A00001C8A00001C8A00001C8A0000D4
:100094001C8A00001C8A00001C8A00001C8A0000C4
:1000A4001C8A00001C8A00001C8A00001C8A0000B4
:1000B4001C8A00001C8A00001C8A00001C8A0000A4
:1000C4001C8A00001C8A00001C8A00001C8A000094
:1000D4001C8A00001C8A00001C8A00001C8A000084
:1000E4001C8A00001C8A00001C8A00001C8A000074
:1000F4001C8A00001C8A00001C8A00001C8A000064
:10010400000000001C8A00001C8A00001C8A0000F9
:100114001C8A00001C8A00001C8A00001C8A000043
:100124001C8A00001C8A00001C8A00001C8A000033
:100134001C8A00001C8A00001C8A00001C8A000023
:100144001C8A00001C8A00001C8A00001C8A000013
:100154001C8A00001C8A00001C8A00001C8A000003
:100164001C8A00001C8A00001C8A00001C8A0000F3
:100174001C8A00001C8A00001C8A00001C8A0000E3
:100184001C8A00001C8A00001C8A00001C8A0000D3
:100194001C8A00001C8A00001C8A00001C8A0000C3
:1001A400000000000000000000000000000000004B
:0C01B4000000000000000000000000003F
:1001C000397101436EC619A0397141536AC866CAB4
:1001D00062CC5ECE19A0397101535AD056D252D496
:1001E0004ED64AD826DA22DC06DE3301614082820E
:1001F00041114AC026C222C406C68282B24D4101C4
:10020000024D924C224CB24B4101024B924A224A7F
:10021000B2494101024992442244B24041018280E4
:100220003D432A876373C3029377F700BDEFADE5C3
:10023000937606FF3D8ABA960CC34CC30CC74CC7D5
:100240004107E36BD7FE11E28280B306C3408A0602
:100250009702000096966780A6002307B700A306C2
:10026000B7002306B700A305B7002305B700A30412
:10027000B7002304B700A303B7002303B700A3020A
:10028000B7002302B700A301B7002301B700A30002
:10029000B7002300B700828093F5F50F9396850091
:1002A000D58D93960501D58D61B79396270097025A
:1002B000000096968682E78086FA9680C1171D8F89
:1002C0003E96E374C3F8A5B73367B500FD530D8BB5
:1002D00079E7B7877F7F9387F7F710419441B3722F
:1002E000F6003363F600BE92B3E262006395720CCF
:1002F0006318D6065041D441B372F6003363F6005A
:10030000BE92B3E262006396720A631BD604104584
:100310009445B372F6003363F600BE92B3E2620016
:10032000639F7208631ED6025045D445B372F6002F
:100330003363F600BE92B3E2620063987208631101
:10034000D60210499449B372F6003363F600BE92A8
:10035000B3E26200639172085105D105E30FD6F64E
:100360001317060193970601631CF7001357060144
:1003700093D706013305F7409375F50F91E9828015
:100380004183C1833305F7409375F50F91E1828076
:100390001377F70F93F7F70F3305F740828010219B
:1003A0009421050585056313D60075FA3305D640FB
:1003B000828011059105E314D6FE01458280210556
:1003C000A105E31ED6FC014582803105B105E31885
:1003D000D6FC014582804105C105E312D6FC0145EA
:1003E0008280EFF2FFDD4111AE8A328901C9AA8510
:1003F00037B500001305C545EF90E07CD6894A8AE1
:10040000C14437BB0000B7BB000037BC0000B7ECED
:10041000000037BD0000138404FF63642401410120
:10042000F1BBA2851305CB46EF90E07963742407F6
:10043000B3878A008C2313054C47EF90C0780504DE
:10044000E39684FE13854C22EF90E0770144C14D82
:1004500063088A02B38789008C232EC6EF90E04799
:10046000B2452E958307150093F7770999E3930515
:10047000E00213050D480504EF90E074E31AB4FDA3
:1004800037E5000013058599EF90E073C104411A28
:10049000C10951B71385CB47EF90E0724DB7EFF22A
:1004A0009FD332843689AA84330AB5008147930AE0
:1004B000E6FF37BB0000638644019389270063E8A9
:1004C000290163E127034A94A30F04FE39A894206D
:1004D00013064B488D4533853A01EF90D0188504BB
:1004E000CE87D1BF3E942300040005B3EFF25FD066
:1004F00065713284AA842E891306401081456801F3
:100500000533B54748102306F108EF6030174A86D7
:10051000A6854810EF60101D13060002A285481042
:10052000EF60501C4C004810EF60502E924768015D
:10053000BECD9147BECBEF1050765961E1B9EFF2D5
:100540003FCB11712A849305C504130640020A8526
:10055000EF90204024449305040B48101386C4F9FF
:10056000EF90203FB70500200A86938604FC938510
:10057000053913050407EF30E021116161B98347A4
:10058000F50A93F7070EB1E3EFF29FC611719304DA
:10059000C5042A84A685130640020A85EF90603BB5
:1005A000032984049305040B48101306C9F9EF903E
:1005B000403A0A86930609FCA68513050407EF3026
:1005C000A01E133515001161B1B101458280EFF213
:1005D0009FC013351500370400206D7145051304C5
:1005E000C43848861306000293054402A808EF9019
:1005F0004036EF80904103474404AADC8546AA892F
:10060000930710086303D702894693072008630EF7
:10061000D7008D46930730086309D70091469307AA
:1006200000086314D700930740083704002013051F
:10063000143D230EF10AEF901011AA842A86930527
:10064000143D1305D10BEF90C03013895406680098
:10065000CACAF53537B50000AC0813060002130509
:10066000455D413337B50000EC181306000413054F
:10067000055E853B37B50000138614006C19130521
:10068000C55E853337B50000CE851305455FEF9015
:10069000805337B500009305143D13058560EF9036
:1006A00080526800CACAA3080100EF10105F5161B0
:1006B000A9BEEFF2FFB3AA8408211971EF60703D63
:1006C0002A8401E9EF60D0381306800B81452A8423
:1006D000813E93854407130600022285EF90602730
:1006E00013060002A68513050402EF908026A68556
:1006F0000A85EF50B02CB7050020130600028800D1
:1007000093850539EF2050748C000810EF508070ED
:100710000A860C1013050404EF508072BC543CD0C0
:10072000FC547CD083C75406BD8B2305F40AEF80AC
:10073000D02D9C502328A40A2326F40A0961D9BC91
:10074000EFF21FAB834755062A849305450713979D
:100750008701618763460700B7B50000938585551B
:100760009D8B91461050638DD7048D46638FD704BF
:1007700089466381D706B7B60000938686586340E2
:10078000070637B700001307C7590328C4063C54AF
:1007900037B500001305455AEF90E04237B5000029
:1007A000A285130600021305455D253937B5000003
:1007B00013060004930544021305055E1D3199BC20
:1007C000B7B60000938646575DBFB7B60000938664
:1007D000C65775B7B7B60000938686564DB737B77C
:1007E00000001307475955B7EFF2FF9E71712A8435
:1007F00013064009814568082534344493074006B0
:10080000B7BA000063E0D702B7B5000037B5000003
:100810001386CA489385454913058549EF90A03A48
:100820004D61E5B22285A13B1386CA4801EDB7B5FB
:10083000000037B50000938545491305C54CEF907E
:100840008038F9BFB7B5000037B500009385C54EB5
:100850001305054FEF902037130AC404854713068C
:100860000002D28568082300F108EF90800E11463F
:100870009305C4066818EF90C00D13060004930595
:1008800004078800EF90E00C8347040B930950069F
:10089000A300F10813F6070119C29309D00613FB50
:1008A0000702CE8463040B009384290013F9070424
:1008B000268763060900138724001377F70F344453
:1008C00063FFE600B7B5000037B500001386CA48DD
:1008D0009385454913058551EF90E02E91B70DC2E0
:1008E00011469305140B48013AC636C4EF906006D2
:1008F00011469305540B2801EF90A0053247A246FC
:10090000630B0B00D29983C709002306F10883C744
:100910001900A306F10863090900D2949C2023075B
:10092000F1089C30A307F108998E93F6F60FFD4766
:1009300013F4F60F63F3D7007D442286B305EA0073
:100940000809EF9000011C193E946808230004FE7A
:10095000C53B6808B93BE9B581476387B7003307F2
:10096000F5000307070019E33E8582808507F5B788
:1009700063050516EFF23F862A84AE89AA8537B54E
:10098000000013054575EF9000240C2037B50000DA
:1009900013054577EF90202337B50000130505793F
:1009A000EF906022854437BA000013091002B307A4
:1009B00094008C2313054A7A8504EF90C020E398B5
:1009C00024FF37E9000013058999EF90C01F2E30EE
:1009D00037B500001305C57AEF90E01E8345440249
:1009E00037B500001305457CEF90E01D0347440236
:1009F0008D47814463F7E70283476402034754024B
:100A000083458402A2075D8F83477402E20537B5F0
:100A10000000C207D98FDD8D1305857EEF90A01AE7
:100A20009144638C0904834744029386340063D65F
:100A3000F604138714001377F70FB3079400229777
:100A400003C6570283475702138724001377F70F13
:100A5000229783455702A207A296C205CD8F83C570
:100A60005602D18F37B50000E2059104DD8D1305E4
:100A7000C57F93F4F40FEF9000158347440263F2AF
:100A8000F404858F93F7F70F414793F5F70F6373DE
:100A9000F700C1451385540222957D3D9379F50FEA
:100AA00037C50000130545812694EF90C01181449D
:100AB00037BA000005046398990013058999EF90EF
:100AC00080106FF08FF48345440213050A488504B3
:100AD000EF90600F93F4F40FF1BF8280EFF2AFEF6D
:100AE0008347C5046571AA849305D50413060002E3
:100AF00013059101230CF100EF80B06583C7E40674
:100B000003C7D40603459101A207D98F231DF10223
:100B1000EF60207837B9000037BA0000631D051E6A
:100B2000EF6000731306800B81452A84EFF04FEFCE
:100B3000B7B50000938585612285EF90C03F13060D
:100B40000002930591012304040613050402EF80BB
:100B5000506093059101C809EF504066B705002029
:100B6000D0099385053913050404EF50602D232027
:100B70000406232204062305040AEF8000692328C3
:100B8000A40A37B50000A286130689629305CA4EEF
:100B900013054563EF902003B4441307D103138674
:100BA000D4069386F6FD9305000213050404EF10A6
:100BB000904AB04437B500009305D1031306D6FD23
:100BC0001376F60F13058569230EC102EFF07F81BE
:100BD0000347E1038347D103914922075D8F834790
:100BE000F103C2075D8F83470104E207D98F2326F3
:100BF000F40AB707002083C5073D8D476393F502CC
:100C00000347210483471104A14922075D8F8347CD
:100C10003104C2075D8F83474104E207D98F232A3D
:100C2000F40AF51593B51500280899338347C103D5
:100C30003808B38737419389590293F7F70FBA9968
:100C4000414793F5F70F6373F700C1454E8529338C
:100C5000937AF50F37B50000D6861306896293059F
:100C6000CA4E1305856AEF8010765686CE85280019
:100C7000EF80304E5686938501762800EF80304B0A
:100C80004DE9854737B50000A286130689629305B2
:100C9000CA4EA305F40A1305856CEF80D07237B5F0
:100CA0000000A286130689629305CA4E1305C56F1C
:100CB000EF807071EF806055AACBEF90E005A30C38
:100CC000010C230D010C8347B40AA30DF10C91C351
:100CD0008D47230EF10C93578500230FF10C93578A
:100CE0000501A30FF10C8547A300F10EA547230CC6
:100CF000F10C9C20A30EA10C61812300A10E898B15
:100D000089E79385540022856523CC09228515291E
:100D100059616FF08FCF2A84B7B5000037B5000056
:100D2000834691011306896293850566130545661E
:100D300095B5B7B5000037B50000A28613068962E5
:100D40009385454913058572A5B7EFF26FCA6D719A
:100D50009307E0025C861C215A2103448502BD8B67
:100D600093E707F9230CF1041C31231DE104A308C8
:100D70000100A30CF1045C4113D70701E183A30E2A
:100D8000F104230EE104994719C8228693058500D2
:100D90001305E105EF80F03B19049377F40F680029
:100DA000BECAEF10806F51616FF0CFC6EFF24FC433
:100DB0002A8437C5000013054586EF80D0600C20DB
:100DC00037C5000013050588EF80F05F0C3037C58C
:100DD000000013054589EF80105F4C4037C50000C7
:100DE0001305C58AEF80305E0C4437C5000013053B
:100DF000458CEF80505D6FF0EFC1EFF26FBF2A843A
:100E000037C500001305C58DEF80F05B0C2037C59A
:100E100000001305858FEF80105B8305140037C534
:100E2000000013058590EF80105A4C4037C5000034
:100E300013058591EF8030590346840237C50000C1
:100E4000930584001305C592EFF0AFD937E5000094
:100E500013058599EF8030576FF0CFBBEFF24FB994
:100E60008347C504930600085D7113F7070F6312EB
:100E7000D70A858B230CF1008347D5040357E5047B
:100E8000A30CF10083570505C207D98F38453ECE24
:100E9000994763F9E7008357450503572505C207BE
:100EA000D98F3ED028081937B70500209385C5385B
:100EB0008347910103C745048583F98FA1CBF2468F
:100EC000930700021306000293854502681036D48A
:100ED00036C62302E1022306F104EF80902783D770
:100EE0006197B24637C60000B7B5000037C50000AD
:100EF00013064682938505661305C582A302F10297
:100F0000EF80704C481091354810C53D61616FF01D
:100F10006FB093060009E31BD7FEBD8B2302F102DD
:100F20008347D5040357E50413060002A302F10228
:100F300083570505C207D98F3ED43C452147E917A1
:100F400093F7F70F6363F7002146930525056810B3
:100F50002306C104EF80F01F45BF03070500930778
:100F6000D00205486314F70005057D5881472546E2
:100F7000A94829A0B38717030505B69703070500FD
:100F8000930607FD93F5F60FE376B6FE9306E002AF
:100F90006314D7041306150085461D050147254334
:100FA000A94883050600938505FD13FEF50F6378B8
:100FB000C30337460F001306F623A9456343D60241
:100FC0003307B702B386B602D5BF3307170305064A
:100FD0002E97B3861603F1B785460147D9BFE316AE
:100FE000A6FEB7460F0093860624B387D702BA97AA
:100FF000338507038280EFF20F9E6D71AA84AE895C
:10100000328981451306401068003684EFF04FA105
:1010100083C7040283C584061307A105230CF104CA
:10102000B707002083C7073BB335B0008505B3E59C
:1010300035014C86A30CF104A2863C004A86930538
:10104000000213850404EF1060772247B7C900003F
:1010500037B9000037C50000A286138649F893050A
:101060000966130585F9EF801036224493858406BE
:1010700013061004090413051101A2CAEF80700DB4
:1010800037C500002286AC08130505FCEFF06FB5EC
:101090006800EF10804037C50000138649F89305BB
:1010A0000966130505FDEF80103251616FF0EF9571
:1010B000EFF20F946D7115E137C60000B7B500006F
:1010C00037C50000130646F893854549130585FF8B
:1010D000EF80702F51616FF0EF938327050B2A8902
:1010E00091EF37C60000B7B5000037C50000130602
:1010F00046F89385454913050501D9BFAE84990586
:101100002E852EC6EF8030649C40D8301374F50FC6
:101110003EC8DC20B2450D8B130614008A07D98F18
:101120001376F60F13055101230AF100EF807002C8
:101130009306640093F6F60F1008A1454A85653DB5
:1011400051BFEFF2EF8AC0219C411171AA8422861F
:10115000950548003EC0EF80C07F930644000A8694
:1011600093F6F60F91452685793511616FF08F8AD8
:10117000EFF26F8680211171AE8922862A8985055A
:10118000130511004080EF80C07C03C6290493073B
:10119000140093F7F70F93042400180293F4F40F4C
:1011A000BA9705C603C7190493853904330591001E
:1011B0002380E7F0EF80E0790A86A6869305000297
:1011C0004A85153D11616FF04F847D572380E7F00C
:1011D000EF80A0031C02BE9493073400180293F71B
:1011E000F70F2380A4F0BA97135785002380E7F008
:1011F00093074400180293F7F70FBA97930464001B
:101200001357050115042380E7F01374F40F1C0233
:101210003E94618193F4F40F2300A4F071BFEFE2D8
:101220003FFD2A8437C50000130505BBEF80B019C8
:101230000C4037C500001305C5BBEF80D0184C200B
:1012400037C50000130505BDEF80F01737C5000056
:10125000130505BEEF803017503037C500009305E9
:1012600064001305C5BEEFF0CF976FE0BFFAEFE261
:101270003FF82A8437C50000130545BFEF80B0143E
:101280000C4037C50000130505C0EF80D01337C5EB
:101290000000130505BEEF801013502037C5000075
:1012A000930554001305C5BEEFF0AF936FE09FF6B2
:1012B000EFE21FF4902111712A84FD578505130573
:1012C0009100A304F104508423050104EF806068B9
:1012D0002C002285713D11616FE0DFF3EFE2BFEF7B
:1012E00031712A842E89EF70507285477C842AC21E
:1012F000230501009307000203070400630DF704B0
:101300002285EF80504491479304A10063F0A70227
:10131000030724009307C007631AF700A2852685F8
:101320000D46EF8000630D049304D100B7C50000A3
:10133000938545C42285EFE03FF905E1B707EFBE8D
:1013400037E700E0938707083CC74C004A858D3398
:1013500029616FE09FEB050445B7B7C50000938591
:10136000C5C42285EFE05FF601ED0545EFF02FA63D
:10137000B7C50000938545C52685EF80D03BF1B702
:10138000B7C50000938585C62285EFE0FFF309ED20
:101390008145130640031385C194EFE07FE8B7C58C
:1013A0000000938545C7C9BFB7E5000093858596C2
:1013B0002285EFE07FF10DE1B7C6000037C60000DF
:1013C000B7C50000938686C8130646C9938505CB2A
:1013D0002685EF80103095BFB7C50000938505CCFA
:1013E0002285EFE07FEE11E5B7C50000938585CC3F
:1013F00061B7B7C50000938585CD2285EFE0DFECAE
:1014000015E5EF10006703C60198938501989431A4
:10141000B821FC3103C8650083D84500B7C500007A
:10142000938585CF2685EF80D02A05B7B7C5000004
:10143000938505CE2285EFE03FE921E513055400B1
:10144000EF80C0482A84EF70505C63778502228564
:10145000EF705061EF10E06103C601989385019829
:101460009431B821FC3103C8650083D84500B7C565
:101470000000938585CE7DB7B7C50000938585D1E3
:10148000E5BDB7C500009385C5D32285EFE0DFE356
:1014900011EDEF70905792476375F50013851700B3
:1014A00045BFB7C50000938585D4F9B5B7C5000021
:1014B000938585D62285EFE03FE115E19305940001
:1014C000414613850176EF803029B7C500001386A9
:1014D0000176938545D72685EF80B01FBDB5B7C58A
:1014E0000000938585D82285EFE01FDE631905147F
:1014F0001104B7C500003946938505D92285EF80D0
:10150000004301E913860177B7C50000938505DA2A
:10151000D9B7B7C500001146938585DA2285EF80DB
:10152000004111E5370600201306163DF1BFB7C58F
:1015300000001946938505DB2285EF80403F15E1C9
:10154000B71700209387C73883C747DE91E737C6B0
:101550000000130606C14DBF37C600001306C6C003
:1015600065B7B7C500000D46938585DB2285EF8002
:10157000003C11E9B707002003A6473FB7C50000AC
:101580009385C5DB89BFB7C500000D46938545DC53
:101590002285EF80C03911E5B707002003A6873FF9
:1015A000F1BFB7C500002946938585DC2285EF8011
:1015B00000380DE5B7C50000938545DD2685EF8031
:1015C00090173705002093066004138624009305C6
:1015D00000021305053BEFE09FEC85BBB7C500009B
:1015E0001146938585DD2285EF80603409E9B707D0
:1015F000002003C5073DEF5010742A8631B7B7C5E8
:1016000000003946938505DE2285EF80403215E1E2
:10161000B71700209387C73803D667DEB7C5000029
:101620009307803EB376F602938505DF3356F602C4
:1016300045B3B7C500002286938585DF69BDB7C570
:101640000000938505E02285EFE01FC863140516AE
:1016500093094400B7C500004146938585E04E8557
:10166000EF80E02C21E95104B7C5000009469385BD
:10167000C5C02285EF80A02B09EDB7170020938706
:10168000C7380547A382E7DEB7C500009385C5E1EB
:10169000E5B1B7C500000D46938505C12285EF80F1
:1016A0000029E31405CAB71700209387C738A3821F
:1016B00007DED9BFB7C500003D46938505E24E85DC
:1016C000EF80E02609E9414693053401138501774F
:1016D000EF80900855BFB7C500001546938505E318
:1016E0004E85EF80C02411E9370500201306000263
:1016F000930594001305153DE1BFB7C500001D46D5
:10170000938585E34E85EF80802239E92D04B7C5A6
:1017100000000D46938505C12285B7190020EF8092
:1017200000219389C93801E9238209DEB7C5000089
:101730009385C5C291B1B7C5000009469385C5C060
:101740002285EF80C01E09E985472382F9DEB7C5EF
:101750000000938545C10DB183C749DEEDFBF9B7A4
:10176000B7C500001146938505E44E85EF80201C27
:1017700011E913058400EFF04FFEB707002023AAFC
:10178000A73E19B7B7C500001146938585E44E857D
:10179000EF80E01911E913058400EFF00FFCB707A3
:1017A000002023ACA73ECDB5B7C500004E8693857B
:1017B00005E515B3B7C50000938545E62285EFE042
:1017C000BFB005E11386C194B7C500008328460267
:1017D000032806025C4E184E5446938545E7104692
:1017E00091B1B7C50000938545EC2285EFE0DFADF0
:1017F0001DE51386C1948316A6021147032806032C
:1018000033C7E6021C4A8316660003164600B7C5B6
:101810000000938505ED2685EF80A06B3DB6B7C52A
:101820000000938585F22285EFE01FAA0DE9EF7095
:10183000D01D83A7C1811384C1941D8D48C823285E
:101840000400EF5030193E201A345448B7C5000048
:101850002A86938545F32685EF80A067FDB4B7C53A
:101860000000938545F709BEEFE2FF962A8437C54D
:1018700000002171130505B3EF80E0348345940B1C
:1018800037C50000130505BDEF80E0330C2037C5D8
:101890000000130545B4EF8000330C3037C500005D
:1018A000130505B6EF8020322E2037C50000130542
:1018B00085B7EF8040314C2037C50000130505A2E5
:1018C000EF806030502037C50000930554001305A9
:1018D00045BAEFE01FB137E5000013058599EF80A9
:1018E000802E8347940B130700026394E70844306B
:1018F000930700042304910C63F3970237C600009A
:10190000B7B5000037C50000130646F89385454972
:10191000130545A3EF80202B39616FE01F8F2686CA
:10192000930564001305910CEF80A00293852400B9
:101930008504502093F4F40FA294DC3093F5F50F56
:101940000D8E95051376F60FA2951305B110A3041D
:10195000F1102305C110EF70D07F8327440C9C2326
:10196000898BDDFB8325040C0325C40BEFF05F940A
:1019700065B7639C072078205C309305A40022079C
:101980005D8F7C3013052101C2075D8F1C24E207A7
:10199000D98F0327C40B3EC62326F70A50201C34D8
:1019A0006D161376F60F2308F100A308C100EF703F
:1019B000507A6800EFF0BF868327440C9C23898B04
:1019C00099E78325040C0325C40BEFF07F8E834732
:1019D00001018549638C37170D47E39FE7F2B24752
:1019E0000327C40B13097006BEC52326F70A930705
:1019F00020102316F10C2307210DEF50E07A8347C6
:101A0000C10C9803935685403E97A306D7F01387E1
:101A1000170094031377F70F3697A306A7F01387E1
:101A200027001377F70F3697A30637F11387370090
:101A30001377F70F369793054007A306B7F083D6C1
:101A4000C19429479003B3D6E60213874700137762
:101A5000F70F3297AA841396060141862186A306C2
:101A6000C7F01387570090031377F70F3297A30639
:101A7000D7F0138767001377F70FB28632970946BE
:101A8000A306C7F0138777001377F70F3697A306DF
:101A9000B7F0138787001377F70F36979D46A30695
:101AA000D7F01387A700938697008C031377F70F5F
:101AB00093F6F60FAE962306E10C930550FBA38632
:101AC000B6F08326C40B83C6B60AA5C69403369720
:101AD000A306C7F01387B7001377F70F3697A3064F
:101AE00027F11387C7001377F70F3697ED46A30644
:101AF000D7F01387E700B5071377F70F940393F731
:101B0000F70F2306E10CB697F946A386D7F0B7077F
:101B100000209387C738B40115073697F057B45B98
:101B2000AC570545EF50E06E8347C10CAD07230667
:101B3000F10C0325C40BAC01EFF0AFE037C500009A
:101B4000A685130505A5EF800008F9B3EF70E06BDB
:101B5000AAC5EF70806B83A7C1811387C1941D8DC7
:101B600048CB130640039385C1941305D10C232859
:101B70000700EF70105E0325C40B93074003AC0110
:101B80002306F10CEFF0EFDB41BB1147639DE70249
:101B900078205C30502022075D8F7C3071161376E0
:101BA000F60FC2075D8F1C24930594001305D10C1A
:101BB000E207D98FBEC52306C10CEF709059A8016A
:101BC000EFF0EFEA91BB2147E398E7D478205C304F
:101BD0008324C40B22075D8F7C309305A40013057A
:101BE000E10CC2075D8F1C24E207D98FBEC523A676
:101BF000F40A1C34502013F737006D16898323062E
:101C0000F10CA306E10CEF70D0548327440C9C2305
:101C1000898B91E78325040C2685EFF06FE98346D5
:101C2000C10C85476383F6049DC28947638AF60425
:101C300037C60000B7B5000037C50000130646F8E8
:101C4000938545491305C5B0EF70F077F1B1AE4605
:101C50000346D10C8325C40B37C500001307E10CE4
:101C6000130545A8EF70307645B98325C40B83C7AB
:101C7000B50AE38307CA1305E10CEFF02FE669B953
:101C80008357E10C68007C868357010D7C87EF50F9
:101C9000C0632E478346D10C8325C40B2A8637C5E3
:101CA00000009307210D1305C5ABEF70D071ADB1E6
:101CB000EFE26FD255712A841306C00B814568008C
:101CC000EFE00FD6930754007844BEC51C203AC4F9
:101CD0003707002093F7C703A300F10C0347073B26
:101CE0008347C404A2C78346D4046312F70437C9E8
:101CF0000000B7B9000037C50000130649F8938506
:101D0000C94E13058593EF70106C8884EF506058AE
:101D1000AAC3AA8405E1B7B5000037C500001306C1
:101D200049F8938545491305C596EF70D0696961F7
:101D30006FE0AFCDEF70604DB70700209387075D70
:101D4000B387F440B736BDE98D879386767AB3863C
:101D5000D70223A8A40A37C50000130649F89385C3
:101D6000C94E13058598EF70106634441307D100EF
:101D70001306E404F9169305000213850404EF002A
:101D8000902D05CDB7B5000037C50000A686130617
:101D900049F8938545491305C59AEF70D06283458C
:101DA000110C37C500001305C5A0EF70D0611C866B
:101DB000BDDF2800EFF05FAB9DBF384437C50000A2
:101DC000130649F879171377F70F9385C94EA6863E
:101DD0001305C59D5886EF70105F13052101EF8034
:101DE0008016930555001386040293F5F50F13052D
:101DF000D100EFE0AFEF65B7EFE2EFBD457103490A
:101E00001500AA84EF706040130780033307E902CE
:101E1000D547370400202306F10C9307C438938577
:101E200094002ACCAA892E852EC6BA9783C7470B61
:101E3000A308010C230E0100230CF110EF80A01069
:101E4000130755009307400B1304C438B24593049D
:101E5000F00A63E3E700AA8426861305D101EF7038
:101E6000502F950437C5000026862C081305450D14
:101E7000EFE02FD7930780033309F902130791117D
:101E800030085C08A686C14502CA1305490A229596
:101E9000EF00D012D2474A94E8018507232C340B77
:101EA000232AF110DD2B79616FE02FB6EFE24FB4FA
:101EB00055712E84B7050020AA849385153D13051E
:101EC0001101EF804007B7C5000093850582130517
:101ED0001101EF806004A68513051101EF80C00396
:101EE0002800C084113F69616FE0CFB2EFE2AFAE6E
:101EF00009712A841306800C81452819EFE04FB23E
:101F00001C20514793F7C7036383E70237C60000DD
:101F1000B7B5000037C50000130646039385454951
:101F200013054504EF70304A19616FE00FAE834727
:101F3000C4048144130BD404230CF10AB7CA000073
:101F400037BA0000B7C900000345810BA685EF50E2
:101F5000803B2A8915E18346810B37C60000B7B55F
:101F6000000037C500001306460393854549130555
:101F70000506EF7050454DBF34440A875A86FD165A
:101F8000C14513050502EF00100D19CD8346810BE5
:101F900013864A0393054A49138589088504EF701F
:101FA000904293F4F40F4DB78247304493055100AB
:101FB0003EDF7D161C821376F60F6D161305110C8D
:101FC0002300F10CEF70F018EF702024232AA902EF
:101FD00037C500001306110CCA851305450BEF70B9
:101FE000903E99B7EFE2CFA02A84412C1420B7C4C9
:101FF000000093F7060C91CFB7B5000037C500007D
:1020000099821386040E938545491305C50EEF701A
:10201000903B9386C194904618209387C1941305F2
:10202000160088C6937627009375C703CDE69453B0
:10203000850694D3F1466393D5022285EFE01FAA6B
:10204000B7B5000037C500001386040E93850566FA
:1020500013058513EF7030376FE0CF9B93060002B6
:102060006388D5001377870301C72147639CE50088
:1020700037C5000013054512EF70F0342285EFF0EC
:102080003FC37DBF3147E38DE5FA41476396E500E5
:102090002285EFE06FF56DB71387C5FE1377870FC5
:1020A00001E72285A13569BF1387C5FD1377870F27
:1020B00041DB1307C002639AE5005C3081E72285AB
:1020C000EFE0DFD9FD571CA0A5BF1307C003E389CC
:1020D000E5F690C7B5B7D4538506D4D3A1BFEFE2D8
:1020E000AF8E4111AA842E843289B689EF60806C4C
:1020F0000989630205181305F03FEF60A03413054A
:10210000B1009305A10023050100A3050100EF60C4
:10211000406C9C850145638107104E86CA852285E7
:10212000EF60E03C1306401081452685EFE04F8FBD
:10213000B7C5000005650546938545291305853813
:10214000EF503028F9475C861C8537150140014661
:10215000C14513050580B16ADC86230701000149EA
:10216000EF6010560144014A814C8149114C938A19
:102170004A15130B00041C08CA9703CDC7FF8D4BEB
:1021800031A08947130DF00FE3F727FF8945373555
:102190000140EF70001E7DD9EA8537350140EF70B0
:1021A000C01C854537350140EF70A01C7DD93735FF
:1021B0000140EF70C01B894763F327031375F50FC8
:1021C000636F8C0093172400D6979C43828788A066
:1021D0000D890544630575013334A00005049C8511
:1021E00005094209135909018D07E36CF9F8371500
:1021F00001400546C1451305058023A43405EF6061
:10220000304CB7C50000056501469385852A130546
:102210008538EF50101B888541016FD07FFE9307F2
:102220001A00269AA300AA0013FAF70FE3F94BFB52
:10223000094475B7C8B06377AB00A38264010D444D
:10224000814C71BF814C65FD114451BF13871C0047
:10225000A69C2383AC00DC30937CF70FE3E1FCF811
:10226000E5B793871900A6992386A90493990701D6
:1022700093D90901ADB7014545B7EFD27FF71C21CE
:10228000094741118D8B2A84638BE70A0D47638DC3
:10229000E70A05476380E70A37C500001305852B69
:1022A000EF70701237C500001305C52EEF70B01126
:1022B0001C20614793F7C7036389E7126369F70A34
:1022C00021476385E7106366F708EDC71147638A06
:1022D000E70E1C2037C500006C0099839387070325
:1022E000130545385C86A3060100EF70D00D1C2055
:1022F0000D478D8B6383E70099EB035634008355BC
:10230000140037C500001305053AEF70D00B4C30B0
:1023100037C500001305853BEF70F00A814437C9CB
:1023200000005C3063ECF40E2945EF70F00D4101C4
:102330006FD05FEE37C500001305852C95B737C504
:1023400000001305052DA9BF37C500001305852D15
:1023500081BF41476381E70851476383E7083147FD
:10236000E399E7F637C500001305453281A8130746
:1023700040026386E708636EF7007147638CE706E7
:1023800013070002E397E7F437C500001305C535CE
:1023900035A01307C0026389E7061307C003638AE9
:1023A000E70613078002E396E7F237C5000013053E
:1023B000C53629A037C5000013050530EF70B00001
:1023C00009BF37C5000013058530CDBF37C50000F4
:1023D00013054531E5B737C500001305C5C4F9BF7E
:1023E00037C5000013054533D1BF37C500001305BD
:1023F0000534E9B737C500001305C534C1B737C583
:102400000000130545365DBF37C50000130585374D
:1024100075B737C50000130505384DB7B3079400ED
:10242000F023A6851305093D8504EF70C07993F468
:10243000F40FC5BDEFD2DFDB59712A842800AE84CA
:10244000EF40D02330449305C4042800EF40902986
:102450002800A685EF40903B65616FD0BFDBEFD2CF
:102460003FD913848181042093071002B387F402BB
:1024700093844184BE94A685753F85472380F402EA
:102480001C201D47850793F7F70F6365F7001CA015
:102490006FD05FD823000400E5BFEFD27FD20111D7
:1024A000AA84753F9C200D4719448D8B6384E700F7
:1024B00091C30944D830BC44BA973E944204418049
:1024C0009307F00F63F1870237C60000B7C500001D
:1024D00037C50000A2861306C61793858518130515
:1024E000C518EF70406E8387F182639507128547A8
:1024F000A387F18293878182B82311E3A0B31946A1
:10250000938581821305C008EF5090271305F03F93
:10251000EF505073B7C50000056505469385051B50
:1025200013058538EF50E06937150140B94701467A
:10253000C14513050580FC86EF60901893072400C1
:10254000316C8149814A0149014D814B014A3EC4A8
:10255000914D130C8C168D4CA24763C5F90C3715A1
:1025600001400546C14513050580EF60701585697A
:10257000B7C5000001469385451C13858938EF5087
:10258000406403C80400D830B44437C90000B7B46D
:10259000000037C50000A2871306C917938504669B
:1025A0001305451DEF70206237C500002287D286D3
:1025B0001306C9179385046613058521EF70A06083
:1025C000138589BBEF60800D37C500001306C9175E
:1025D0009385046613058524EF70E05EEF60801D2F
:1025E0002A8437CA000093771420638B070E37C5FF
:1025F00000001306C917938504661305C527EF70FD
:10260000805C370500017D150588A3870182EF50A6
:10261000F07311E483A70183850723A8F182056184
:102620006FD0DFBD854763E437051C103387370162
:102630000347C7FF8945373501403AC6EF607053FD
:1026400032476DD9BA8537350140050AEF60F05140
:10265000854537350140EF60D0517DD98509373543
:102660000140C209EF60B05093D90901F5B51307D5
:10267000F00FE3E1ADFD13172D00629718430287B9
:1026800098209377370063849701094D91E3054DB6
:10269000014A4DB793861A00A69A03C71A0093FA07
:1026A000F60FE3F95CF9094D71B7D83001490D4DCA
:1026B00051F3114D41B7D430130619002699034741
:1026C00069001379F60FE367D9F6E5B793861B0027
:1026D000A69B03C7CB04939B060193DB0B0199BF19
:1026E0002945EF605058EF60E00C8387E1822A842F
:1026F000E38B07EEAA861306C917938504661305B4
:102700004A26EF70404CC5B5EFD2FFAC01118A8567
:102710002A84EFF03FD283C48181930710022149BC
:10272000B387F40293844184BE9483C9040263890D
:102730000900130600028A852685EF70401F05C137
:102740007D191379F90FE31409FE1C2013F7170004
:102750001DCB1307F00F6397E70044308DE8056148
:102760006FD0BFAA5C301307E003636EF7001387D6
:10277000170058B0370700200347073BA297228570
:10278000F8A3EFF09FD11C208D8BF1DBF9B7B707D1
:102790000020782083C7073BE313F7FCFD1493F474
:1027A000F40F44B026869305740013056400EF709F
:1027B0006025D5D42285EFF05FCE55B7D9CA5D71BB
:1027C000A6C29384F60086C6A2C4CAC080084EDEA4
:1027D00052DC56DA5AD85ED6C198330191402A8A23
:1027E000B28B2E8B268681450A85BE8A3A89B689A8
:1027F000EFD01FA34E86DE850A85EF708015930902
:1028000029004E87A6860A86C1455285EF400003FF
:10281000130704FBA6864E86DA855285EF402040DA
:10282000834704FB890401452300F900834714FB17
:10283000A300F90023A09A00130104FBB64026442C
:1028400096440649F259625AD25A425BB25B6161C0
:1028500082807D55828009486376D804EFD2BF9785
:102860001384E6FF9376F4000111130A260089C64B
:10287000795505616FD07F99B284BA8952860A87EB
:10288000A2862A89EF40A03909468A852685EF70FD
:10289000000A79FD4E87A2865286C1454A85EF30EF
:1028A000307EC1BF7D558280EFD29F94411102C41A
:1028B000CD475C84280085473EC6EF6060614101DA
:1028C0006FD05F959377350099EF13074006337704
:1028D000E502854719E7930700193375F502933729
:1028E00015003E8582808147EDBF1308E5844208CC
:1028F000135808019308100863E5080DEFD25F8CA8
:10290000373CE101B78CE2013E8B3A84B68A3289CA
:10291000AE89AA8B8144130A207B130C0C38938C4C
:102920000C5063964B07FD19B16C556C014A93F935
:10293000F90F938C4C3E130C0C18854D131D0A0196
:10294000135D0D0163603D071307C0038566330403
:10295000E402938606E15566130606187D1985453F
:1029600037050018B38ADA025A943309C90256941B
:10297000EF60C07C0545EF60605B4A942694228539
:10298000EF60500EEF60B01301456FD03F87528566
:10299000153F19C5E694050A420A135A0A0151B7B0
:1029A000E294D5BFB3874C019C235E85B387870330
:1029B000BE94EFF03FF101C56313BD01E294050A37
:1029C000B5BF05458280EFD2BF82B1679387073FCD
:1029D00081459306A004130650071305E00631470E
:1029E0000388070085056318D8020388170063145D
:1029F000C802038827006310A80293F5F50F930718
:102A0000800313078002D94665461305A07EEFF0C8
:102A1000DFED6FD03F8093F5F50F8D07E392E5FC76
:102A20008145F1BF13074006B377E5023355E50250
:102A30004D471375F50F6374A7009387470613D5A9
:102A400027003E951D473375E5023167130787411F
:102A50002E970347F7FF8D8B3A962A9699E7894779
:102A600063E5B7007D16420641821D453375A60217
:102A70008280EFD26FF55564EF602079130404185B
:102A800033548502938701829A23AA8463058704BD
:102A900082A39309207B1309C016130AD016636022
:102AA000890893870198B16A2392370113890198A5
:102AB00081496D4B938A4A3E854B714C138A1900AC
:102AC000636F8B06137AFA0F05042303490113740D
:102AD000F40FA3038900D56793870718B3F4F402B2
:102AE0008567938707E11384019833D7F402B3F421
:102AF000F4021377F70F18A01307C003B3D7E4024B
:102B0000B3F4E40293F7F70F1CB024A04A206C2022
:102B10007030EFF03FF108A401456FD06FEE4E85A5
:102B2000EFF05FDA11C9E30E44F7130424E98509D5
:102B3000C20993D90901A5B7130434E9CDBF0355E0
:102B40004900EFF03FD819C9639A7901E30C84F783
:102B50000D1493190A0193D909018DB7D69983C72A
:102B60000900E361F4F61D8CEDB7EFD26FE88545FF
:102B700037050018EF60805C0545EF60203B094594
:102B8000EF6060780545EF600078EF6060230545F1
:102B9000EF60403C01449304A00F13051004EF6064
:102BA000A05F09ED6315940005456FD0AFE60504FD
:102BB00051451374F40FEF60100BC5B79307A00FC6
:102BC0000545E304F4FE13050010EF60203B0545C6
:102BD000EF60803BEF60A06EEF60606F8145054560
:102BE000EF60605E81450945EF60E05D814511451C
:102BF000EF60605DEF60A06CEF60805E21657D1529
:102C0000EF600069EF60A06BEFF0FFDBEF60605EEC
:102C1000A9659385151A1145EF60801BEFF0DFC899
:102C2000EFF03FE5014551B781466393C6008280CE
:102C30009C21983183C82500E2074207D98FA2085A
:102C4000B3E7170183C84500F83103C33500E20834
:102C50003367170183C85500139836002A98C208B5
:102C60003367170183C86500B3E767002322F800C4
:102C7000A208336717012320E8008506A10575B770
:102C80001C411971A2DE3EC25C41A6DCCADA3ED408
:102C90001C45D2D6E6CC3EC45C45EEC8CED83ED666
:102CA0001C49D6D4DAD23EC65C49DED0E2CE3ED84C
:102CB0001C4DEACAB1633EC85C4D130905043EDAF7
:102CC0001C513ECA5C513EDC1C55E256C24D3ECC06
:102CD0005C55624F525A3EDE1C59F254B2483ECE09
:102CE0005C59F24EC25FBEC01C5D064422433ED01A
:102CF0005C5D025EB252BEC2938783423EC09307C0
:102D00000504BEC69307050CBEC4964CD2471247B5
:102D100022569383834283AA030083250900032854
:102D2000490083A94300D695B3BA5501C299CE9AFA
:102D3000139B260193D9E700336C3B0113D8E600BF
:102D400093992701B3EB0901139BE60093D927015F
:102D500033683B0113DB26019399E700B3E969016E
:102D6000B3C93B01334B0C0193DB970013987601F9
:102D7000B3EB0B01139C770113D8960033688801DD
:102D8000334B0B01B3C979012E9BB335BB00CE9AEF
:102D900093CBF7FFAE9A93C9F6FFB3F5E701B3FB08
:102DA000DB0133F89600B3CBBB00B3F98900DA9BA3
:102DB000B3C90901D69933BB6B015E9E4E9BB33BF1
:102DC0007E01DA9C9315E601935A26001318E70159
:102DD00093592700DE9CB3E9B900B3EB0A019315C0
:102DE00046001358C701B3E50501935AC6011318ED
:102DF00047003368580133C80901B3CABB0093596F
:102E0000770093159601B3E9B900131B9701935509
:102E10007600B3E56501334B1301B3C5BA00B3497E
:102E20003801337BEB00B3CAF20133781301B3FBF3
:102E3000F20133480B01B3FACA00B3CA7A012E98E3
:102E4000B335B800CE9AB38B5501330CBE017298DE
:102E5000669A333BCC01DE9C333EC801B3059E012C
:102E60002ED22E8DA645529B2109E289DA8AC28B89
:102E7000A103C68D7E8A768EA28C639B2537024B7A
:102E8000B643F68C228CFA8E26843E8FB68446D2C8
:102E9000FEC49A88968F3A83B282CE87D6865E87A2
:102EA0006A86795A9375FA00A1058E05AA9503A939
:102EB0000500CC41A10313583901939BD500B3EB16
:102EC0000B01931AD90013D83501B3EA0A019359BB
:102ED000D90113983500131E3900B3E9090113D83D
:102EE000D5013368C801B3C93A0113596900939AEF
:102EF000A50133C80B0133E92A013349280103A88E
:102F000083FF03AEC3FF99814A98B3C9B90033392F
:102F10002801F299330E390113093AFF1379F900A8
:102F200021090E0923AC03FF23AEC3FF2A9983298D
:102F3000490083250900210B139DF90113D91500C0
:102F4000336D2D01939BF50113D91900B3EB2B01C0
:102F5000939A890113D9850093DD8900B3EA2A0188
:102F6000139985013369B90133C92B019D81939B65
:102F70009901B3E5BB00B34A5D01B3CABA0093D966
:102F800079009305BAFF569833493901BD89729982
:102F9000B33A5801A105CA9A8E0523AC03FF23AEAC
:102FA00053FFAA9503A90500CC41939927014299A3
:102FB000AE9A33380901569893D5E700939A2601C3
:102FC00013DEE60033EDBA00B3EBC90193D5270158
:102FD0009399E70093DA2601139EE600336EBE0054
:102FE000B3E55901B3C9BB00B34ACD0193D59700EE
:102FF000139E7601B3E5C501939B770113DE96001E
:1030000013CDF7FFB3C5B900336E7E01337DDD010B
:1030100093CBF6FFB3F9E70133CECA01B3FB8B00C4
:10302000B3493D01B3FA960023AC23FF23AE03FF5F
:10303000F299B3CA5B01AE9A33BEC901832D8B07E7
:10304000569E832ACB07CE9DB3B93D01569E6E99FD
:10305000F299C299B33DB901CE9D9355C701931919
:103060004600B3EBB9001358C60193154700B3EA05
:103070000501135E26001318E601131DE7019355A1
:103080002700B369AE01B3E50501135E770013189D
:103090009601B3C5BA00336E0E01931A9701135807
:1030A0007600CA9CB3C93B0133685801B34A130187
:1030B00033B92C0133C8090133CEC501E29DB3FAFF
:1030C000EA00B3C9F201B3751301330CB901B3C5FA
:1030D000BA0033F9F201B3F9C900B3C92901C295A5
:1030E00033B80501F299330938011258E695050AFB
:1030F000338E0C012648B33D9E01B3BC9501629806
:103100004A9CC29D46D233888C01FEC43949F2895B
:10311000EE8AAE8B428DF68C228C63182A0F824386
:10312000938303081EC00249B16393838362E398CB
:1031300023D5924322599E95B3B375004A981E98A1
:103140000CC1A2452322050132582E97B335B70092
:1031500042962E9618C5324750C542563A93333799
:10316000E300B292BA924247525623286500BA98B9
:1031700033B7E800B29FBA9F52476256232A5500E0
:103180003A9E3337EE00B29DBA9D624772562322B3
:10319000B503BA9733B7E7001CD5B296F247BA9693
:1031A00006473E9FB337FF00BA94BE948257164736
:1031B00044D9BE9EB3B7FE003A943E94232C150129
:1031C000232EF5012320C50354D52328E503232C02
:1031D000D50340DD7654E6545659C659365AA65A98
:1031E000165B865B764CE64C564DC64D0961828077
:1031F000FA8E26843E8FB6849A88968F3A83B2825E
:10320000E287DA864287125639B6FA8E26843E8FD6
:10321000B6849A88968F3A83B282F287EE862E879A
:10322000428649B1EFC2DFFC0326050DE157137456
:1032300086FF1D8A3306F6022A942E8581451306E1
:103240008603EF60E02B3C405D8D7C4028C0DD8D27
:103250006CC06FC03FFCEFC21FF88329050D2A84A4
:103260002E8993F77900B28485C3B309304193F96D
:10327000790063733601B289014AB30749016314C7
:103280003A0D3E89B38444418327040D13F7F707B1
:1032900005CF3307F0401377F70793D9340063E481
:1032A000E40093593700E19B130504044E86CA8558
:1032B0003E95EFF07F978327040D8E094E99CE97A8
:1032C0002328F40CB38434410327040D930700082A
:1032D0006311F7068327840C8326C40C13870740E9
:1032E000B337F700B6972324E40C2326F40C95E3B8
:1032F0009307F03F63EFE7008327040C8326440C19
:1033000013871700B337F700B6972320E40C232266
:10331000F40C2285EFF0DF96930704042328040CB5
:103320001307040C0146814690C3D4C3A107E31BD5
:10333000F7FE93F904F8CA99130A0404930AF03FBC
:10334000130B040CADA88C232285050AEFF09FED2A
:103350008327040D85072328F40C05B74146CA8549
:103360005285EFF07F8C8327840C8326C40C13874F
:103370000740B337F700B6972324E40C2326F40C58
:1033800085E363EFEA008327040C8326440C13874C
:103390001700B337F700B6972320E40C2322F40C70
:1033A0002285EFF0FF8DD2872328040C8146014748
:1033B00094C3D8C3A107E39B67FF13090908E31F60
:1033C00039F913F9F4076305090213563900CE855C
:1033D00013050404EFF05F858327040D93F484073D
:1033E00033099940A6972328F40C014A6314490134
:1033F0006FC0BFE1B3874401CE978C232285050AB5
:10340000EFF05FE28327040D85072328F40CF9BF52
:10341000B7C7000003A7876A83A7C76A014818C116
:103420005CC1B7C7000003A7076B83A7476B18C52C
:103430005CC5B7C7000003A7876B83A7C76B18C914
:103440005CC9B7C7000003A7076C83A7476C18CDFA
:103450005CCDB7C7000003A7876C83A7C76C18D1E2
:103460005CD1B7C7000003A7076D83A7476D18D5C8
:103470005CD5B7C7000003A7876D83A7C76D18D9B0
:103480005CD9B7C7000003A7076E83A7476E18DD96
:103490005CDD81472320F50C2324F50C2322050D48
:1034A0002326050D2328050C930705041305050C99
:1034B0008146014794C3D8C3A107E39BA7FE82803E
:1034C00019C6EFC2FFD2EFF01FD96FC0BFD4828000
:1034D000EFC21FD28327050D2A84AE8481EF9307A4
:1034E00005041307050C0146814690C3D4C3A10708
:1034F000E39BE7FE930500082285EFF0BFD2032689
:10350000040D8327840C8325C40C93163600B697CC
:1035100033B7D7002E972324F40C2326E40C05E3BD
:1035200063FFD7008327040C8326440C13871700FE
:10353000B337F700B6972320E40C2322F40C93074B
:10354000F00663F0C7022285EFF08FF393070404BF
:103550001307040B0146814690C3D4C3A107E39B24
:10356000E7FE0327040C8327440C22852328E40A62
:10357000232AF40A0327840C8327C40C232CE40A8F
:10358000232EF40AEFF0CFEFA287A685138604045A
:10359000D4439843A10513D58601238CA5FE13D5EA
:1035A0000601A38CA5FEA38DD5FE13D586009356E8
:1035B0008701238ED5FE93560701A38ED5FE935621
:1035C0008700238DA5FE238FD5FEA38FE5FEA107DF
:1035D000E390C5FC9305800D2285EF20200E6FC07F
:1035E0007FC3EFC2FFC029712A84A81042C446C21B
:1035F0003AC83EC636CA2ECE32CCEFF07FE16246E4
:10360000F245A810EFF0DFEBD246A8101306000237
:10361000B685EFF05FC4B2474247A8103E86BA8530
:10362000EFF01FEA92482248A8104686C285EFF0C4
:103630003FE92C10A810EFF0BFE92C102285EF20F5
:10364000100331616FC01FBDEFC29FBA51712A8450
:1036500028082EC632C4EFF0BFDB2246B245280848
:10366000EFF01FE62808A285EFF09FE66D616FC0BE
:103670007FBAEFC25FB63571B2842A8413060002A6
:1036800088103689BA893E8AAE8AEFF0FFFB8C102B
:103690002E85EF20207881480148D2874E8714017B
:1036A0004A86A6850A85EFF0DFF38A858800EF2039
:1036B000902E9307000213870A02D2884E88940046
:1036C0004A86A6850810EFF0DFF181471307000254
:1036D00090003E961022B306F400850790A2E3996D
:1036E000E7FE8A8690100C1013050402EF20A07AE2
:1036F000881093050004EF10707C0A859305000282
:10370000EF10D07B0D616FC05FB0EFC27FAE39713B
:103710002A84AE84814713070002B305F6008C218A
:10372000B306F10085078CA2E399E7FE930500023A
:103730003285EF10B0788147130700023306F1009D
:103740001022B306F400850790A2E399E7FE130662
:1037500000028A850A85EFF03FEF8A850A85EF200F
:10376000606B8A852685EF201023814713070002AE
:10377000B386F4009022B306F40085072380C602C6
:10378000E398E7FE0A8593050004EF10307321618A
:103790006FC05FA8EFC2DFA5B687328781460146BA
:1037A000EFF03FED6FC01FA7EFC29FA401112A8465
:1037B000B6873287AE86AE8481480148AA85130653
:1037C00000020A85EFF0FFE10A86A6852285EF2038
:1037D000F00005616FC01FA41C3138210821A20729
:1037E0004207D98F5D8D82801C311821A2075D8F21
:1037F0003C212831C207D98F62055D8D8280EFC2DE
:103800003F9FAA84EFF05FFE2A8413854400EFF007
:10381000BFFDAA8522856FC0FF9F93D785000CA1AD
:103820001CB193D70501E1813CA12CB18280EFC28C
:103830003F9C41112A899314260001443385850059
:103840002EC6EFF07FFAB307890088C31104B24592
:10385000E31694FE41016FC0FF9BEFC2DF972A89F8
:10386000AE89931426000144B38789008C43330545
:1038700089001104EFF07FFAE31894FE6FC0FF98FF
:10388000EFC27F952E8AAA84EFF07FF72A895285AE
:103890002E84EFF0DFF63349A900138584002D8CC8
:1038A000EFF0FFF5AA8913058A00AE84EFF03FF52B
:1038B00033C5A900A58D33652501C18D6FC0FF9467
:1038C000EFC27F912A89AE89EFF09FFB2E84AA84F4
:1038D0009385090113050901EFF09FFA458DC18D0C
:1038E0006FC0BF9293078502232005001105E31DD9
:1038F000F5FE828085471CC19307450013058502AC
:1039000023A007009107E39DA7FE8280814713074C
:103910008002B386F5009042B306F500910790C28D
:10392000E399E7FE82808147930680023387F500A2
:1039300018433306F50091073307E04018C2E397B8
:10394000D7FE82808147930680023387F500B30853
:10395000F600184383A808003308F500910746973E
:103960002320E800E393D7FE8280814793068002FC
:103970003387F500B308F600184383A8080033081E
:10398000F5009107330717412320E800E392D7FEA3
:10399000828041113306C04018419C4132C6B24674
:1039A000B98FF58F3D8F18C19841B246B98F9CC130
:1039B0005841DC41B98FF58F3D8F58C1D841B2468F
:1039C000B98FDCC118459C45B98FF58F3D8F18C55F
:1039D0009845B246B98F9CC55845DC45B98FF58FDF
:1039E0003D8F58C5D845B246B98FDCC518499C49AA
:1039F000B98FF58F3D8F18C99849B98F9CC958491F
:103A0000B246DC49B98FF58F3D8F58C9D849B246C7
:103A1000B98FDCC9184D9C4DB98FF58F3D8F18CDEE
:103A2000984DB246B98F9CCD584DDC4DB98FF58F6E
:103A30003D8F58CDD84DB246B98FDCCD18519C5131
:103A4000B98FF58F3D8F18D19851B246B98F9CD15F
:103A50005851DC51B98FF58F3D8F58D1D851B98F5E
:103A6000DCD14101828041113306C04032C69C4105
:103A70001841B246B98FF58FB98F1CC1DC4158414E
:103A8000B246B98FF58FB98F5CC19C451845B246D7
:103A9000B98FF58FB98F1CC5DC455845B246B98F33
:103AA000F58FB98F5CC518499C49B246B98FF58F1F
:103AB000B98F1CC95849DC49B246B98FF58FB98F07
:103AC0005CC9184D9C4DB246B98FF58FB98F1CCD8E
:103AD000584DDC4DB246B98FF58FB98F5CCD18517A
:103AE0009C51B246B98FF58FB98F1CD15851DC511A
:103AF000B246B98FF58FB98F5CD141018280EFC298
:103B0000AFEC4111AA842E852E8432C6EFF0DFCDB2
:103B10002A8B13054400EFF03FCC131D65001305FD
:103B20007400EFF07FCB131C55001305A400EFF0D9
:103B3000BFCA931B35001305D400EFF0FFC9931AD9
:103B4000250013050401EFF03FCAAA8C13054401B8
:103B5000EFF09FC8131A750013057401EFF0DFC76B
:103B6000931955001305A401EFF01FC71319450061
:103B70001305D401EFF05FC63246B70700013707DF
:103B80000002938EF7FFB3DECE403306EB00B33670
:103B900066019A066982558EB305CD00935366007F
:103BA000131EA6013386EA00B33656013383F500AF
:103BB0009A066982558E33BDA501B336B300330E24
:103BC000CB41EA96333BCB019E06B30370401353BF
:103BD0009301B38363419318A601135B660033E33B
:103BE000660066963308F600931693016293B3025B
:103BF000E300B33C9601B3FEAE003335C800958DAB
:103C00006695B336830133BC62001E05369C13589B
:103C10009801336805011A0C93D2A201131598017B
:103C2000B3625C005298330FE800098E33354801C7
:103C3000338A5B00B30FFA00B3360F01B33C7A014D
:103C4000AA96B3BB4F019A06E69B135FAF0133EF11
:103C5000E6019E0B93DF9F013384E901B3881A418B
:103C6000B3EFFB01333C3401B389F801B3BA1A0155
:103C7000B3B61901B3865641B3866641330BF400DF
:103C800033358B006295B388E9001E05135B9B01F9
:103C9000336B650133B53801AA96B30A69019A06F8
:103CA00093D8A801B3E81601B386EA00B3BB2A0192
:103CB00033B956015E991A09E9828A0EB366D900B2
:103CC0003389DE00CA973335D901B3BE2701AA9ED6
:103CD0009E0EE583B3E7FE00CD4E3385FE02EA0279
:103CE000E60F6A0F660BEA06330464413303534060
:103CF000330AFA414696B3BEFE022A9E72973335C6
:103D0000AE00E6073308E841B386DA40B307F9406E
:103D100023A4640023A64401F6931E95B333C70180
:103D20001E951A056983498F1315A701BA95139734
:103D3000A801330EAE40B389E94023A0C401CCC032
:103D400023A83401D0C823AC0401C0CC94D0DCD06B
:103D500041016FC0EFCA79716EC083AD050056CCCA
:103D600083A34500B30AB60394496AC266C422D647
:103D700026D44AD24ED05EC8DC51B31DB60383A907
:103D80008500C44583AB450103A98501C04D83A2CD
:103D90000502B70500023387BA005ACA330D76020E
:103DA00052CE62C6B30CD602B3137602B316D60255
:103DB00033083603B30E9602B3087603B30F260317
:103DC000330F860233035602330BF60233192603F0
:103DD000B3193603B3149602B31B76033314860269
:103DE000B31256023316F602B3375701EE97139EFD
:103DF000670069833367EE00E987135E6700139CF1
:103E0000A701131AA701336C8E016A97338A4A41BE
:103E100033BE4A01333DA701B38A8D41338CF30091
:103E2000B387BC006A9C33BD9701369DB38ACA41F3
:103E3000E983131E6D00B367FE00135DAD4193D39C
:103E40006700131EAD0133EEC3019393A701C6971C
:103E5000B3837C40B3B81701338EC641EA9BB706E3
:103E60000001B3BC7C00C69BB308D700330E9E4153
:103E7000B3BCE800669C931C7C0093D89801B3E81F
:103E80001C01939C9801135C9C41C29833B80801B3
:103E9000E299C2993388D700333DF800EA9B139C1E
:103EA0007B001358980133680C01131C980193DBB5
:103EB0009B417E98B33FF801CA9BFE9BB38FB8002D
:103EC000B387874133BC1F01E2991399690093DFDF
:103ED000AF01B36FF90113D9A941B389FE01B3BE94
:103EE000D901CA94338C9E00B30EB80033B90E01C9
:103EF0005E999314690093DEAE01B3EED401B3046E
:103F0000DF011359A94133BFE4014A94B30B8F0079
:103F1000338FD90033343F01629413197400135F57
:103F20009F01336FE9013389E30165847294B333F0
:103F30007900338ED400A29333349E005E94931B99
:103F40007400135E9E0133EECB01135C9441330485
:103F5000C30133336400E292B30B5300B302B900E0
:103F600033B322019A939A033303B40093D2A2018C
:103F7000B3E25300B3338300DE93939B6300135388
:103F8000A30133E36B0093DBA341B3036B005E96A5
:103F90009E9633BB6301329B33B676005A96131B51
:103FA0007600E582B366DB00CD4B6586338BDB02A2
:103FB00033079741EA0F660FEA0E660E6A03B3896C
:103FC000E941B384C441330464403386CB025A9A36
:103FD000333B6A01D295B388F84196973308D841AC
:103FE0002326350144CD23241501B3BBDB02E606AD
:103FF000B386D3405CC9232C050100D154D15E9611
:1040000056965A9633BB45015A961A06E981D18DC8
:104010001396A501BA951397A201330ACA40330932
:10402000E94023204501232825014CC13254A254E4
:1040300012598259724AE24A524BC24B324CA24C3C
:10404000124D824D45618280D845757122C73AC4B0
:10405000D849404A26C53AC6D84D4AC34EC13AC887
:10406000D851D2DED6DCDADADED8E2D6E6D4EAD22D
:10407000EED03ACA83A805029C4103A88500944962
:1040800003A385011842032E8600032FC600832256
:10409000060103A945004C4222CC004E131A190018
:1040A000B383E70222D4404E22D60052505222D887
:1040B00032DC22464D44B39DE70293191600324686
:1040C000060632CE4246060632D05246B38B8202F4
:1040D000060632D26246B30A86022256B30486022C
:1040E0003256B30F86024256B30E8602625633062C
:1040F0008602330BCA02331DCA021E9BB3337B00F8
:104100006E9D1E9DB303D803B31DD803DA9333BB52
:1041100063016E9D6A9B338DF903B39DF9031E9D68
:10412000B3337D006E9BDA93338B9602B39D960278
:104130006A9B333DAB01EE931E9DF243F24D330C6F
:104140008F02B3835303B39D5D03DA9333BB6301E3
:104150006E9DB30D73036A9B331D73039E9DB3B3B2
:104160007D005A9D1E9D8253025BB30C8E02B38369
:104170008303331B8B03EE93B3BDB3016A9B338D73
:1041800098036E9BB39D98031E9DB3337D006E9B79
:10419000DA93338B8502925D1EDE9253B30DBB031F
:1041A000331B7B02B303BD011EDA33BDA301F253FF
:1041B0001E9BB3036D019EC2338BB702B30327036B
:1041C000B39DB702DA9333BB6301331D27036E9DA2
:1041D0005A9D330B0603B31D06031E9BB3337B00AE
:1041E0006E9DEA93224DA24D338DAE03B39DBE0367
:1041F0005A9D333B6D01EE93B38DDF02DA93339B0F
:10420000DF02EA9D33BDAD01DA931E9DB243338BCD
:104210007402B39374026E9BB33DBB011E9DB383C6
:104220006A02EA9D339D6A02DA9333BB6301EA9D19
:10423000424D6E9BC24D338DAB03B39DBB031E9DA0
:10424000B3337D006E9BDA93330B1C03B31D1C0349
:104250006A9B333DAB01EE931E9DD243D24DB38397
:104260007C02B39CBC03DA9333BB63011EDE669D04
:10427000B303AB01B38CC7039EC6330BBA02339DA5
:10428000C703669BB33C9B01B31DBA02B303BD01D8
:10429000330D0703E693B31C07035A9D333B6D01AF
:1042A000B30D3603E693DA93331B3603EA9D33BD31
:1042B000AD01B38CDE02DA93EA93339DDE02EE9C0D
:1042C000B3BDBC01EA939E9DF243339D7F02338BC5
:1042D0007F02EA9DB3836402669BB33C9B01EE9C24
:1042E000339D6402DA9333BB6301EA9C669B825C74
:1042F000338D9A03B39C9A031E9DB3337D00669B56
:10430000DA93338B1B03B39C1B036A9B333DAB01D6
:10431000E6931E9D9253B39CE703B30D7C02331CBE
:104320007C02DA9D33BB6D01629DB303AB01338C1C
:10433000E7039EC8330BC903331DC903629B333C9B
:104340008B01B383AC01B30CB802E293331CB80207
:10435000DA9C33BB6C01E293DA93224B330CD60226
:10436000330D6703331B6703669DB33C9D016A9C55
:10437000333DAC01DA93E693B31CD602E6931E9D5F
:10438000B243B39C7E02338B7E02669DB3836F0281
:10439000629B333C8B016A9CB39C6F02DA9333BB04
:1043A0006301669C629B424CB38C8403339C840300
:1043B0009E9CB3B37C00629BDA93338B1A03339CCD
:1043C0001A03669BB33C9B01E2939E9CD243339CB1
:1043D0005702338D7B02B39B7B02B303AB0133BB2C
:1043E00063019EC0DE9CB3039B01B38B57029ECA40
:1043F000330BEA03B31CEA035E9BB33B7B01B303BD
:104400009C01330CC803DE93B31BC8035A9C333B97
:104410006C01B38CB902DE93DA93339BB902E29C50
:1044200033BC8C01B30BD702DA93E293331CD7026F
:10443000E69BB3BC9B01E2939E9CF243331C760245
:10444000330B7602E29CB3836E025E9BB33B7B012F
:10445000E69B339C6E02DA9333BB6301E29B5E9B67
:10446000825B338C7F03B39B7F031E9CB3337C0042
:104470005E9BDA93338B1403B39B1403629B333C30
:104480008B01DE931E9C9253B38C7A02B39A7A020C
:10449000DA9C33BB6C01569CB3038B019EC4E24390
:1044A000B30A5902338B7702331C5902DA9A33BBB1
:1044B0006A01B39B7702B3838B01B30BE803DA93F2
:1044C000331BE803D69BB3BA5B01DA93D693A24AB7
:1044D000338BB602338CCA03B39ACA035E9CB33BD8
:1044E0007C01629B333C8B01D693DE93B39BB60277
:1044F000DE931E9CB243B31B7702B30A77025E9C25
:10450000B3036602DA9A33BB6A01629BB31B66028D
:10451000D693B3BA53015E9BDA9A424BB38B6E03C8
:10452000339B6E039E9BB3B37B00DA9AD693B38A18
:104530001F03339B1F03DE9AB3BB7A01DA939E9B62
:10454000D243338C7402B3947402338D8A01B33A2C
:104550005D01E243A69BB3847A01A6CCA254B31BAF
:104560007A02B38A9702339B9702E244B3049A0219
:10457000B3037B01D694B3BA5401D693B30A58025D
:10458000331B5802A69AB3B49A00DA93A693B39455
:10459000E903338BE903A693B384C603569BB33A6E
:1045A0005B01D693F24A339CC603DA9433BB6401B1
:1045B000E2931E9BF243339CBA02B383B302629B25
:1045C000A693B3B49300B38B6401330B6702825498
:1045D000331C67021E9BB3337B00B38A8B019E9A08
:1045E000B3039602B31B9602DA9333BB6301B38421
:1045F0007A01B38A1E03DA94339B1E039E9AB3B3E7
:104600007A00DA94A6939254125BB3849F02B39F0C
:104610006F03D694B3BA54019E9F338CFA01B25FF4
:10462000A25AB383F703339BF703A25FB30FF903D7
:10463000B31B59039E9FB3B37F00B30A7B019E9ABD
:10464000E243624BB3037802331B6803FE93B3BFAC
:10465000F301DA9AD69FA24A224BB38A5A02331B3D
:104660005B029E9AB3B37A00DA9F338BE6039E9F78
:10467000B393E603569BB33A5B019E9FFE9AB24FFB
:10468000B383CF03B39BCF03DA9333BB6301DE9ACB
:10469000B30FB302569BB31AB3029E9FB3B37F000E
:1046A000569BC24ADA93424BB30A5703331B670344
:1046B000FE9AB3BFFA01DA939E9FB3031603331B2E
:1046C0001603D693B3BA5301DA9FFE9AD24FB38B37
:1046D000FE03B39EFE039E9BC25FB3B37B00F69ABC
:1046E000B38E5301F6CEB393F703C25EB25FB25AF4
:1046F000B38ED703B30FFA03331A5A03F69FB3BE30
:10470000DF011E9AB3834E01A25E338A5602B30ABA
:10471000D803B31ED803FE9AB3BFFA01F693E24E54
:104720009E9FB303C303338BD903B399D903569B1D
:10473000B33A5B015A9A333B6A01F24ECE9FB3996A
:104740005602D69FCE9F7E9BF24FB38EEE03B39F51
:10475000EF03D29E33BA4E01F693B3BED3017E9BD4
:10476000B31FC303529B7E9B825F330A1703DA9EFB
:10477000B389BF02B39FBF029E99B3B379004E9A2B
:10478000B3393A01FE9EB31F17039E9EC253FE9E8D
:10479000F699925EE25FB30AD6033316D603B30EE0
:1047A0005A0133BA4E01B2996256D2993386C70282
:1047B000B397F703C25FB30FF90333197902B29FBE
:1047C00033B6CF00CA973E96B257B303F8023318F8
:1047D000F802FE93B3BFF301A2474296B29F22565E
:1047E000B387C70222462258331606039E97B3B3F7
:1047F0007700B29F6246FE933388C602B396C60224
:104800003E98B337F800B693B2469E973386560269
:10481000B392560242963338060196973E98C247A5
:10482000B306E3033313E303B29633B6C600B38F84
:10483000C7031A984296339EC703B69FB3B6DF00EC
:10484000B387B8027296B2961646264EB395B80252
:10485000FE97B3BFF7019648AE96B69FD246330394
:10486000D7023317D7023E93B337F3007E973388CE
:10487000E700D25737070002B386E700B3B7F60068
:10488000B29713966700E982D18EE98713D6660046
:10489000139BA701336B660152569395A601338B88
:1048A0006841B305B6403336B600B308CB40725604
:1048B000B296B3B3C6003646330BF6003386EC002F
:1048C000B3379601F297139E670069823366CE0074
:1048D000E987135E6600DA93139BA701336B6E01C1
:1048E000264E131FA601338FEC41330B6E41664EEB
:1048F000B3BCEC0133099B41B30AFE00B7070001CA
:10490000338EF600333BDE00DA93939F7300135E21
:104910009E0133EECF0193129E01B3825640C646EC
:104920006A9613DB9341333DA601369BB306F6002E
:10493000EA9A33BDC600EA9A939F7A00E582B3E60D
:10494000DF006E9E939F9601B33CBE01A696330690
:10495000F64193DA9A41B30FEE00669BB3B496002A
:10496000B3BCCF01E29ADA9CA69A864493936C007A
:1049700093DFAF01B3EFF301338CF401333D9C00BF
:10498000D64493DCAC41EA0FA69CB384E600B3B3F3
:10499000D4009E9A93936A00E980B3E49300F643AF
:1049A00093DAAA41EA9C9E9AB303FC0033BD8301CB
:1049B000EA9C139A7C0093D39301B3637A00330D7E
:1049C0007F0093DC9C41338B9B00CA9C333FED01FD
:1049D000B33B7B01669FB30CFB00B3BD6C01D69B60
:1049E000EE9B330AED0013997B0093DC9C01B36CC2
:1049F00099013339AA014A9F93DD9B411A0FB38B6A
:104A00009E01135AAA01B3BADB01336A4F01EE9932
:104A1000338FEB00D699B33A7F01CE9A939E6A000A
:104A2000135FAF0133EFEE013309E30193DAAA41DB
:104A30005698CA9733336900429333B827011A98BE
:104A400013137800E583B367F300135898413303D9
:104A5000F402EA04E60CE6036A0F330B9B41330CC5
:104A60007C405296858EB38BEB41330804039A95B4
:104A700033B365002E97330EFE4123268501232E86
:104A8000650123207503AA442324C5013334F402AD
:104A9000E607B307F94050C91A4914CD5CD14294D6
:104AA000A2989A983333B7009A989A08698333E7A3
:104AB000E8003A441318A701169758C11317AA0122
:104AC000330DED40B38505412328A5010CC18A496A
:104AD000765AE65A565BC65B365CA65C165D865D0A
:104AE000496182805D7166D483AC450256DC930ACD
:104AF000600233865C03A2C6C04183A805005ADA6F
:104B00009316140003AB0502CAC252DE9397180035
:104B10003389180362D66ED04D4C984903A38501A2
:104B20005ED803AF850083ABC50183A34501338AFB
:104B3000C60283AFC500931E1F00A6C413981F00B2
:104B4000CEC093191700139E13006AD2139D1B0049
:104B5000B39DC6024A9A33392A01B3981803B305A4
:104B60008B03EE98CA983389BE02B3825B035299D5
:104B7000333A4901B39DBE02EE98B30D5802469AEE
:104B8000B3185802CA9D33B92D01B3048303D298D8
:104B90004699B3989902CA9833895303338A990284
:104BA000B30A79026E9AB33DBA01EE9833197902CD
:104BB000D29A33BA4A014699B3082A01338A870246
:104BC00046C63309E603B39D87025299333A490139
:104BD000B318E603EE98D298338A0503B39D050314
:104BE0004A9A33392A01EE98B38DE202CA98339972
:104BF000E202D29D33BA4D01CA983389C403D298D8
:104C0000339AC4036E99B33DB9014AC4D298EE9861
:104C100046C833898602B388E703339AE703469987
:104C2000B3381901339486025294A29833040603D0
:104C3000331A06034A9433392401B38D3503D298CD
:104C40004699B3993503A29D33B48D00B388C2034E
:104C50004E9922993394C203EE98B3BDB8012299BC
:104C6000CA9D33896402B39464024699B33819012A
:104C7000EE9433849800B388F70322CAB384E60322
:104C8000B399F703C694B3B81401339AE603338497
:104C900049014694B308E602B319E602A698B3B4F4
:104CA00098004E94B389C5032694B394C503C6995E
:104CB000B3B819012694A29833846202B3946202B5
:104CC0004E94B3393401A698B3841901B389E7022D
:104CD00026CCB3880603339A0603CE98B3B93801BD
:104CE000B394E702B30DEF03D294A699331FEF03F9
:104CF000C69DB3B81D01B304C603FA99C699331F04
:104D0000C603EE94B3BDB401FA99CE9D9319130076
:104D1000338FB902B399B902269FB3349F00338A07
:104D20007203CE9DEE94B39272037A9A333FEA01F6
:104D3000A692B3085F00338FF302B382E602B39901
:104D4000F302FA9233BFE201B39DE602B384B901E4
:104D5000FA94338FFE03B399FE03169FB3325F00BC
:104D6000CE94A692B3046602B3196602FA9433BFD6
:104D7000E401CE92FA92339FA503B389A503FA9278
:104D8000B39D6702A699B3B49900969426CE339F3B
:104D9000C603B38267026E9FB384C603B39DEE025F
:104DA0009694B3B25400169FB382EE026E9FB30D79
:104DB000F803A692B3B49200FA94B31FF803969D39
:104DC000B3B25D00330FA603FE949694B312A6030C
:104DD0006E9FB33DBF019694A69DB3846503B395C2
:104DE0006503FA9433BFE401EE95B30FBF00B39DA2
:104DF0006602339F7703B38277036E9FB3856602A3
:104E0000B38D7E029695B3B25500FA92B3937E02AB
:104E1000AE9DB3B5BD009E92AE92B315E802330FBE
:104E2000E802AE92B30366036E9FB33DBF01969D49
:104E3000B3156603FA9333BFE301AE9DB382A603B5
:104E40006E9FB3856703B39D6703AE92B3B5B2009F
:104E5000339DA6036E9D2E9DB3856E02B39D6E029B
:104E60009695B3B255006E9DEA92330DC803B31DFB
:104E7000C8032E9DB335BD00EE929695B302E702AE
:104E8000B31DE702EA9233BDA201EE952E9DB30554
:104E90009603331696039695B3B25500329DEA9267
:104EA00033869703338D6603B3979703329D33366A
:104EB000CD00B3966603B38D7E03B6973E96B39E40
:104EC0007E03EA9D33BDAD01330B68027696329DB9
:104ED0003246331868026E9BB33DBB013243B30EBA
:104EE000C703429DEA9D3317C703DA9E33BB6E01A9
:104EF0006E97330EEB0037070002B386EA00B3B7B4
:104F00005601B29713966700E982D18EE98713D8CC
:104F100066001396A7013366C8001398A60133886C
:104F20000A413306C340B3BA0A01B30A56412246C6
:104F30004243B29633B6C600B30DF300B29D3306BA
:104F4000EA00B3374601C697139367006982336658
:104F5000C300E987135B66001393A70133636B00FB
:104F6000B38868407243131BA6014E969A97B339D3
:104F70003601330B6A41BE99B70700013383F6004F
:104F8000333A6A01B3884841333AD300D29D139A29
:104F90007D001353930133636A00931B9301B38B1A
:104FA0007641D2464A9393DD9D4133392301338ABA
:104FB000B601B306F6004A9A33B9C600CA991399E6
:104FC0007900E582B366D90093D999411399960186
:104FD000CE9FB309E300A6963306264133B9690094
:104FE000B3B496005299A69F93D9A901931469006E
:104FF000B3E93401E244B30C34011359A9412699B1
:1050000033B48C004A943389E600B334D900A69FA8
:1050100093946F001359A90133E9240193D4AF414C
:10502000B38F2301B3B37F00269FB384FC001E9F80
:10503000B3B394011E94135A944193137400D298FD
:10504000E580338AFF00B3E49300B333FA011E9F77
:1050500093137F00135A9A0133049B0033EA4301F0
:1050600093539F41333B64019E92B303E400DA986B
:1050700033BB8300DA98338F45019A0893D3A30199
:10508000B335BF00B3E37800B308EF00AE92B3B519
:10509000E80196959392650093D8A801B3E81201B0
:1050A000338B1E01E9852E9EDA97B33EDB01F29E1B
:1050B00033BE6701769E93157E00E583CD8F135E28
:1050C0009E41B305FC02EA09E6046A09660AEA0899
:1050D000B38C9C4033033341B3862641B38F4F4199
:1050E000330ECC032E98B335B80042971E96330F7B
:1050F0001F41232695012324650050C914CD333C5C
:10510000FC02E607B307FB40232EF5012320E5034D
:105110005CD1A64416498649725A729CE29AAE9AAC
:10512000B3350701AE9A9A0A698333E7EA0093150B
:10513000A7015E9758C11397A301198C00C9364483
:105140003308B84023200501E25A525BC25B325C4F
:10515000A25C125D825D6161828063CB050093D7A2
:1051600035403E9508219D893355B540058982809B
:1051700001458280138E0502930E0602B2882A88AA
:1051800001479C4103A3080091081108B3866702F8
:1051900033B367028327C8FFB6973E97B3B6D700ED
:1051A000232EE8FEB337F7009A963387D700E39AA9
:1051B0001EFD18D191051105E312BEFC8280B16578
:1051C0008146854793850571130800023387D50012
:1051D0003306D5001843104291061347F7FF3A965D
:1051E000B2973337E600B3B7C700BA97E39006FF2C
:1051F0003E858280EFA2DFFF41112A842E852EC6D4
:10520000EFF0FFFBB24531661358F5413303A04080
:1052100081461306067193080002B307D6009C432B
:105220003387D500184393C7F7FFB3F767003E975E
:10523000B337F7003A95C2973308D4002320A8006B
:105240003337E50091063305F7000148E39716FD73
:1052500041016FA03FFCEFA2BFF92A84EFE08FE885
:1052600013058402EFE00FE913050405EFE08FE872
:1052700013058407EFE00FE76FA0DFF9EFA25FF7F8
:10528000138985022E842E86CA85AA84EFE08FEBCF
:105290002286CA8513858402EFE02FED930504056D
:1052A00013850405EFE08FE631661306866E9305DD
:1052B000840713858407EFE03FD96FA0BFF5EFA205
:1052C0009FF15D7113848502AA84328A2E892E860D
:1052D0000A85A285EFE00FE74A86A2852810EFE055
:1052E000CFE852868A850A85EFE01FD62C10130678
:1052F0008A022E85EFE05FD5938A840230108A857A
:105300005685EFE02FE430108A852685EFE0EFE543
:105310001384040513060905B2852285EFE08FE2A8
:1053200013060A05A2852285EFE01FD29389840720
:1053300013068A07930589074E85EFE0FFD04E8656
:10534000A2850A85EFE00FE04E86A2852810EFE0E7
:10535000CFE15686A6854E85EFE01FCF3010A6859B
:105360002685EFE07FCE0A86D6855685EFE0DFCD35
:1053700030108A852285EFE03FCD61616FA0FFE8A4
:10538000EFA29FE4138A85022A89AE893685B28B03
:105390002E86D2853684BA84EFE0CFDA4E86D28567
:1053A0002685EFE08FDC5E86A2852285EFE0DFC9EF
:1053B00013868B02A6852685EFE01FC9130B890291
:1053C0002686A2855A85EFE0EFD72686A2854A85F4
:1053D000EFE0AFD9130A090513860905B285528596
:1053E000EFE04FD6930A890713860B05938589074B
:1053F0005685EFE07FC55686D2852285EFE08FD4B3
:105400005686D2852685EFE04FD65A86CA855685C0
:10541000EFE09FC32686CA854A85EFE0FFC2228659
:10542000DA855A85EFE05FC22686A2855285EFE0D5
:10543000BFC16FA0FFDCEFA21FDA32842A8AAE8AD6
:10544000328593048402EFF0EFE9138B8A02DA8548
:10545000268513090405EFF0EFE893850A054A85D0
:10546000EFF04FE8CA854A85094693098407EFE0C3
:105470009F8E5A86D6854E85EFE0CFCC930A8A0759
:10548000CE855685EFF00FE62286A6854E85EFE0A5
:105490006FCB2286A6852685EFE02FCD4E86D6855A
:1054A0002285EFE08FCC2686CA854A85EFE0EFCBD8
:1054B0004A86A2855285EFE03FB92686CE85130540
:1054C0008A02EFE07FB84A86A68513050A05EFE059
:1054D000BFB74E86A2855685EFE01FB76FA0FFD2FB
:1054E000EFA21FD1AA842E891304C00FA2854A857A
:1054F000EFF0BFC619E17D1475F80504FD57A0B0A3
:105500009EA0BCA06FA01FD1EFA21FCC2431AA89FE
:1055100032896393C402AE8A3685B285368B130A0C
:10552000F9FFEFF09FC32A84D2855A85EFF0FFC2BE
:10553000631DA400A3814901839709000145639479
:105540002701038529006FA0BFCB138A140063D302
:105550004A01568A1305FAFF3314A400330480402D
:10556000814A330C4941D68B850A63185A05E28576
:105570005A85EFF09FBE2295B307A040E98F13F440
:10558000A70A13F7C70C3334800011C3094793F7F8
:10559000070F598C91C3914713071900C18F330727
:1055A00047413E973355F540B38444412390E90089
:1055B0002381A900A381990041B7B3055C015A85F5
:1055C000EFF0BFB9331575012A9471BFEFA25FBF29
:1055D00041112E892A8AC2853E853E8BC28B3AC6EE
:1055E000B289B68AEFF07FB793850B022A845A8579
:1055F000EFF0BFB693850B04AA845A85EFF0FFB590
:105600000A058604AA9493850B065A852694EFF022
:10561000DFB41374F40F0E0522951375F50F135BA9
:1056200035003247930CFBFF33C5AC00937C75000B
:10563000BA84014D130C8902930B0905A14D33C4A3
:10564000AC017D1421800588A68522864A85EFE07D
:105650008FC19385840222866285EFE0CFC0938557
:10566000040522865E85050DEFE0EFBF9384840775
:10567000E317BDFDDE854E85EFE0EFAA134B1B005F
:105680005A86CE855E85EFE0CFB05A86E2854A85A0
:10569000EFE02FB05687CE864A86D2855285EFF04E
:1056A0003FCE41016FA09FB5EFA29FB4EFE04FA1A5
:1056B0004D8D133515007D156FA0DFB581476393C0
:1056C000B70082803307F500230007008507C5BFB8
:1056D000EFA21FB279712A848147130780023386B3
:1056E000F50010423400BE9690C29107E399E7FEA0
:1056F0003257CD471018B387E70237070001BA9732
:105700003800E587BA868C42A106AE9783A5C6FF0E
:10571000E987AE97E587E318D6FECD46B387D70273
:1057200014432107B69793D6A7419395A6018D8F71
:10573000232CF7FE8327C7FFBE9693D796419395F8
:1057400097018D8E232ED7FEE31CE6FCB247A245BF
:105750002285EA07DD8DEFE04F8CB245C247130585
:1057600044009981CE07DD8DEFE02F8BC245D247F3
:1057700013058400B581B607DD8DEFE00F8AD245B1
:10578000E2471305C400CD819A07DD8DEFE0EF8875
:105790008257F24513050401E607DD8DEFE0EF8740
:1057A00082559257130544019D81CE07DD8DEFE0B0
:1057B000CF869255A25713058401B581B207DD8DBE
:1057C000EFE0AF85A255B2571305C401D1819A0706
:1057D000DD8DEFE08F84280093058002EFF01FEE4F
:1057E00045616FA03FA3EFA2BFA039712E84AA85A7
:1057F0000A85EFF0FFEDA2850810EFF07FED0C10A9
:105800000A85EFF07FEA2A84930500020A85EFF00B
:10581000FFEA081093050002EFF05FEA1305140099
:1058200021616FA03F9FEFA21F9B19712A89280059
:105830002E84EFF02FAB2C000818EFF0AFAA0C1855
:105840002E85EFF02FAA10183285A285EFE0CFFF4A
:105850002C0010182E85EFE02FFF2C002E85EFF086
:105860006FA8300032850C18EFE00FFE2C000818EE
:10587000EFF04FA791440C182E85FD14EFF08FA682
:10588000FDF8300032850C18EFE00FFC2C000818F2
:10589000EFF04FA5A5440C182E85FD14EFF08FA452
:1058A000FDF80C182E853000EFE00FFA0C18A80850
:1058B000EFF04FA3CD44AC082E85FD14EFF08FA27E
:1058C000FDF810183285AC08EFE00FF80C182E85A3
:1058D000EFF04FA1A5440C182E85FD14EFF08FA01A
:1058E000FDF8300032850C18EFE00FF62C00081898
:1058F000EFF04F9F930410030C182E85FD14EFF06A
:105900006F9EFDF80C182E853000EFE0EFF30C18B9
:10591000A808EFF02F9D93043006AC082E85FD14E7
:10592000EFF04F9CFDF810183285AC08EFE0CFF196
:105930000C182E85EFF00F9B930410030C182E8586
:10594000FD14EFF02F9AFDF8300032850C18EFE0CF
:10595000AFEF2C002E85EFF0EF982C002E85EFF0A6
:105960006F982C0022862E85EFE00FEE2C00081891
:10597000EFF04F970C1822862E85EFE0EFECA80889
:10598000EFD05FF6AC082285EFF0FFE52A84A80887
:10599000EFD05FF6AC080818EFF0FFE4AC08AA8A75
:1059A0002E85EFD05FF8AC080818EFF0DFE3356A1A
:1059B000AA8993054A32A808EFD0FFF6AC08081868
:1059C000EFF07FE213064A322C00AA844A85EFE00A
:1059D000AFE7B3E499000546058E2C004A85EFE059
:1059E0008F88280093058002EFF05FCD081893059B
:1059F0008002EFF0BFCCA80893058002EFF01FCC27
:105A0000336554013365350109616FA01F80EFA232
:105A10002FFE39712A8428082EC6EFF0AF8C2C088F
:105A20002E85EFF05FE02C082E85EFF0AF8B32462D
:105A30002C082285EFE04FE1280893058002EFF063
:105A4000FFC721616FA00FFDEFA2EFF82D712A8A29
:105A50002E8B2800B2850546B684EFE04F8A0818E1
:105A6000EFD05FE9A808EFD0FFE72C000801EFD0E6
:105A7000FFE928117969EFD0FFE7FD14014413090C
:105A800029B4FD5AA6855A85EFF02FED298C228680
:105A9000AA890C010818EFD0DFEF22862C11A80884
:105AA000EFD03FEF30110C018809EFD01FECB008A8
:105AB0000C18A819EFD07FEB0C182E85B008EFD08A
:105AC0007FE830110C01A808EFD0DFE710188C092F
:105AD0002811EFE06FD7AC08B0192E85EFE0CFD6D4
:105AE000AC198809EFF00F800C18A819EFE09FFFA0
:105AF000B0082C110801EFD0FFE4B00832852C115A
:105B0000EFD0BFE69009AC190818EFE0EFD3AC195D
:105B100090092E85EFD07FE5AC082E85EFE09FFC45
:105B20004A86AC192811EFE00FA30C012E85EFE097
:105B30007FFB8C092E853011EFD0DFE0B0082C0000
:105B40002811EFE06FD09009AC19A808FD14EFE020
:105B5000AFCF4E84E39854F34E860C010818EFD073
:105B60005FE34E862C11A808EFD0BFE2AC082E856B
:105B7000EFF0FFE90C18B0082E85EFE0EFCC0C1821
:105B80005285EFF0FFB4280093058002EFF01FB3B9
:105B9000081893058002EFF07FB2A80893058002F1
:105BA000EFF0DFB1880993058002EFF03FB1080103
:105BB00093058002EFF09FB0281193058002EFF06B
:105BC000FFAFA81993058002EFF05FAF15616FA0DA
:105BD000CFE3EFA2EFE159712E84AA848145130629
:105BE00040066800EFA0CFE36C00B56E2E8801433D
:105BF000938E0E30930F040493024002B3876E001D
:105C000003AF07002286A2884285014783A70800C8
:105C100091081105B306FF02333EFF028327C5FF3B
:105C2000B6973E97B3B6D700232EE5FEB337F700FD
:105C3000F2963387D700E39BF8FD2320E804110395
:105C40001108E31D53FA02C602C802CA02CC02CEF2
:105C500002D002D202D41308C100A148316F930EC2
:105C60000F714285014E81468327080403A30E006D
:105C7000050E110533876702910E33B36702832740
:105C8000C5FFBA97BE9633B7E700232ED5FEB3B74C
:105C9000F6001A97B386E700E3681EFDFD181108A9
:105CA000E39F08FA13040402854698411C4211063A
:105CB0001347F7FFBA97BE9633B7E70094C1B3B75F
:105CC000F600B386E7009105E31186FE6C002E8591
:105CD000EFF04FD221466C002685EFD01FB8680048
:105CE00093054006EFF09F9D65616FA0AFD2EFA2D4
:105CF0002FD00111AA850A85EFF09F9D00800A85AB
:105D000093050002EFF09F9B0588228505616FA037
:105D10006FD0EFA24FCC130985022A8405464A852D
:105D20002E8A93090405EFD09FDD4E8593048407E6
:105D3000EFD05FBCCA852685EFE0DFDA3566130653
:105D40000627A6852285EFE02FB04E86A6852685FC
:105D5000EFD0BFC14E86A2852285EFD0BFBEA685FB
:105D600022852286EFE04FAEA2852285EFF0BFAB01
:105D700015C92286A6852285EFE00FAD2285EFF0BA
:105D80001FF78347FA019D836316F500A2852285DC
:105D9000EFD07FB926854A86A285EFE0EFAA0145BC
:105DA0006FA0AFC67D55EDBFEFA28FC419712A84D5
:105DB000AE84280093850505EFF07FC53000A685E9
:105DC0000818EFE06FA8300093858402A808EFE080
:105DD000AFA7AC082285EFF0BF8F0818EFF03FF1B6
:105DE000A167938707F81E057D8D7C3C9305800293
:105DF0003D8D68BC2800EFF07F8C08189305800269
:105E0000EFF0DF8BA80893058002EFF03F8B09616C
:105E10006FA04FC0814713070002B386F5009022A0
:105E2000B306F500850790A2E399E7FE1C21E19BEC
:105E30001CA17C3D93F7F70793E707047CBD8280A4
:105E4000EFA20FBB79712A84080832C6EFF09FFCDD
:105E500032469306F00F0C082285EFF0FFBE0808CB
:105E600093050002EFF09F8545616FA0AFBAEFA2E6
:105E70002FB839712A8441460A85EFD05F9B8A8505
:105E80002285EFF01FD50A8593050004EFF01F83EC
:105E900021616FA02FB8EFA2AFB575712A84B284CB
:105EA0000808214636C6EFD09F98A68508182146D7
:105EB000EFD0FF97B24688082146B685EFD03F97CE
:105EC00010180C08880882D882DA82DC82DE02C1CF
:105ED00002C302C502C7EFF0EFA98C082285EFF0DC
:105EE0005FCF880893050004EFF04FFD0808930585
:105EF0000002EFF0AFFC081893050002EFF00FFC72
:105F000049616FA02FB1EFA20FAD6571B56635661F
:105F10009386062E1306062C2A842800EFF0BFF77E
:105F2000A818EFD03F9D0811EFD0DF9CA801EFD05B
:105F30007F9B2285EFF02FB2B5697D483C00138727
:105F400009AF94083010AC182285EFF02FE83169C2
:105F50001308F0093C001307097394083010AC18BB
:105F60002285EFF0AFE6F9447D5A9019A28522858B
:105F7000EFF06FCC26883C00138709AF94083010EF
:105F8000AC182285EFF08FE4138804083C00130757
:105F9000097394083010AC182285FD14EFF00FE35C
:105FA000E39544FD281093058002EFF02FF1881946
:105FB0009305000AEFF08FF0880893058002EFF058
:105FC000EFEFA81893058007EFF04FEF2800930537
:105FD0000002EFF0AFEE59616FA02FA3EFA2AF9FC9
:105FE000130101BE130A0502AE842A84D2858815E6
:105FF000B28A2146EFD0BF83A6858810EFF07FD10B
:1060000011C57D55130101426FA02FA0A285080282
:10601000EFF03FD07DF58815EFF06F9A7DF1900499
:106020008C100813EFF02FC18C108815EFF00FA51E
:1060300090150C138804EFF08FA88C040807EFF07C
:10604000EFA3D6852800EFF0AFC9D2856800EFF046
:106050002FC99C870349B1006373F9003E898810FA
:10606000B5691379F90FEFF00F9F094B938909EB8D
:106070008C102E851013EFF00FBCD6864A868D4506
:106080002800EFF06FC82A84D2864A8695456800BA
:10609000EFF08FC7AA846352800805841306000AB4
:1060A0003306C4029C153E968C102E85EFF02FA16E
:1060B0006359900A8584130680073386C402381812
:1060C00014084E968C102E85EFF08FAB7D19FD577E
:1060D000E310F9FA0C028804EFF04F9A8C10900448
:1060E0002E85EFF0CF9D8C1010022E85EFF0AFB40F
:1060F0008C1010022E85EFF00FB48C1010022E853C
:10610000EFF06FB38C100813EFF01FCAB5659385DD
:10611000C5340813EFF04FD9F5B559D833446403AB
:10612000930500F69C15A8143304B402B3858700C8
:10613000EFD0CFFD9C1593058402BE958804EFD067
:10614000EFFC9C1593050405BE95080DEFD00FFCE0
:106150009C1593058407BE95281DEFD0CFFC9004B5
:10616000A1B7ADD4B3C46403930780F8A814B38473
:10617000F402CE94A685EFD06FF99385840288044B
:10618000EFD0CFF893850405080DEFD0CFF938187C
:106190001408900405BFEFA2AF8535712A840A85E3
:1061A000EFF07FD68A852285EFF01FC00A85930520
:1061B000000AEFF0AFD00D616FA0CF85EFA24F8343
:1061C0005D71AA8405462810EFD07F9335643010A6
:1061D000930584290A85EFD0EFF6301032859305B8
:1061E0008429EFD08FF82C102E85EFF05F823010CD
:1061F0008A850A85EFD05FE58A852685EFF04FCD49
:106200000A8593058002EFF06FCB2810930580027A
:10621000EFF0CFCA61616F90FFFF1C211831E207D8
:106220004207D98F38312821D98F22055D8D828090
:10623000935785019CA1935705019CB19357850005
:10624000BCA1A8B1828098411C41B98F1CC1D84122
:106250005C41B98F5CC198451C45B98F1CC5D845B8
:106260005C45B98F5CC58280032805005041370327
:1062700000FFB708FF001445B375160133776800B7
:106280005C454D8FC165938505F033FEB6003367DD
:10629000C70113FEF70F3367C70118C133FE16019C
:1062A000337766003367C70133FEB7003367C70132
:1062B000137EF80F3367C70158C133FE170133F758
:1062C00066003367C701B3F76700337EB8003378E1
:1062D00018013367C701B3E70701137EF60F6D8E10
:1062E000D18F93F6F60F3367C701D58F18C55CC5FC
:1062F0008280370701019357750013071710F98F34
:106300006D47B387E7023707FFFE1307E7EF060580
:10631000798D3D8D8280EF92BFED2A84EFF07FFD75
:10632000135704019317040193168401D98F13574F
:106330008400558FB98F298CA98F13158400618033
:10634000418D3D8D6F901FED14415C45370300FF7B
:10635000B708FF0003288500B3F5170133F766007F
:1063600050414D8FC165938505F0337EB80033678A
:10637000C701137EF60F3367C70118C133FE16013C
:10638000337766003367C70133FEB7003367C70151
:10639000137EF80F3367C70158C1337E1601337778
:1063A00068003367C70133FEB6003367C70133782F
:1063B000180113FEF70FB3F76700B3E707016D8EFF
:1063C000D18F93F6F60F3367C701D58F18C55CC51B
:1063D0008280EF92FFE12A84EFF0BFF12A89EFF08B
:1063E0005FF1AA84EFF0FFF0218DB3C7A4009316EC
:1063F000850133442401135785003349A90013153F
:1064000089003D8C558F1359890133692501398CD9
:1064100013950701C183334424015D8D218D6F9055
:106420007FDF935F0501135F850093538501814EE4
:106430000143014E0146014893FFFF0F137FFF0FF9
:106440001375F50F93020010B387050183C8070089
:10645000B3C7030193F7F70F93C6F7FFFD17FD8E40
:10646000E206FD8693C7F6FF7D8EB3C70F0193F753
:10647000F70F13C7F7FFFD177D8F93F8F80F62072B
:10648000B3F6D8007D87558E9346F7FF33FEC601DD
:1064900033F7E800336EEE0033470F011377F70F41
:1064A0009347F7FF7D17F98FE207FD8713C7F7FFC3
:1064B0003373670033470501B3F7F8001377F70F1D
:1064C0003363F3009347F7FF7D17F98FE207FD87EA
:1064D00093C6F7FFB3F6D601B3F8F8000508B3EE9C
:1064E0001601E31358F69316860113170E01D98E81
:1064F000B3E6D60113158300558D8280EF925FCCF1
:10650000044113592600411185042A84328A8A04E1
:10651000931A2900814963933A03B569930D4400A6
:10652000CA8C5694014C054DB56A9389C9366D4B9A
:10653000914B63E09C0241016F905FCC3385350144
:106540002EC6EFF09FCDB3073401C8C39109B24501
:10655000D9B70840631A2C03050D93178500618194
:106560005D8D93858A37EFF0DFEBB387A9019C231C
:10657000014CE2073D8D83A70D00850C050C3D8D78
:1065800048C0910D110475B7E3090CFCE3754BFF8E
:10659000E3137CFF93858A37EFF0BFE8E9BFEF9202
:1065A0003FC52A840841B56493858437EFF07FE7BF
:1065B00008C0484093858437EFF0BFE648C00844E0
:1065C00093858437EFF0FFE508C44844938584370A
:1065D000EFF03FE548C46F90FFC3EF92DFBF1C416F
:1065E0002947411193F6B7FF2A89AE843284638725
:1065F000E60031476384E700EF30602C2685EFF03A
:10660000DFC12AC013854400EFF03FC12AC21385C1
:106610008400EFF09FC02AC41385C400EFF0FFBFD1
:106620002AC6930549000A85EFF0FFC1930449018A
:106630008549832709000A8563E1F904EFF03FF6F5
:106640000A85EFF07FC2A6850A85EFF0DFBF02451D
:10665000A285EFF0FFBD124593054400EFF05FBD4A
:10666000224593058400EFF0BFBC32459305C4007A
:10667000EFF01FBC41016F905FB9EFF05FF20A8548
:10668000EFF09FBE02458509EFF0FFC82AC0124512
:10669000EFF07FC82AC22245EFF0FFC72AC4324577
:1066A000EFF07FC72AC6A6850A85EFF0DFB9C104DF
:1066B00049B7EF92FFB32A840841B56493858447B4
:1066C000EFF03FD608C0484093858447EFF07FD570
:1066D00048C0084493858447EFF0BFD408C44844B9
:1066E00093858447EFF0FFD348C46F90BFB2EF9219
:1066F0009FAE0041A94741111377B4FFAA892E89A3
:10670000B2846307F700B1476304F400EF30201B45
:106710004A85EFF09FB02AC013054900EFF0FFAFA4
:106720002AC213058900EFF05FAF12042AC41104D6
:106730001305C900EFF07FAE4E942AC6A2850A85E4
:10674000EFF07FB003A90900130A04FF9309F9FFD2
:1067500063960904C1553309B9020A85EFF0DFBE1B
:106760000A85EFF01FF50A854A94A285EFF0BFADC8
:106770000245A685EFF0DFAB124593854400EFF0AC
:106780003FAB224593858400EFF09FAA3245938565
:10679000C400EFF0FFA941016F903FA70A85EFF019
:1067A000BFBA0A85EFF0FFF0D2850A85EFF0BFA9E6
:1067B0000245411AFD19EFF0DFC12AC01245EFF082
:1067C0005FC12AC22245EFF0DFC02AC43245EFF094
:1067D0005FC02AC6B5BFEF92BFA12E84B2848145A7
:1067E0001306400FEF90DFA36147AA876382E4029C
:1067F000130700026382E40241476394E4022947DD
:1068000018C14146A2853E85EFF05FCF6F909FA0F3
:10681000314718C16146FDB7394718C11306000258
:10682000D5B7EF30C009EF92BF9C1306400F8145EA
:10683000EF901F9FAA879C236F90DF9DEF92BF99D7
:1068400013F4F60011711DE832892E86AA856800BE
:10685000BA89B684EFF03FF8636994006800EFF0FE
:106860009FFC014511616F905F9A33868900B305E3
:1068700089006800EFF07FD64104F9BF7D55DDB790
:10688000EF927F9513F4F60011711DE832892E8680
:10689000AA856800BA89B684EFF0FFF363699400B3
:1068A0006800EFF05FF8014511616F901F96338625
:1068B0008900B30589006800EFF07FE34104F9BF68
:1068C0007D55DDB7EF925F9019C5AA8A88412E8A5F
:1068D00032896364C500EF20907EB6843A84BE8B13
:1068E000428C468B91E265FBE3870BFEE3050BFED2
:1068F00005CD1DC8B309A94063733401A2894E8632
:10690000A6855695EF30E00483270A00CE94330421
:106910003441BE9923203A0163982901D6855A85CE
:1069200009E8029C23200A00637724011DE06F9090
:106930003F8D829BC5BF83270A00D1FFA6855A855C
:1069400063172401029CCA9433042441F1BF829B43
:10695000DDBF03250A00B309A94063733401A2898E
:106960004E86A6855695EF20D07E83270A00CE94CA
:1069700033043441BE9923203A01E3E929FBA1BF46
:10698000EF921F87C2883E88EFF0DFF36F909F88F9
:10699000EF929F832A8BAE89328AB68B3A893E8CDE
:1069A000C28C814A631409006F909F8583A40900FB
:1069B00033049A40637389004A8463980A002286EC
:1069C000DE8533059B00EF90BF8581E463138A0069
:1069D000854AA294639A4401DA856685029C23A0C5
:1069E0000900330989407DBF03A70900229723A02E
:1069F000E900C5BFEF922FFE41113A8BD4875C8727
:106A000005474684C2546300E804428963060804CB
:106A10008947AA892E8AB28A6303F8042688C68722
:106A20009306F1000547EFF0BFF514872688A2878B
:106A3000638766051307E9FFDA865686D2854E8599
:106A4000EFF01FF525A0BD8ED4872688C6870547A1
:106A50009306F100EFF0DFF241016F900FFB268803
:106A6000C68705479306F100EFF09FF12688A287BD
:106A700005479306E1005686D2854E85E1BF130790
:106A8000F9FF5686D2854E85EFF09FF0F1B7EF9271
:106A90002FF6257119E1EF2090621C452A84280801
:106AA00036C632C42EC2829722465C4492452808DC
:106AB0008297B2461C482808B6858297130680182C
:106AC00081452808EF90CFF5834781011D616F90C4
:106AD0006FF4EF924FF0117119E1EF20505E2E84A8
:106AE000EDDDB289814513068031AA843689EF90A5
:106AF0002FF39C205C4080C063FB270B1840E3EE23
:106B0000E7FC4A868A86CE852285EFF05FF8032966
:106B10000400832944006379390133862941814582
:106B200033052101EF90CFEF8147639CF9041C44AA
:106B3000138984004A8582975C4450400C014A8541
:106B40008297544081476399F6041C449384041946
:106B5000268582975C4450400C0126858297130657
:106B6000000881450801EF90AFEB83470108130649
:106B7000000881450A85EF90AFEA1C8011616F9093
:106B8000CFE81801B306F7003307F1001823850793
:106B90001347670398A251BF18013306F700330764
:106BA000F100182385071347C70518A269BF4A8655
:106BB000CE850A85EF20F059A9BFEF926FE319C186
:106BC0001C4199E3EF20B04FDC47210582976F907D
:106BD0006FE4EF92EFE1397101C51C412A8499E31A
:106BE000EF20F04D2E89EDDD9C4B8A8521058297A3
:106BF0001C40930404198A85D84790432685029740
:106C00001C40CA8526859C4B82971306803181459E
:106C10002285EF90EFE01C2021616F90AFDFEF92B3
:106C20002FDD130101CDB684AE86B5653284938520
:106C300085672A8628083AC6EFF0BFE92686A2852E
:106C40002808EFF09FF732472808BA85EFF07FF861
:106C50000145130101336F90EFDB935785019CA130
:106C6000935705019CB193578500BCA1A8B18280C0
:106C70001971D6D4DAD21841832E4500032E85002F
:106C8000032BC5001C49832F4501032F8501832A4F
:106C9000C501B562A2DEA6DCCADACED8D2D6E6CC71
:106CA000EACADED0E2CEEEC89382825781463A8AA3
:106CB000F6897289DA843E84FE837AC456C63D4DD5
:106CC000930C00046363DD1283CB0500903113083D
:106CD0000101E20B4206B3EBCB00B0319105B3EBFF
:106CE000CB0003C6E5FF2206B3EBCB0013962600CC
:106CF00042962320760113D867009398A701B368C2
:106D000018011396570113D8B7003366C80033C86B
:106D1000C80093D89701139677003366160133465F
:106D2000C80013C8F7FF3378E801B3F8F701334818
:106D30001801429603A80200850691024296B29B72
:106D40001318E70113562700DE9A33680601935B98
:106D5000D70013163701B3EBCB0033467801135835
:106D60006701931BA700B3EB0B01B34B760133C64E
:106D7000CE01798E33F8CE0133460601B29BD69B05
:106D800033866A01728BFA8A639A96059E975CC96C
:106D9000A247329400C9BE9FB2477654D29B3E9F11
:106DA0003C514E97CA9E269E85072320750158C1E7
:106DB0002324D5012326C501232CF501232EE5012B
:106DC0003CD1E6545659C659365AA65A165B865BCC
:106DD000764CE64C564DC64D096182807E8F768E8C
:106DE000BE8FBA8EB2875E87F1BD1386E6FF3D8AFD
:106DF000130801050A064296032306FC138616FFB4
:106E00003D8A0A064296832806FC138696FF13F8ED
:106E1000F6003D8A930B01050A060A085E985E9605
:106E2000832B06FC032608FC131CF300935D33013F
:106E3000B29B13561301336CCC001316D300336688
:106E4000B6013346CC001353A30033466600B29B11
:106E500013D37800139698013366C30013DC28011E
:106E60001393E800336383013346660093D83800F8
:106E7000B3481601C69B232078FDB5BDEF924FB7EE
:106E80002A8413068004814513050502EF904FB94B
:106E9000B7E7096A938777661CC0B7B767BB938764
:106EA00057E85CC0B7F76E3C938727371CC4B7F729
:106EB0004FA59387A7535CC4B7570E519387F72705
:106EC0001CC8B777059B9387C7885CC8B7E7831F43
:106ED0009387B79A1CCCB7D7E05B938797D15CCCEC
:106EE0006F904FB3EF92CFB0B77700002A88328708
:106EF000AE86938707C7930545061306000413055E
:106F00000502EFF0FFA76F90EFB0EF92CFAC3C51CE
:106F100003294506011113D7A7019A073E99B334F7
:106F2000F900BA949357D9018E04DD8C9307890038
:106F300093F7F703B7780000130800042A84330896
:106F4000F8402AC0938808C7814701479306000884
:106F500013060004AE899305450613050502EFF0FC
:106F60007FA9131A390093D78400230DF10093579A
:106F70008A01230EF10093570A01420A135A0A01AB
:106F80002E09135A8A003369490121462C082285AB
:106F9000A30EF100231C0100A30D9100231F21016A
:106FA000EFF05FF47C5099C3EF2070110840CE855C
:106FB000EFF0BFCA484093854900EFF01FCA08446C
:106FC00093858900EFF07FC948449385C900EFF0AD
:106FD000DFC8084893850901EFF03FC8484893850A
:106FE0004901EFF09FC7084C93858901EFF0FFC678
:106FF000484C9385C901EFF05FC6130680068145B2
:107000002285EF90EFA105616F902FA0EF924F9E28
:1070100059712E8413068006AA852800EF2070136C
:107020002800A285EFF07FEE65616F90AF9EEF9232
:107030002F9C01111306000281450A85EF904F9E97
:10704000854513050020EF20800D31653724014070
:10705000EF10306F13050440EF101025B7070E0036
:107060003EC68A85854713050440230AF10002C005
:1070700002C202C402C8EF10302785451305044040
:10708000EF10F02B814513050440EF10B03E1305BF
:107090000440EF10D02B930404402685EF10D02B32
:1070A0006DFD1305044037240140EF10702B93044D
:1070B00004402685EF10702B6DFD13050440EF1082
:1070C000F03C2391A182854513050440EF10903ACE
:1070D0000545EF10903705616F90CF93EF924F9178
:1070E00037240140AA859D46054613050440EF104C
:1070F000D029854513050440EF10B02793040440C0
:1071000089452685EF10703665DD13050440EF10C4
:1071100050336F902F90EF92AF8D41112A89014427
:1071200081446319B40033D5840241014205418191
:107130006F904F8E4A852EC6EFF05FFAAA941545E0
:10714000EF20603205041374F40FB245D9BF0397E2
:10715000218281472A97634F070009CD0566930670
:10716000F6FFB6876358C700AA876305D500931753
:107170000701C1833E858280B7F7FF1F83A707728F
:10718000A94613D70701C207C1831D8D9307400687
:107190003305F5029307B00255053345F502330771
:1071A000D7023305A7408280EF928F84A9454145DD
:1071B000EFF07FF642054185EFF07FF98567938711
:1071C00047CE3305F5023185EFF01FFB42054185BF
:1071D0006F904F84EF92CF81A9450545EFF0BFF343
:1071E00042054185EFF0BFF68567938747CE3305AB
:1071F000F50231856F900F8263550500B7070001D6
:107200003E95935705419CA1935785409CB1A8A1F9
:107210008280EF82FFFD3A84AE8708A3130780F8CF
:1072200041113E8518B09305240036C432C6EFF0F4
:10723000BFFC3246930554003285EFF0FFFBA246B7
:10724000930584003685EFF03FFB41016F809FFC82
:10725000B707002005679387C738130707B83705B6
:1072600000203E971305055DFD5583C6D72E858A00
:1072700091EA83A6472F1386472491CA63F4B60088
:107280003285B6859387870BE391E7FE828032854E
:107290008280370700209306C73881471307C73815
:1072A000414683C546266389A50085079386860BDC
:1072B000E399C7FE014582801305800BB387A702BF
:1072C000938747243305F7008280EF82DFF0AA8995
:1072D000370500209304C53805690144138A442604
:1072E000130909B81146CE8533058A00EF202064C2
:1072F00019E51304840BE31724FF6F801FF11305B6
:1073000044242695DDBF370700201306C738814780
:1073100081461307C73821488348460B6397A80066
:10732000850693F6F60F63E9D500850713068603F5
:10733000E39407FF0145828013058003B387A7020A
:10734000938747083305F7008280EF82DFE8370430
:1073500000209304044175712A89AE898146130483
:1073600004417D572146DC58ADEB37D60000B7B558
:10737000000037D500004A8713068671938505669D
:1073800013050572EF2030042684130600028145A0
:107390002285EF80FFE8CA85130600022285EF20D0
:1073A000B03B93040402CE8541462685EF20605A07
:1073B0002810EFF0BFAC4146A6852810EFF09FB231
:1073C0002C002810EFF09FC41C842308F402EF1057
:1073D000D06348D849616F805FE38385040099EDED
:1073E00037D60000B7B5000037D500004A8713062E
:1073F0008671938505661305C57669B763F4E70062
:1074000026843E87850693848403E39EC6F4B5BF35
:10741000EF829FDB37E5000013054581370400202C
:1074200037E90000B7E90000EF20500E1304C4381C
:10743000814437EA0000B7EA000037EB0000B7EB01
:1074400000001309C980938909818327442F638C25
:10745000070CA68513054A82EF20E07693054424A5
:1074600013850A83EF202076130600029305442635
:107470001305CB83EF80FFF6130600029305442823
:1074800013854B84EF80FFF537E5000013058599E0
:10749000EF2060730326842A8325442A37E5000001
:1074A0001305C584EF20207237E5000013054586DB
:1074B000EF2060718345D42E37E500001305058960
:1074C000EF2060708345E42E37C50000130505BD2D
:1074D000EF20606F8347F42ECA8591E3CE8537E5B0
:1074E00000001305458AEF20006E8325042F37E541
:1074F00000001305C58BEF20006D8325442F37E571
:1075000000001305C58DEF20006C8325842F37E51F
:1075100000001305858FEF20006B37E50000130591
:107520000591EF20406A8504C1471304840BE39E54
:10753000F4F06F80FFCC7D151375F50F8D4763E96F
:10754000A700B5679387C7690A053E950841828001
:1075500037D500001305857B8280EF827FC901113A
:10756000B7D50000130600029385057C0A85EF203D
:10757000403EB7050020370500200A869385053B6D
:1075800013050539EFC06F98370400201304C43881
:10759000854723A001762302F404B7D50000938722
:1075A000017623A2070023A4070023A607009385E2
:1075B000057E13850176EF201018B7D5000037053A
:1075C00000209385C57E1305153DEF20D016D147C9
:1075D000230AF406B757D433938707753CDC930727
:1075E0008030231EF4069147230FF4068564B70705
:1075F0009808C1074146A294930544071385C19892
:107600002320F408239304DEEF20A034B96537D596
:107610000000938585931305C57FEFF01FD3B565F3
:1076200037E500009385C56813054580EFF0FFD16D
:10763000930710102392F4DEB757DF029387475B5E
:107640003CD4B7E703019387C7C97CD49967938774
:1076500087B63CD805616F80FFBBEF827FB9B7D496
:107660000000B7B5000037D50000138684719385FC
:1076700045491305C56AEF2000555D260145252BB8
:107680001384C19872248305040048408146EF00AA
:10769000D03A05CD37C4000037D500001386847179
:1076A000930584181305056CEF20E05137D90000CD
:1076B0001305803EEF10305B1386847193058418A8
:1076C0001305C96EEF202050E5B7562430240C3442
:1076D0000824014885470147EF0050716F809FB330
:1076E00001A0B707EFBE37E700E0938707083CC764
:1076F00001A0EF827FAD69710945EF10007DEF10A9
:10770000001FEF10B053116585451105EF103021B2
:1077100037140140930700208D4413050480FC803A
:107720000C08E14726CA3ECCEF10E06C93070040FE
:1077300013050480FC800C08914726CA3ECCEF104C
:10774000806BF1673744014093870720130504805D
:107750003ECE6C08B7070C003ED202D023140102C3
:10776000EF10D041854513050480EF10304A37E50E
:10777000000013054597EF200045B707002083A6BA
:10778000071F37C40000B7B4000037E50000130638
:10779000040E9385046613050598EF20C042EF1090
:1077A000E064AA8637E500001306040E938504669C
:1077B0001305C599EF202041EFF03FDAEFF0FFE924
:1077C000EFF0FF86EFB06FBAEF10302423AEA18048
:1077D0001306400381451385C194EF807FA40145C2
:1077E000EF80FFDE0547371A00202382E182814ABD
:1077F000014BB7EB000037EC0000130ACA38B7445E
:1078000001409305000213850480EF1090428547E4
:107810006313F50E13850480EF1030419314850136
:10782000E1849307D0046391F408B7B5000037E50D
:1078300000001306040E9385C54E1305859BEF20AB
:10784000803837E600009305400B5687DA87130629
:10785000469D6810EF20206185456810EFA00FE578
:10786000930730046399F408B7040020938404411B
:107870008149A14C8387040095C3D45885C203C7AE
:1078800004032686CE851385CBA7EF20C03341465F
:10789000938504021305CC83EF80BFB485099384DC
:1078A0008403E39999FD81A8930700036392F4028E
:1078B000B7B5000037E500001306040E9385C54EEA
:1078C0001305459EEF2020300145EF805FD049BF72
:1078D00093076004639EF40AB7B5000037E5000023
:1078E0001306040E9385C54E130585A0EF20A02D29
:1078F0000545EF80DFCD9306F1001306E100930507
:10790000D1006810EFA0AFFD31CD565637E500002D
:10791000AC18130585ABEF80DFAC8307F10083065D
:10792000D1001387C1943EB776A30307E100B7B532
:10793000000037E500001306040E9385C54E1305BD
:1079400045ACEF2040286810EFA0CFE983474ADE1E
:1079500081C76810EFA05FDB1306401081456810F7
:10796000EF801F8CA12CAA8609CDB7B5000037E5A2
:1079700000001306040E93854549130505B0EF205A
:10798000802493871A0033B757013A9BBE8A85BD7E
:107990009307E0046395F400EFF09FA7A9BF930756
:1079A0004004E39FF4EAEF10500637E600002AD6C1
:1079B0005687DA871306C6A29305400B13052103E9
:1079C00023180102EF20204A37E50000130505A522
:1079D000EF20601F370500206C101305055DEF9048
:1079E0002FED11BFEF82DF808387E18285C3AA86F6
:1079F00037E60000B7C5000037E500001306C6BC37
:107A000093858518130545BDEF20E01B37E4000082
:107A1000130544BFEF20201B0545EF10D024CDBF38
:107A2000EF826FFB0111A387018285453705420074
:107A30002387018202C002C202C402C602C802CA6F
:107A400002CC231E0100EF10606F0565854513050C
:107A5000C505EF10C06C37140140C1490D4AC1473C
:107A60008A85130504807C804EC452C2EF10A03872
:107A70006149930700028A85130504807C804AC40B
:107A800052C2EF1040379144930700048A851305D2
:107A900004807C8026C4EF100036930700088A8596
:107AA000130504807C80372401404AC452C2EF1081
:107AB000803485478A85130504807C804EC4EF108E
:107AC000803389478A85130504807C8026C4EF10A3
:107AD00080328A8513050480648026C4EF10A031AB
:107AE000A1478A85130504807C804EC4EF10A03026
:107AF000B70704013EC6B70700023ECA6C009D47A7
:107B000037350140FC864ACC02C8EF10900005468C
:107B100013050480A145EF10A03A85453735014093
:107B2000EF10100305616F804FEEEF82CFEAAA8459
:107B3000371501402E89328AC1450146130505805B
:107B4000EF1000380144631C44013715014005461D
:107B5000C14513050580EF10A0366F800FEB930928
:107B6000F00F63060900B307890083C90700894540
:107B700037350140EF10E07F7DD9CE8537350140A4
:107B8000EF10A07E854537350140EF10807E7DD90E
:107B900037350140EF10A07D81C4B387840088A3EE
:107BA000050455B7EF82CFE42E86AA850145EFF094
:107BB000DFF76F802FE62387A182828003A50183F0
:107BC0008280EF824FE1AA84B729014005452E8AC1
:107BD00032840149EF1030099389098063079900C5
:107BE00089454E85EF10202D09ED37250140894547
:107BF00013050580EF10202C11E9054422856F80C4
:107C0000CFE02945EF1030060509C9BF37E600006F
:107C100037E500002687D2861306C6BC01CCB7C55F
:107C20000000938585181305C5E2EF10D079514502
:107C3000EFF05FDBB7B50000938545491305C5E25A
:107C4000EF10707865BFEF82AFDA2945EF10B00111
:107C5000372401400146A14513050480EF1040265A
:107C60005145EF105000130504800546A145EF1063
:107C7000202537E60000B7B5000037E50000130601
:107C8000C6BC93854549130505CEEF10D073294531
:107C9000EF10607DB7E50000056505469385C5CF0B
:107CA00013058538EFF0FFF16F80CFD6EF82CFD18B
:107CB00085642E8B0144014993848438854BB7EA4F
:107CC000000037BA0000B7E90000254C4A86DA8583
:107CD0002685EFF01FEF63027503A2861386CABCE8
:107CE00093054A49138509E6EF10F06D2945EF1019
:107CF00080770504A9476314F4006F806FD0E31701
:107D000084FD0549E1B7EF822FCCAA892E8A05654B
:107D1000B7E500004111B28A938545F40546130585
:107D20008538EFF01FEA8387E182A1E3B5475686E5
:107D30005C80D28593D7890013053100DC80230154
:107D40003101EF10104193853A000A85EFF09FE56D
:107D5000B7E5000005650146938585F5130585386F
:107D6000EFF03FE641016F80AFC9B7E4000037B9DB
:107D7000000037E50000CE861386C4BC9305C94ECB
:107D80001305C5F6EF1030645284338B4A01B7EB0C
:107D90000000E30D64F914201386C4BC9305C94E9A
:107DA00013854BF9EF1030620504E5B7EF82AFC2DF
:107DB000AA892E840565B7E500000111B284938578
:107DC00085C4054613058538EFF0BFDF8387E18260
:107DD00037EA00001389E182B7BA000081CF37E5A6
:107DE0000000CE861306CABC9385CA4E1305C5C5CE
:107DF000EF10705D3946814513052100EF804FC2B9
:107E0000F5475C8093D78900DC808307090002C8AE
:107E100002CA02CC02CE2301310199CB37E5000022
:107E20001306CABC9385CA4E130505C8EF10B05996
:107E3000138644008A850808EFF03FCF37E500003D
:107E40001306CABC9385CA4E1305C5C9EF10B057B7
:107E500026864C082285EF10D02F8307090091C792
:107E6000A29437E90000631F9400B7E500000565A0
:107E70000146938545CB13058538EFF09FD4056106
:107E80006F80AFB814201306CABC9385CA4E130581
:107E900089CCEF1050530504F9B7EF826FB541114B
:107EA0002A8405469305F10013056073A3070100BA
:107EB000EFF0DFEF988785469377B70F6304D40020
:107EC000936747009305F100054613056073DC874F
:107ED000EFF07FE341016F80EFB3EF826FB1AA84CF
:107EE0002E890565B7E5000041113284938585EF41
:107EF000054613058538EFF0DFCC8387E18285C323
:107F000037E60000B7B5000037E50000A686130687
:107F1000C6BC9385C54E1305C5F0EF10D04A228626
:107F2000CA85130511004480EF10B0228A8513061C
:107F300014002E85EFF07FBF8880A9471374E500F9
:107F400063EE87028547B397870013F7075409EB61
:107F500013F517083335A0003305A0401374F50F4F
:107F6000B7E5000005650146938505F313058538DF
:107F7000EFF03FC5228541016F80CFA90144CDB705
:107F8000EF820FA42A8BAE8B328C854437E9000038
:107F900037BD0000B7ED0000B7BA000037EA0000B7
:107FA000A9496286DE855A85EFF03FF38387E18237
:107FB0002A8491CBAA861306C9BC93050D66138546
:107FC0008DE8EF10504015CC2687A2861306C9BC59
:107FD00093854A4913050AEA8504EF10D03EE392DF
:107FE00034FDB7C5000037E50000A2861306C9BC02
:107FF00093858518130505EDEF10F03C5545EFF01E
:108000007F9E6F80AF9FEF82AF9E4111C88793051F
:10801000F100054613050008EFF09FF641016F805F
:108020006F9FEF82EF9C1307206741118147630226
:10803000E5041307606D8547630DE5021307A07320
:1080400089476308E50205679306C78F8D4763027A
:10805000D5029306479C9147630DD500930627B23E
:1080600095476308D5001307C7C19D476313E50013
:1080700099475C869307803EB385F50291679387A5
:1080800097D0114613057009B3D5F50293D70501B2
:10809000DC8693978500C205C181A181DD8D6C8747
:1080A0006C00EFF0FFED41016F80CF96EF824F94AF
:1080B0004111C8879305F100054613059008EFF0BC
:1080C0003FEC41016F800F95EF828F924111C8877D
:1080D0009305F10005461305D009EFF07FEA410151
:1080E0006F804F93EF82CF90B7F7A43593870790B7
:1080F000411163FFA700FD779387179E7C866C0074
:10810000094613058009EFF0BFE741016F808F90AA
:10811000B707AA329387078863F6A700F977938792
:1081200077BDE9BFB747E52D9387074863F6A700FA
:10813000F1779387175CD9B7B7176B1B938707B095
:1081400063F6A700E177938757174DBFB707551917
:10815000938707C4E3F5A7FA9D679387B7F679BFBE
:10816000EF820F8941112A84EFF0DFF73756E801DB
:108170008146130606801315940193557400EF1081
:10818000E03A935785015C8693570501DC86931787
:1081900085004205418121815D8D68876C00114613
:1081A00013056008EFF0DFDD41016F80AF86EF82DD
:1081B0002F844111C8879305F10005461305600916
:1081C000EFF01FDC41016F80EF84EF826F8241117D
:1081D0004886CC8609466C001305F008EFF05FDA9C
:1081E00041016F802F83EF82AF8075574111F557A2
:1081F0006343E500AA8793968701E1865947635355
:10820000D700D947CC8609466C001305E0085C8688
:10821000EFF01FD741016F70FFFFEF727FFD41113B
:108220004886CC8650876C00114613055009D487C8
:10823000EFF01FD541016F70FFFDEF72FFF8F557AA
:108240002A8B4111B28A368A755563C3F5002E8593
:10825000131785016187D94763D3E7005945931404
:108260008501EFF05F9E09466C0013050074EFF086
:10827000FFB300869C86B7E9000022043E944204C6
:10828000418037B9000037E50000A2861386C9BCDB
:108290009305C94E1305C5B1EF10F0128967938796
:1082A000474BE184CE8B6307F4028567938747428F
:1082B0006302F402B7C5000037E500001386C9BCAD
:1082C00093858518130585B3EF10F00F41454101E3
:1082D0006F701FF337E500001386CBBC9305C94EC2
:1082E0001305C5B6EF10300E0145EFF0DFD105459F
:1082F000EFF09FDD63880A00856593858538568594
:10830000EFF03FD21305F007EFF05FDA37E500003A
:10831000D2861386CBBC9305C94E130585B8EF10E2
:10832000900A014563130A000545EFF05FE88145B7
:108330000145EFF09FE9854601469D451145EFF067
:10834000DFED0565E14705469305B1001305758E20
:10835000DC85EFF05F9B91452685EFF0DFE85A85DD
:10836000EFF01FE00145A5B7EF729FE89317850076
:1083700021815D8D93978500A181DD8D9317860006
:10838000218241115D8E93978600A18268846C855D
:108390007086DD8E2C00214621457487EFF05FBE8C
:1083A00041016F703FE7EF72BFE42A84AA8637E687
:1083B0000000B7B5000037E5000041111306C6BC48
:1083C0009385C54E130585D4EF10E07F09ECA30714
:1083D00001009305F10005461305F009EFF05FBABF
:1083E00041016F703FE38547DC87E5B7EF725FE0DF
:1083F0004111C8879305F10005461305000AEFF007
:108400003FB841016F701FE1EF729FDE4111C887D5
:108410009305F10005461305A008EFF07FB6410172
:108420006F705FDFEF72DFDC41114886CC865087CA
:108430006C0011461305B008D487EFF07FB44101FA
:108440006F705FDDEF72DFDA9317850021814111D4
:108450005D8D68866C0009460945EFF07FB24101E9
:108460006F705FDBEF72DFD82A89AE840565B7E5F0
:1084700000004111938505C0130585383284EFF063
:10848000FF828387E18285C337E60000B7B500002D
:1084900037E50000CA861306C6BC9385C54E130592
:1084A00045C1EF1040728A8502C0130614002E8564
:1084B00002C202C402C623002101EFF00FE781C807
:1084C00019C42286930511002685EF1080480545C2
:1084D000EF007079B7E5000005650146938585C317
:1084E00013058538EFF0EFED41016F70BFD2EF72E9
:1084F0003FD041112A89AE8432846C001146514527
:10850000EFF05FF69C878583B307F0402300F90006
:108510001C871397870161876348070089839CA0A4
:1085200018A041016F701FCF938707F08987C5BFDF
:10853000EF721FCC41119305F10005461305000CA5
:10854000EFF05FF2888741016F70DFCCEF725FCA96
:108550008387E18241112A8485C3AA8637E6000019
:10856000B7B5000037E500001306C6BC9385C54EBD
:10857000130545D0EF1020650145EFF0DFA89357B4
:1085800004015C860D46935784006C001305200897
:108590004087DC862944EFF0BF9E93040005EFF08E
:1085A0003FF9137505076307950005457D14EF0036
:1085B000906B75F4EFF0DFF713750507930700056F
:1085C0006303F50237E60000B7C5000037E5000099
:1085D0001306C6BC93858518130585D2EF10A05EDF
:1085E0004945EFF02FC041016F70DFC2EF725FC0ED
:1085F00001112A840145B6843ACA3EC842C62ECE2D
:1086000032CCEFF05FDA0145EFF05FDE0545EFF0C9
:10861000BFDF6246F24581462285EFF0BFE09396C8
:1086200084005247A180D58C2394918293868182C5
:108630003248C24725C30546B0A2B8B2333500015F
:10864000B337F000DCA2C8B2EFF03F85938581829A
:1086500019461305C008EFF0BF92814601468145D7
:108660001305F03FEFF05FD037E60000B7B500002C
:1086700037E500001306C6BC9385C54E130585BAC1
:10868000EF106054370500017D15EFF03FEC0561F8
:108690006F705FB8130700F0BAA24DB7EF725FB505
:1086A0008387E18241112A899384E18285C3AA8666
:1086B00037E60000B7B5000037E500001306C6BC7A
:1086C0009385C54E1305C5D7EF10E04F0145EFF078
:1086D0009F93838704004164130404A03304890238
:1086E0008DC337E60000B7B5000037E500002287EC
:1086F000CA861306C6BC9385C54E130545DAEF102E
:10870000804C935704010D4621806C0013053008FE
:108710005C86C08623070100EFF09F8683870400F4
:1087200099CF37E60000B7B5000037E50000130623
:10873000C6BC938505661305C5DCEF10C0485144DF
:1087400013090006EFF0DFDE137505076307250147
:1087500005457D14EF00305175F48387040099CFEF
:1087600037E60000B7B5000037E500001306C6BCC9
:108770009385C54E130545DFEF10E044EFF05FDB56
:1087800013750507930700066303F50237E600003B
:10879000B7C5000037E500001306C6BC93858518F1
:1087A0001305C5E0EF1020424D45EFF0AFA34101A6
:1087B0006F705FA6EF72DFA341116C000D46494553
:1087C000EFF05FCA9C860887A2075D8D41016F703C
:1087D0007FA4EF72FFA141112E84AA846C000D4684
:1087E0004D45EFF03FC89C869CA01C871CA0410112
:1087F0006F705FA2B71702409843B706FFF04111B0
:108800001367170098C3D84337060200758FD8C383
:108810009843B706F7FEFD16758F98C39843B706C1
:10882000FCFFFD16758F98C3D843B70601FFFD16F0
:10883000758FD8C39843B70600ECFD16758F98C3A3
:108840003707FF0098C723A6070202C402C6984351
:10885000C166558F98C3B716024005679C42F18FD9
:108860003EC6A24785073EC4B24781E7A247E397C9
:10887000E7FEB71702409C431397E70063570706CC
:1088800085473EC632478547631FF704B717024046
:10889000D843B706C1FFFD16D8C3D843D8C3D843C1
:1088A00013670740D8C3D843758FD8C3D843B706DA
:1088B0002900558FD8C39843B7060001558F98C338
:1088C000984393166700E3DD06FED843B7160240CF
:1088D000719BD8C3D84313672700D8C32147DC4214
:1088E000B18BE39EE7FE4101828002C661BFB716ED
:1088F0000240D842B70700201146318B9387071FEB
:108900006305C70021466308C70237177A001307BB
:10891000072098C337170240584311839376F70016
:10892000370700201307070036971423984333575F
:10893000D70098C38280D842D442416649833D8B98
:10894000F18E1306270015CF3D47630FE60241471E
:10895000630FE602454781456313E6004146A1E205
:108960003747024003270780418B0DC737177A002E
:10897000130707203306C70290C3C9DD9843058358
:1089800049BF81454946E1BF85453546C9BF814557
:108990003D46F1B737173D0013070790E1BF371584
:1089A000024058559316F700585563DF06041183AB
:1089B0003D8B9306170037177A00130707203357AC
:1089C000D70298C35455A182BD8A8DE295463307DC
:1089D000D702058398C337170240585794433D8BFD
:1089E000050733D7E60298C3984369B705456394F2
:1089F000A600E546E9BF3D456396A600D14633870C
:108A0000E602C9BF8906E5BF3D8B930617003717FD
:108A10007A00130707203357D702F1B701A09781D7
:108A2000FF1F938121FD17F1FF1F1301A15D176542
:108A300000001305E5829775FF1F9385A55C1386DB
:108A4000818163FAC5008322050023A0550011052A
:108A50009105E3EAC5FE13858181938501796377EA
:108A6000B500232005001105E36DB5FEFD427390AE
:108A700002BCAD4273904280B762000093828208CC
:108A8000739002309772FFFF9382025893E2320094
:108A900073905230EFF01FD697F2FFFF9382A2C57A
:108AA0007390123473002030EF728FF4B7270140B7
:108AB00093870740631CF500854513050020712D41
:108AC000814513050020512D6F70CFF4B737014059
:108AD00093870780E31AF5FE854513050040B52D01
:108AE000814513050040C5B75C413707F1E0130726
:108AF000F7EF944D7D8F9C41D58FD44DD58FD441C8
:108B0000A206D58FD98F5CC11C4537F7F1FF13073B
:108B1000D77FD4457D8F9C49D58F94458606D58FC8
:108B2000D98F1CC55C55370710FF7D177D8FDC2959
:108B3000FD1793F7F70FD207D98F5CD582801C45BC
:108B400089C593E717001CC58280F99BEDBF1C45C2
:108B500093E787001CC5828008450D8105898280C6
:108B60001C4593E747001CC582800845098105899B
:108B700082801C4591C537075000D98F1CC5828063
:108B80003707B0FF7D17F98FD5BFA54763F7B70447
:108B90008D47138765FF3307F7020328C5009D47FC
:108BA000B397E70093C7F7FFB3F70701B396E60063
:108BB000DD8E54C5994763E3C70495477D16330698
:108BC000F6025859FD47B397C70093C7F7FFF98FCF
:108BD0003396C5005D8E50D982800D473387E502FC
:108BE000032805019D47B397E70093C7F7FFB3F745
:108BF0000701B396E600DD8E14C96DBFB14763E28D
:108C0000C702954765163306F6021859FD47B39714
:108C1000C70093C7F7FFF98F3396C5005D8E10D953
:108C2000828095474D163306F6025855FD47B39797
:108C3000C70093C7F7FFF98FB395C500DD8D4CD5FD
:108C400082806845420541818280B7270140938731
:108C50000740984711C5B7068000558F98C7828096
:108C6000B70680FFFD16758FD5BF08416D8D333572
:108C7000A00082805C4191C537070004D98F5CC198
:108C80008280370700FC7D17F98FD5BFEF724FD672
:108C900001112A8423040100A5441C8463F9F4040F
:108CA00023040100A54621461C8463FFF606231514
:108CB00001002304010095461C8463F1F60E3885FB
:108CC0003C8599460D46B3F7D70205651305058027
:108CD000B3D7C7023357D702BA97C207C1837C857F
:108CE0003C8505611D8D420541856F70AFD21C44E6
:108CF00093E787001CC42285EFF01FE66DFD1C443E
:108D000093E747001CC42285EFF03FE66DFD7844F1
:108D10001C8414108607B6972396E7FE1C848507EB
:108D200093F7F70F5C8495BFA30401009C846378DC
:108D3000F6001C84850793F7F70F5C84B5B7988419
:108D40009C840C100607850786072E97AE9703575D
:108D5000C7FE83D7C7FE63FDE7029C848607AE97F4
:108D600083D7C7FE7C859C84988485078607AE9749
:108D700083D5C7FE931717001810BA972396B7FE2E
:108D80009C8438850C1085078607AE972396E7FEEE
:108D90009C84850793F7F70FDC8449BF1C8410106F
:108DA000388589078607B29783D7C7FEBA97C20767
:108DB000C1837C851C84850793F7F70F5C84EDBD28
:108DC000EF720FC305454D2E01457D266F708FC490
:108DD0004111B777004002C6938707C03EC6B2472D
:108DE0003E952AC6B2478CC341018280B7F7FF1F68
:108DF00003A5477082809C4513F7070113F8F7001D
:108E000001C7D8413368E8008E2113F7F50F39C345
:108E100018418146854E3D4F930F80029302800496
:108E2000214E3396DE00B3F8C50063111603939804
:108E3000260033131F011343F3FF3377E300B31806
:108E4000180133E7E800639FF70550C98506E39AE8
:108E5000C6FD18C11307F00F6375B70454412146CE
:108E6000854E3D4F930F800293028004414EB3988C
:108E7000CE0033F715016392E8021317260001179D
:108E80003313EF001343F3FFB376D3003317E80037
:108E9000D98E639DF701232A15010506E319C6FD46
:108EA00054C18280E39457FA10C94DB7E39757FE37
:108EB00023281501DDB708456D8D3335A00082806C
:108EC00019C20CC982804CC9828023AAA1828280E7
:108ED00003A74183894710216311F70214318D479D
:108EE00063EDD7003C219A0637E700E09607D58F5F
:108EF00093F7F70F32972300F740544105479357F4
:108F000056003317C70089CA938707048A07B7E654
:108F100000E0B69798C3828093870706B7E600E023
:108F20008A07B69798C30F100000828037770040F9
:108F30001C4309C593E707101CC3828093F7F7EF22
:108F4000E5BFB7160240DC4251777D17F98F5D8D82
:108F5000C8C28280B717024023800702238007021D
:108F600005476306E50011476306E500828023801C
:108F7000A702828015472380E702828037170240CC
:108F80001C535D8D08D3828001C9371702401C53E2
:108F9000A166D58F1CD38280B71602409C526177A0
:108FA0007D17F98F9CD28280371702405C4391462F
:108FB000B18B6385D700A1466382D706B7177A00C5
:108FC000938707201CC1371602405C4237070020F8
:108FD000130707019183BD8BBA9794231C41B3D724
:108FE000D7005CC15442A1829D8ABA969422B3D61E
:108FF000D70014C55442AD829D8A36971823B3D743
:10900000E7005CC558423983937637001387418067
:1090100036971823B3D7E7021CC982805C435843B4
:10902000C166C983758FB7F6FF1F83A6C670BD8B57
:1090300089071396160163480600C54601466392E8
:10904000D702C94739A88946638FD702BD46638EC8
:10905000D702C146638ED702C54601466393D70047
:10906000C1471DEF3747024003270780418B05C7E3
:1090700037177A0013070720B307F7021CC121D660
:109080001C41858381B701466DBF0546B547D1BFF9
:109090000146BD47F9B737173D0013070790E9BFF1
:1090A000B7150240D8559316F700D85563DF06046C
:1090B00011833D8B9306170037177A00130707209B
:1090C0003357D70218C1D455A182BD8A8DE2954687
:1090D0003307D702058318C1371702405857144188
:1090E0003D8B050733D7E60218C1184171B7854596
:1090F0006394B600E546E9BFBD456396B600D14628
:109100003387E602C9BF8906E5BF3D8B930617008A
:1091100037177A00130707203357D702F1B799C5DD
:10912000371702401C4F5D8D08CF8280B717024071
:10913000984F1345F5FF798D88CF828099C53717F1
:1091400002405C4F5D8D48CF8280B7170240D84FF8
:109150001345F5FF798DC8CF828099C53717024036
:109160005C475D8D48C78280B7170240D8471345DA
:10917000F5FF798DC8C7828001C9371702401C539B
:10918000C166D58F1CD38280B71602409C524177AE
:109190007D17F98F9CD282809357550005476399BC
:1091A000E700B71702409C4333D5A70005898280AA
:1091B00009476396E700B71702409C53F5B7B71706
:1091C0000240DC53D5B7B737004003D7078089C5C5
:1091D000598D2390A78082801345F5FF798DD5BFE7
:1091E000B737004003D74780136707012392E78012
:1091F00082803737004083574780C207C183BD9BB9
:10920000C207C1832312F78082803736004083561D
:1092100086810357868142074183E31AD7FE37369A
:1092200000408356C6818357C681C207C183E39A33
:10923000D7FEB735004003D6858103D58581420529
:109240004181E31AC5FE630CA700B736004003D77F
:10925000C68183D7C681C207C183E39AE7FE420570
:109260005D8D8280EF62DFF841112AC6EFF05FF773
:109270003245B7370040135705014205239CE7806C
:109280004181239EA780EFF0DFF641016F609FF8D8
:10929000EF621FF641112AC6EFF09FF43245B7374F
:1092A0000040135705013D8B42052394E78041811F
:1092B0002396A780EFF0FFF341016F60BFF53737CA
:1092C00000408357478093F70702E5DF82803737F6
:1092D000004083574780C207C183DD9BC207C1831B
:1092E0002312F7803737004083574780A18BEDDF8B
:1092F0008280B737004003D747801345F5FF798D4B
:109300002392A7808280EF62BFEEEFF09FFE6F6036
:109310007FF01A218D6793870704B6217D8F9E21E8
:10932000D58FD621D58FF621D58F9625D58FB62509
:10933000D58FD625D58FF625D58FD98F1EA15A2D3D
:10934000FD779387F77FF98F5EAD9E291EA98280F6
:109350001E2189C593E707041EA18280C207C1832D
:1093600093F7F7FBC207C183C5BF4EA582804A258C
:1093700082800A256D8D3335A0008280EF625FE721
:109380001629F577FD17F58FF621DA257971D58F36
:109390001EA95625FD779387379FF58FD6212A84FE
:1093A0002EC6D58F9625D58FB625D58F5EA55E297D
:1093B000C207C18393F7F7CFD98F5EA96808EFF092
:1093C000BFBEB747014093870780B245631EF402D2
:1093D000A2576547B387E7029841930640060A07FC
:1093E000B3D7E70233D7D702B3F7D70212079207F2
:1093F00093872703B3D7D702BD8BD98FC207C18309
:109400001EA445616F601FE19257E1B791C55E25CB
:109410000967D98F5EA582805A25F977FD17F98FE4
:10942000D5BF93F5F51F4EA182804A211375F51F14
:1094300082800A216D8D3335A0008280B70700201D
:1094400083A7071F37177A0013070720B3D7E70250
:1094500093F7F70F238DF1821307803EB387E7025E
:10946000239CF1828280B7F700E0D8438146799B44
:10947000D8C303D781833306A70290CBD4CB9843BC
:109480001367070198C398431367170298C3D8431B
:10949000058B75DF9843799B98C38280EF62BFD3B9
:1094A000B7440140AE893289014493840480634506
:1094B00024014A856F607FD5930500042685EFF06F
:1094C0005FF77DD9B387890083850700268505046A
:1094D000C205C181EFF0FFF4D9BF138781801C431F
:1094E000938601793E95636BD500B78600209386FD
:1094F000068063E5A60008C33E858280FD57EDBF68
:1095000011CE93070002918F635BF000B395C50005
:10951000B357F5003316C500DD8D32858280930583
:1095200006FE0146B315B5003285CDBFB687B288B9
:109530002A832E88639B061463F8C50A4167636B10
:10954000E61AB70700016360F63493568601E147D7
:1095500017570000130707A636971823BA97130763
:1095600000021D8F19CB3398E500B357F500B318EF
:10957000E60033E807013313E50013D6080133553D
:10958000C80293960801C182935703013377C8023A
:10959000B385A60242073368F700637AB80046989D
:1095A0009307F5FF636418016365B8303E8533089F
:1095B000B8403357C8024203135303013378C8023B
:1095C000B386E602420833686800637BD800469899
:1095D0009307F7FF6365180179176363D8003E8727
:1095E0004205598D8145828001E60547B358C7027F
:1095F000416763E8E80EB707000163EAF82893D6ED
:109600008801E147175700001307C79A36971423BC
:10961000BE9693070002958FFDE7939E080133875E
:10962000154113DF080193DE0E01854593570301B1
:109630003355E7033377E703B306D5034207D98FE2
:1096400063FAD700C6971307F5FF63E4170163E5D4
:10965000D7263A85958F33D7E70342031353030187
:10966000B3F7E703B30ED703C207B3E7670063FBA3
:10967000D701C6979306F7FF63E51701791763E3F0
:10968000D70136874205598D828063E1D504C167D1
:1096900063E1F604B707000163E3F61E13D7860102
:1096A0006148975700009387E790BA979823130E65
:1096B00000024297330EEE40631A0E0C63EDB61CA7
:1096C0003335C5001345150081458280814501452C
:1096D00082809307F00F63F3D71C13D786002148CD
:1096E000C9B71307F00FC686E37E17F193D688003B
:1096F000A14709BF1307F00FB286E37BC7E4935677
:109700008600A147B1B5B398F80033D6D50013DF72
:109710000801335EE6033397F500B356D500558F45
:10972000939E080193DE0E013313F5009355070154
:10973000B376E603B387CE03C206CD8E63FBF60095
:10974000C6961306FEFF63E4161763F2F616791E3B
:10975000C6969D8E33D6E60393170701C183B3F6F1
:10976000E6033385CE02139706015D8F637BA70066
:1097700046979307F6FF636817136376A712791667
:10978000469793150E01098FD18D4DB5B357E6005D
:10979000B396C601DD8E33D3E50013DF0601B35760
:1097A000E303939E060193DE0E013398C501335700
:1097B000E50033680701935808013316C601337377
:1097C000E303B385FE024203B368130163FBB800F1
:1097D000B6981387F7FF63EAD80C63F8B80CF9174B
:1097E000B698B388B84033D7E80342081358080145
:1097F000B3F8E8033383EE02C208B3E5080163FB64
:109800006500B6951308F7FF63EDD50863FB65089F
:109810007917B695C207416FD98F1307FFFFB3F6CB
:10982000E70093D80701718F4182B38EE602B385BA
:109830006540B386C60213D80E013387E802BA9694
:10984000C2963386C80263F3E6007A9693D806017F
:10985000469663E2C5026385C5003E8581458280E8
:1098600041677D17F98EC206B3FEEE003315C501C0
:10987000F696E374D5FE1385F7FF8145828013D7F2
:109880000601414839BD93560601C147D1B193D66F
:109890000801C14785BB814505458280368701485F
:1098A00009B5428785BF3E86E9BDBA871DBF328EA6
:1098B0004DB579154698E5B97915C69761BB411143
:1098C000194506C69D230545EF10103929468145E7
:1098D0006F00607E0325C50E82809387C1809C4304
:1098E0009C5389E79767FF1F9387C77303A5C70E2C
:1098F00082809387C180AA858843E5AA91ED4111B2
:109900006C00014501CA795591C61C229CC10822F0
:109910003335A00041018280014509CA795599C6B5
:109920001C229CC108223335A0008280828001471E
:109930006314E60001458280B307E5000507B3869E
:10994000E5009C2383C6F6FFE384D7FE3385D7402A
:109950008280B3C7A5008D8B3307C50081E78D4793
:1099600063EDC700AA87637EE50894218507850516
:10997000A38FD7FEE3EBE7FE828093763500AA87BC
:1099800089CA942185078505A38FD7FE93F63700F2
:10999000C5BF9376C7FF138606FE63F0C70683A391
:1099A000050083A2450083AF850003AFC50083AEE9
:1099B000050103AE450103A3850183A8C501938575
:1099C000450223A0770003A8C5FF23A2570023A4C4
:1099D000F70123A6E70123A8D70123AAC70123ACD7
:1099E000670023AE17019387470223AE07FF75B7C1
:1099F00090419107910523AEC7FEE3EBD7FEE3E666
:109A0000E7F6828063F1A504B386C500637DD502C5
:109A10009345F6FF8147FD176393F50082803387F6
:109A2000F600034807003387C7002A972300070181
:109A3000DDB73387F50014233307F500850714A33A
:109A4000E319F6FE82808147E5BFDDC183A7C5FF2C
:109A5000411122C406C626C21384C5FF63D3070082
:109A60003E94AA84EF00B04F9387C1839C4381EF5B
:109A70002322040023AE81822244B24026859244F0
:109A800041016F00F04D637EF40014403307D400B1
:109A90006396E7009843DC43369718C05CC0D9BF93
:109AA000BA87D84319C3E37DE4FE94433386D700D5
:109AB000631F86001040B29694C33386D700E31D1F
:109AC000C7FA10435843B29694C3D8C375B76375A9
:109AD000C400B1479CC04DB71040B306C400631624
:109AE000D70014435843B29614C058C0C0C369B7D6
:109AF0008280011126CA93843500F19806CE22CCCB
:109B00004AC84EC6A104B14763F3F404B14463E20A
:109B1000B4042A89EF00B0449387C18398433A8400
:109B200039E0938701849C4391E781454A85852CE0
:109B300023A0A184A6854A859D24FD596319350774
:109B4000B1472320F9004A85EF00904129A0E3D0D6
:109B500004FCB1471CC10145F2406244D244424971
:109B6000B249056182801C40858F63CF0702AD46F4
:109B700063F6F6001CC03E9404C031A05C40631341
:109B8000870223AEF1824A85EF00903D1305B400B1
:109B90009307440061993307F5405DDF3A94898F5C
:109BA0001CC05DBF5CC3C5B72287404095BF13048E
:109BB00035007198E30285FCB305A4404A85C522AF
:109BC000E31C35FBB5BF39713EDA2ED232D436D61E
:109BD0003AD842DC46DE9387C18022CC804326CA35
:109BE00006CEAA8411C41C4C81E72285EF00101117
:109BF0000C4454102686228536C6EF001072F240BF
:109C00006244D2442161828001119387C18022CCB9
:109C1000804306CEAA8501C81C4C91E72AC622853E
:109C2000EF00D00DB245104422856244F240056138
:109C30006F102052011126CA4AC806CE22CC4EC649
:109C400052C4AA842E8909C51C4D99E3EF00100B5C
:109C50009C4C804481E72685EF00500A974700001E
:109C600093874758631BF402C0405E24A18BB1C7A1
:109C70001C48A1C7FD59294A1C4483450900FD170A
:109C8000B1E91CC463DD07062286A9452685992112
:109C9000FD576308F502294535A0974700009387D3
:109CA00067566314F4008044C9B797470000938750
:109CB0006751E31CF4FAC0444DBFA2852685C5292F
:109CC00055D97D55F2406244D2444249B249224AB4
:109CD000056182801CC4050963D70700184C63CA5C
:109CE000E700638845011C401387170018C08CA348
:109CF00061B722862685F92EE31035F9D9B71C40C5
:109D00001387170018C0294798A371B79387C1809C
:109D1000AA8588436FF01FF241119387C18022C446
:109D2000804306C61C5C95EB6145EFF09FBCB737DE
:109D3000CDAB08DC9387E7301CC1B7176DE693877E
:109D400047235CC1B7E705009387C7EE1CC5AD4745
:109D50005EA50547814718C95CC9105C3787954CDB
:109D6000B7F75158144A484A1307D7F29387D74296
:109D7000B387F602B24022443305E5023E95B3872D
:109D8000E60233B7E6029386170014CA2A9733B562
:109D9000F6003A9548CA06050581410182804111C5
:109DA00022C42A842E8523A6017806C6EFF0EFF29E
:109DB000FD576317F5009387C1789C4391C31CC07E
:109DC000B240224441018280FD4763F6B700D94783
:109DD0001CC17D5582807C41011122CC06CE2E868D
:109DE0002A8491C713972500BA97984319EB2285C7
:109DF00032C68528AA85228562443246F240056132
:109E00001DA8854601456308D700FD566319D70094
:109E1000D9471CC00545F2406244056182802E8509
:109E200023A0070002970145FDB79387C180AA854B
:109E300088436FF07FF9411122C42A842E85B285B0
:109E400023A6017806C6EF10E05EFD576317F50004
:109E50009387C1789C4391C31CC0B2402244410106
:109E600082806F10A05B35713ECBA6DA36C73AC947
:109E700042CD46CF9387C18086DEA2DC844363DB7C
:109E800005009307B0089CC07D55F6506654D65423
:109E90000D61828093078020FC822AC42ACC8147EE
:109EA00099C19387F5FF3EC83ECE7401FD572E84BD
:109EB00026852C00FC8336C2EF00F018FD57635551
:109EC000F5009307B0089CC069D0A2472380070023
:109ED0006DBF35713ECBB707008093C7F7FF3ECE0D
:109EE0003EC8C1779387872032C536C73AC942CD6D
:109EF00046CF3ECA9387C1802AC42ACC8843340106
:109F00002E862C0086DE36C2EF00F013A247238097
:109F10000700F6500D618280AA8798239386170068
:109F200009EB850503C7F5FF8507A38FE7FE75FBE2
:109F30008280B687DDB7AA87982185078505A38F1C
:109F4000E7FE7DFB8280AA87850703C7F7FF6DFFC9
:109F50003385A7407D158280AA8709CA850503C776
:109F6000F5FF85077D16A38FE7FE65FB3E9663939D
:109F7000C70082808507A38F07FED5BF79714AD0BD
:109F80004ECE06D622D426D2AA892E899304190051
:109F900003C4F4FF3A8536C632C42EC23AC0EFF08D
:109FA0007F9322951C3102479245A18B2246B246EF
:109FB000D1E39307D0026311F4089C200543930476
:109FC0002900E5C641476390E60213070003639C3E
:109FD000E7009C201307800593F7F70D6392E70CC9
:109FE0009C30C1468904B70800806314030093C8FD
:109FF000F8FF33FFD80201480145A54FE54EFD5259
:10A0000033DED802138707FD63E3EF04BA8763DE0C
:10A01000D704630D58007D58636AAE006314AE0028
:10A020006346FF0005483385A6023E95850483C735
:10A03000F4FFC9BF268999BF9307B0026305F400F6
:10A04000A2870143BDBF9C2093042900DDBF138775
:10A05000F7FB63E5EE00938797FC55BF1387F7F98D
:10A0600063E5EE00938797FA5DB7FD57631FF8002D
:10A070009307200223A0F900468519EEB25022541E
:10A0800092540259F249456182806304030033050A
:10A09000A0406DD6630408009385F4FF0CC2F9BF9D
:10A0A00093070003A9F2A1463DBF13070003E38213
:10A0B000E7F2A9460DBF9387C1809C43B2869853AF
:10A0C00009E71767FF1F1307E7F52E86AA853E8568
:10A0D0006FF0DFEA011122CC26CA4AC806CE4EC66E
:10A0E000AA842E89328401C51C4D91E3012997472A
:10A0F00000009387270F6317F406C0401C4C1CC454
:10A100005E24A18BC1C31C48B5CF1C48084093797D
:10A11000F90F1379F90F1D8D5C486346F500A28590
:10A120002685752C25E51C440505FD171CC41C401F
:10A130001387170018C0238037015C486388A70085
:10A140005E24858B81CBA9476316F900A2852685FD
:10A1500079240DEDF24062444A85D2444249B24925
:10A1600005618280974700009387C7096314F40054
:10A17000804469B7974700009387C704E310F4F859
:10A18000C044ADBFA28526851D2041D17D59D9B7D8
:10A1900089CD9307F00F63F7C7009307A0081CC190
:10A1A0007D55828090A105458280014582804111C4
:10A1B0009387C18026C2844322C44AC006C62A8926
:10A1C0002E8489C49C4C99E326850D2E9747000068
:10A1D00093874701631BF402C0400317C400931721
:10A1E0000701C18393F68700B5EA93F6070195EE60
:10A1F000A5472320F900136707045AA47D55B240F0
:10A20000224492440249410182809747000093878B
:10A2100067FF6314F4008044C9B797470000938731
:10A2200067FAE31CF4FAC0444DBF918B85C74C58C4
:10A2300091C9930744046385F5004A85EFF0FF80D8
:10A24000232A04025E242322040093F7B7FD5EA4B0
:10A250001C481CC05E2493E787005EA41C4899EB51
:10A260005E241307002093F707286385E700A28583
:10A270004A85A1295E2413F717001DC35C482324D7
:10A280000400B307F0401CCC1C480145ADFB83170C
:10A29000C40013F7070825D793E707045EA4B9BFE6
:10A2A000898B014791E3584818C4F9BFDE25011195
:10A2B00022CC26CA06CE4AC84EC613F78700AA8407
:10A2C0002E8461EFD841634DE000B841634AE0005D
:10A2D0000145F2406244D2444249B249056182805C
:10A2E00058547DD703A904009396370123A0040096
:10A2F00063DC060670485E24918B99C75C401D8E16
:10A300005C5899C33C401D8E5C540C508146268598
:10A310008297FD575A24631DF5009440F54763E981
:10A32000D706B70740208507B3D7D700858BADC3C5
:10A330001C48232204001CC09317370163D8070070
:10A34000FD576314F5009C4091E368C84C5823A066
:10A350002401BDDD930744046385F5002685EFF0F5
:10A36000CFEE232A0402ADB70C5001468546268560
:10A370000297FD572A86E310F5F89C40ADDF75473C
:10A380006385E70059476393E70423A0240189B755
:10A39000136707045AA47D552DBF83A90501E389DE
:10A3A00009F203A905008D8B23A03501330939413A
:10A3B000014791E3D84918C4E35C20F11C540C50C8
:10A3C000CA864E86268582976347A0005E2493E75F
:10A3D00007045EA4C9B7AA993309A940F1BF9C49F3
:10A3E000A5C3011122CC06CE2A8411C51C4D81E7DC
:10A3F0002EC62922B245974700009387A7DE639CAB
:10A40000F5004C408397C5009DC722856244F24009
:10A4100005616FF0BFE9974700009387A7DE63945B
:10A42000F5000C44C5B7974700009387A7D9E39B75
:10A43000F5FC4C44C1BFF240624401450561828095
:10A4400001458280411122C406C62A844EA572A508
:10A4500023200500232205002324050023220506CE
:10A4600023280500232A0500232C050021468145C9
:10A470001305C505EF50DFDA971700009387E7D57E
:10A480005CD097170000938707D81CD4971700005B
:10A490009387E7DB5CD497170000938747DE00D0F3
:10A4A0001CD8B24022444101828097050000938568
:10A4B00045F399AA411126C2130680069384F5FF3D
:10A4C000B384C4024AC02E8922C406C693854407B9
:10A4D000EFF02FE22A8401CD23200500232225015D
:10A4E000310508C4138684068145EF507FD3228549
:10A4F000B240224492440249410182801C4DA5E7AA
:10A50000411106C622C497070000938747FA1CD55D
:10A51000938701819C4323240504232605042328D3
:10A5200005046314F50085471CCD2A84352848C0EE
:10A5300022851D2808C42285052848C448400146B4
:10A540009145EFF03FF008440546A545EFF09FEF39
:10A5500048440946C945EFF0FFEE85471CCCB240A0
:10A56000224441018280828041119387018126C269
:10A5700084434AC006C69C4C22C42A8981E72685AA
:10A58000EFF0DFF7938484048044DC40FD1763D64A
:10A5900007009C40B9CF8440C5BF0317C40039E70A
:10A5A000C177850723220406232004002322040008
:10A5B000232404005CC423280400232A0400232C41
:10A5C0000400214681451305C405EF507FC5232AA9
:10A5D0000402232C040223240404232604042285D9
:10A5E000B24022449244024941018280130484060D
:10A5F00071BF91454A85EFF0FFEB88C049FDB14737
:10A600002320F9000144E1BF797122D44AD052CC11
:10A6100056CA5AC85EC606D626D24ECE2A8AAE8AF8
:10A62000130485040149054BFD5B09ECB25022542B
:10A630004A8592540259F249624AD24A424BB24B7D
:10A6400045618280044483294400FD1963D40900D4
:10A650000040E1BFDE24637BFB008397E400638757
:10A660007701A6855285829A3369A900938484066E
:10A67000E9BF1971A6DAAE848395E500A2DC86DE17
:10A68000328463DB0500DE2423A0060093F707086D
:10A6900085E7930700401DA0300836C6EF00B043A1
:10A6A000B246E34205FE7247BD67F98F7977BA97E4
:10A6B00093B717009CC2F1BF930700041CC0F6506B
:10A6C0006654D654014509618280DE25011122CCF1
:10A6D00006CE26CA4AC8898B2E8489CF9307740474
:10A6E0001CC01CC885475CC8F2406244D244424941
:10A6F0000561828074003000AA84EFF09FF7A245C4
:10A700002A892685EFF0EFBE19E98317C40013F7F5
:10A71000072079FBF19B93E727005EA4C1B7970759
:10A7200000009387C7D89CD45E2408C008C893E76C
:10A7300007085EA4A2475CC8B24781CF8315E40036
:10A740002685EF00F03B11C55E24F19B93E71700CF
:10A750005EA45E243369F9002316240171B7828058
:10A76000828001114AC803A9850022CC52C45AC074
:10A7700006CE26CA4EC656C22E84328B368A63E96E
:10A780002609DE2513F7074851C304408C49584871
:10A79000AA8AB389B4408D44B384E4020947B3C4A0
:10A7A000E402138716004E9763F3E400BA8493F72C
:10A7B0000740BDCFA6855685EFF0AFB32A891DE1CE
:10A7C000B14723A0FA005E247D5593E707045EA4F9
:10A7D000F2406244D2444249B249224A924A024B70
:10A7E000056182800C484E86EFF0AF965E2493F7A9
:10A7F000F7B793E707085EA42328240144C84E99BD
:10A80000B38434412320240104C4528963732A0190
:10A81000528908404A86DA85EFF0CF9E1C440145F4
:10A82000B38727411CC41C403E99232024014DB707
:10A8300026865685EF0090332A895DFD0C485685A3
:10A84000EFF0AFA0B5BFDE25717126D34AD14ECF50
:10A8500006D722D552CD56CB5AC95EC762C566C34C
:10A8600093F70708AA892E89B284B9C39C49A9E342
:10A870009305000436C6EFF0CFA72320A9002328B4
:10A88000A900B24615E1B14723A0F9007D55BA50A1
:10A890002A549A540A59FA496A4ADA4A4A4BBA4B34
:10A8A0002A4C9A4C4D61828093070004232AF900B8
:10A8B00093070002A30CF1029307000302DA230DB1
:10A8C000F10236CE930B5002974A0000938A8A9584
:10A8D000054C294B26841C2099C363997709B30C36
:10A8E0009440638E0C00E6862686CA854E85EFF07E
:10A8F0005FE7FD57630BF518D256E69636DA1C2053
:10A9000063850718FD579304140002D002D63ED287
:10A9100002D4A301010682DC8C2015465685EF0087
:10A92000702313841400825721E513F7070109C728
:10A9300013070002A301E10613F7870009C71307F5
:10A94000B002A301E10694201307A002638AE60285
:10A95000B257268481462546182093051400130714
:10A9600007FD6372E6068DC63ED61DA00504A5B799
:10A97000330555413315AC00C98F3ED0A28469BF61
:10A98000724793064700184336CE634707023AD60C
:10A9900018209307E002631DF70418309307A00204
:10A9A000631BF702F2470904138747009C433ACE22
:10A9B00063C107023ED22DA83307E04093E727008A
:10A9C0003AD63ED0F1B7B387670385462E84BA974F
:10A9D00061B7FD57C5B7050402D2814681472546B8
:10A9E000182093051400130707FD6376E606F9F2B5
:10A9F0000C200D461745000013054583EF00901508
:10AA000011CD97470000938767821D8D930700043F
:10AA1000B397A700025505045D8D2AD00C20194676
:10AA2000174500001305C58093041400230CB102E0
:10AA3000EF00501225C59757FFFF9387A75C95E756
:10AA40000257F2471377071009CF91073ECED2572E
:10AA5000D2973EDA41B5B387670385462E84BA970D
:10AA600041B79D07E19BA107D5B77808970600007D
:10AA7000938666CF4A860C104E8597000000E7004B
:10AA80000000FD572A8AE314F5FC8357C9007D5561
:10AA900093F70704E39D07DE5255D5BB7808970668
:10AAA0000000938646CC4A860C104E851121D1BFFA
:10AAB0001C46FD171CC663DA0700184E63C5E70085
:10AAC000A9476394F5006FF0EFE01C422E851387D1
:10AAD000170018C28CA38280011122CC26CA4AC852
:10AAE0004EC652C406CE2A89AE893284B304D6003B
:10AAF0007D5A63149400014509A80C204E864A85AE
:10AB0000EFF01FFB0504E31645FFF2406244D24418
:10AB10004249B249224A05618280357122CD26CB55
:10AB20004AC94EC706CF52C556C35AC1DEDEE2DC63
:10AB3000E6DAAA89AE843289368409C51C4D99E3C8
:10AB4000EFF0DF9B973700009387C7696399F40C98
:10AB500083A44900DE24A18BEDC79C48FDC3930765
:10AB60000002A304F1029307000302D22305F102BD
:10AB700022C6930B5002973A0000938AAA6A054CAA
:10AB8000294B4A841C2099C36390770FB30C24414E
:10AB9000638E0C00E6864A86A6854E85EFF0DFF3CD
:10ABA000FD576300F51E9256E69636D21C20638A46
:10ABB000071CFD571309140002C802CE3ECA02CC7E
:10ABC000A309010482D48345090015465685EF0088
:10ABD000607813041900C24751E913F7070109C748
:10ABE00013070002A309E10413F7870009C713073D
:10ABF000B002A309E104834609001307A002638F92
:10AC0000E606F2474A84814625461820930514003B
:10AC1000130707FD6377E60AB5CA3ECE85A89737C6
:10AC200000009387275E6395F40083A489001DB715
:10AC30009737000093870759E39EF4F083A4C90077
:10AC400011BFA6854E85EFF08FD611D97D55FA40FC
:10AC50006A44DA444A49BA492A4A9A4A0A4BF65B94
:10AC6000665CD65C0D618280050429BF33055541C1
:10AC70003315AC00C98F3EC82289B1B7324793065D
:10AC80004700184336C6634707023ACE1820930799
:10AC9000E002631DF70418309307A002631BF7025C
:10ACA000B2470904138747009C433AC663C10702B1
:10ACB0003ECA2DA83307E04093E727003ACE3EC8AE
:10ACC000F1B7B387670385462E84BA973DBFFD571A
:10ACD000C5B7050402CA8146814725461820930559
:10ACE0001400130707FD6374E606F9F20C200D4605
:10ACF0001735000013058553B12D11CD973700008E
:10AD00009387C7521D8D93070004B397A700424550
:10AD100005045D8D2AC80C2019461735000013055F
:10AD20002551130914002304B1022D2535C197576D
:10AD3000FFFF9387272D95E74247B2471377071008
:10AD400009CF91073EC69257D2973ED21DBDB38719
:10AD5000670385462E84BA9751B79D07E19BA107EB
:10AD6000D5B7780097060000938646D726860C084C
:10AD70004E8597000000E7000000FD572A8AE31483
:10AD8000F5FCDE2493F70704E39207EC1255C1B5F6
:10AD9000780097060000938666D426860C084E85B8
:10ADA000012AE1BF797156CA9C49BA8A984522D4D2
:10ADB00026D24ECE52CC06D64AD05AC85EC6AA89F2
:10ADC0002E84B284368A63D3E700BA879CC00347D7
:10ADD000340419C385079CC01C4093F7070281C740
:10ADE0009C4089079CC00329040013796900631AF9
:10ADF0000900130B9401FD5B5C449840998F634CF0
:10AE0000F9041C408346340493F70702B336D0009C
:10AE1000A5EB13063404D2854E85829AFD57630351
:10AE2000F5041C4011469840998B54448144639723
:10AE3000C700B384E64063D3040081441C4418482F
:10AE40006354F700998FBE94014969047D5B639850
:10AE50002405014509A885465A86D2854E85829AE1
:10AE6000631E75017D55B250225492540259F24925
:10AE7000624AD24A424BB24B456182800509ADBF5E
:10AE80003307D40013060003A301C7040347540487
:10AE900093871600A2978906A381E7049DBF854684
:10AEA0002286D2854E85829AE30E65FB050945B759
:10AEB000797122D426D24AD04ECE06D652CC56CA6A
:10AEC0005AC8B689942D930790063289AA842E8495
:10AED00013863504638DF60263E2D7069307800577
:10AEE0006386F61863EDD700638E0620930730045F
:10AEF000638EF60A930A24042301D404C9A093079D
:10AF000030066385F60A93074006E395F6FE1C407B
:10AF1000084393F6070893054500C5C61C410CC3BA
:10AF200063D807001307D002B307F040A301E4047D
:10AF30009736000093864630294765A89307000797
:10AF40006382F61663E5D7029307E0066389F61875
:10AF50009307F006E390F6FA0C401C4313F805083B
:10AF6000138547006307080608C39C4385A8930719
:10AF70005007E383F6FE930780076389F612930771
:10AF80003007E399F6F61C43D0418145938647008C
:10AF900014C383AA07005685752E01C53305554194
:10AFA00048C05C401CC8A301040461A81C43930A68
:10AFB0002404938647009C4314C32301F40485476B
:10AFC000D5B793F607041C410CC3B9DAC207C18791
:10AFD00081BF93F5050408C3C9D99E231307F00662
:10AFE0006387E60E97360000938606252947A3015E
:10AFF00004044C400CC463C5050008406D9908C0AA
:10B0000099E3B28A89CDB28AB3F5E702FD1AB69503
:10B010008C212380BA00B3D5E70263F0E70CA14787
:10B02000631EF7001C40858B91CB58401C4863C7BA
:10B03000E70093070003A38FFAFEFD1A330656417B
:10B0400010C84E87CA867000A2852685EFF09FD56E
:10B050007D5A631D450B7D55B250225492540259BE
:10B06000F249624AD24A424B45618280A382D504AA
:10B07000973600009386461C0C40084313F80508D9
:10B080001C411105630D080208C313F7150001C721
:10B0900093E505020CC04147B9FB0C4093F5F5FD63
:10B0A0000CC0B1B79C4193E707029CC1930780078E
:10B0B000A302F404973600009386461975BF13F86F
:10B0C000050408C3E30308FCC207C1837DBF9736AC
:10B0D000000093866616214719BFAE8735B79441A5
:10B0E0001C43CC4913F80608138547006306080083
:10B0F00008C39C438CC339A008C393F606049C4341
:10B10000F5DA8EA323280400B28A25BF1448568698
:10B11000CA8526858299E30045F51C40898B8DE719
:10B12000B2474844E35AF5F23E853DB78546568618
:10B13000CA8526858299E30065F3050A5C44324797
:10B14000998FE345FAFEE9BF014A930A94017D5BBA
:10B15000F5B7011122CC06CE2A8409C91C4D99E706
:10B1600032C62EC4EFF08FB93246A24597370000A1
:10B17000938747076316F60250401C46FD171CC60E
:10B1800063D00704184E63C7E70093F7F50F29470C
:10B190006398E70222856244F24005616FE09FF305
:10B1A00097370000938707066314F6001044F1B741
:10B1B0009737000093870701E311F6FC504475BFF1
:10B1C0001C4213F5F50F1387170018C28CA3F24029
:10B1D000624405618280411122C42E848395E5007A
:10B1E00006C6CD22634905007C48AA977CC8B240B8
:10B1F0002244410182805E247D777D17F98F5EA411
:10B20000FDB7DE25011122CC26CA4AC84EC606CE9D
:10B2100093F70710AA842E843289B68991C7839543
:10B22000E5008946014609225E247D777D17F98F66
:10B230005EA48315E4006244F240CE864A86B24999
:10B2400042492685D244056125A8411122C42E8495
:10B250008395E50006C6C928FD575A24631AF500F0
:10B26000FD77FD17F98F5EA4B24022444101828030
:10B270008567D98F5EA468C8C5BF8395E50005A81A
:10B28000411122C42A842E85B285368623A60178F0
:10B2900006C6EFE0AFA0FD576317F5009387C178AE
:10B2A0009C4391C31CC0B2402244410182804111A1
:10B2B00022C42A842E8523A6017806C6A122FD5722
:10B2C0006317F5009387C1789C4391C31CC0B240BB
:10B2D000224441018280411122C42A842E85B285F4
:10B2E00023A6017806C62D22FD576317F500938724
:10B2F000C1789C4391C31CC0B2402244410182806A
:10B30000411122C42A842E8523A6017806C6292A43
:10B31000FD576317F5009387C1789C4391C31CC008
:10B32000B240224441018280411122C42A842E85E8
:10B33000B285368623A6017806C61922FD57631703
:10B34000F5009387C1789C4391C31CC0B24022444E
:10B350004101828093F5F50F2A966314C5000145DB
:10B3600082801C21E38EB7FE0505C5BF81E5B2854D
:10B370006FE02FF8011122CC06CE26CA4AC84EC66D
:10B38000328401EEEFE06FEC0149F24062444A85FD
:10B39000D2444249B24905618280AE84AA89892893
:10B3A0002689E37485FEA2854E85EFE08FF42A8915
:10B3B00069DDA6852286EFE0CFD9A6854E85EFE030
:10B3C000CFE8E1B7411122C42A842E85B2853686A2
:10B3D00023A6017806C69D28FD576317F5009387BD
:10B3E000C1789C4391C31CC0B24022444101828079
:10B3F00083A7C5FF1385C7FF63D50700AA959C41A6
:10B400003E9582809307800523A6F1787D55828042
:10B410009307800523A6F1787D55828093078005E8
:10B4200023A6F1787D5582809307800523A6F178C5
:10B43000014582809307800523A6F1787D5582809F
:10B440009307800523A6F1787D55828093078005B8
:10B4500023A6F1787D55828001A000002573202865
:10B460006C656E3D2575293A0A000000253034755B
:10B47000202000002530325820000000202020002D
:10B4800025630000253032780000000041647665B5
:10B4900072740000570000005B25735D2025733A2D
:10B4A000204164766572746973656D656E7420669B
:10B4B00072616D6520746F6F2073686F72742028DD
:10B4C0002564203C20313031290D0A005B25735D55
:10B4D0002025733A20496E636F727265637420731E
:10B4E00069676E61747572650D0A0000490000009D
:10B4F0005B25735D2025733A20416476657274691B
:10B5000073656D656E74207369676E6174757265BD
:10B51000206F6B2E0D0A00005B25735D2025733AAA
:10B52000204164766572746973656D656E7420661A
:10B5300072616D652077697468206461746120743C
:10B540006F6F2073686F727420282564203C20255B
:10B5500064290D0A000000006E616D656C657373EF
:10B56000206E6F64650000007265706561746572BD
:10B570000000000073656E736F720000726F6F6D74
:10B58000207365727665720063686174206E6F6403
:10B59000650000006B6E6F776E000000756E6B6E5D
:10B5A0006F776E002573206F6E20256C642077699D
:10B5B00074682074797065202573206F6E20257360
:10B5C000206C6F636174696F6E20256C6420256C3C
:10B5D000640A00005075626C6963206B6579000035
:10B5E0005369676E61747572650000004170706424
:10B5F0006174610054696D657374616D7020697365
:10B6000020256C750A0000004E6F64654E616D6503
:10B610002025730A00000000416E6F6E796D6F7512
:10B6200073206E6F64650000416E6F6E796D6F758B
:10B63000730000005B25735D2025733A204E65770B
:10B6400020616E6F6E796D6F7573206E6F6465200B
:10B65000637265617465643A2025730D0A00000009
:10B66000440000005B25735D2025733A204578690E
:10B670007374696E67206E6F646520666F756E64A3
:10B6800020666F72207075624B65795B305D3D306E
:10B6900078253032580D0A00416E6F6E5265712068
:10B6A0007061796C6F6164005B25735D2025733A6E
:10B6B0002050617373776F7264206C656E206973BC
:10B6C0002025642E0D0A00005B25735D2025733A4A
:10B6D0002050617373776F726420636F7272656359
:10B6E000742C206E6F646520257320617574686505
:10B6F0006E746963617465642E0D0A005B25735D69
:10B700002025733A204C6F67696E20726573706FE5
:10B710006E73652073656E7420746F206E6F646540
:10B720002025732E0D0A00005B25735D2025733ADA
:10B730002050617373776F726420696E636F7272E9
:10B7400065637420666F72206E6F64652025732EAA
:10B750000D0A0000416E6F6E796D6F7573526571E1
:10B76000756573745061796C6F6164206174202514
:10B77000700A0000202064657374696E6174696FDB
:10B780006E20686173683A203078253032580A009C
:10B79000202073656E646572207075624B65793A1E
:10B7A000200000002530325800000000202063698E
:10B7B00070686572204D41433A2030782530345806
:10B7C0000A0000002020646563727970746564204B
:10B7D0007061796C6F6164202825752062797465C9
:10B7E00073293A0A000000002020202074696D654A
:10B7F0007374616D703A2025750A000020202020A6
:10B8000073796E632074696D657374616D703A202D
:10B8100025750A002020202070617373776F726491
:10B820003A200000436F6E74726F6C005B25735D8D
:10B830002025733A205265706C79696E6720746FA9
:10B84000206120646973636F76657220726571751B
:10B850006573742077697468207461672025640DAE
:10B860000A0000003D3D3D20446973636F766572B8
:10B870002052657175657374203D3D3D0A000000DE
:10B880007072656669784F6E6C79203A2025750A6A
:10B89000000000007479706546696C746572203A26
:10B8A000203078253032580A00000000746167208B
:10B8B000202020202020203A2030782530386C5855
:10B8C0000A00000073696E63652020202020203A62
:10B8D0002030782530386C580A0000003D3D3D206E
:10B8E000446973636F76657220526573706F6E730F
:10B8F00065203D3D3D0A00006E6F646554797065BA
:10B90000203A2025750A0000736E72202020202026
:10B91000203A2025750A000074616720202020202D
:10B92000203A2030782530386C580A007075626BE8
:10B9300065792020203A20005B25735D2025733A2D
:10B940002046696E64696E672072656D6F7465204C
:10B950006E6F64652C20736F7572636548617368E0
:10B960002069732025640D0A000000005B25735DCB
:10B970002025733A204E6F6465206E6F7420696EC7
:10B980002044420D0A0000005B25735D2025733AB8
:10B9900020466F756E64206E6F64652077697468E9
:10B9A00020696E6465782025640D0A005B25735D4F
:10B9B0002025733A20484D4143206661696C6564D7
:10B9C000206F6E20656E63727970746564206D659A
:10B9D00073736167652025730D0A00005B25735D35
:10B9E0002025733A20484D41432073756363657386
:10B9F000732066726F6D2025732C20257520627967
:10BA0000746573206C6F6E670D0A000020205479F6
:10BA100070657864643A203078253032580A000026
:10BA200020205061796C6F61644C656E3A202575F9
:10BA30000A0000005B25735D2025733A2050617475
:10BA40006820746F6F206C6F6E670A0D0A0000002B
:10BA500053656E7420726573706F6E73652C2074FD
:10BA600068652074656D70657261747572652069B2
:10BA700073202564206465636963656C73697573FD
:10BA80000A000000506C61696E74657874206D6501
:10BA900073736167652066726F6D2025732C20615A
:10BAA0007474656D70742025642C2074696D6573E1
:10BAB00074616D702025643A20257300506C6169B3
:10BAC0006E74657874206D65737361676520667246
:10BAD0006F6D207365727665722025732C207365F7
:10BAE0006E6465722069732025732C2061747465FF
:10BAF0006D70742025642C2074696D657374616D9C
:10BB0000702025643A202573000000005B25735DDA
:10BB10002025733A20556E6B6E6F776E20746578B2
:10BB20007420747970653A2025640D0A00000000C5
:10BB3000456E637279707465645061796C6F61648D
:10BB40003A0A0000202044657374696E6174696F5D
:10BB50006E486173683A203078253032580A000008
:10BB60002020536F75726365486173683A2030789E
:10BB7000253032580A000000202043697068657241
:10BB80004D41433A203078253034580A00000000F7
:10BB900020205061796C6F61644C656E3A20257A83
:10BBA000750A000020205061796C6F61643A2000B2
:10BBB000526571756573743A0A000000202054695B
:10BBC0006D657374616D703A2025750A0000000080
:10BBD0002020547970653A203078253032580A0098
:10BBE0002020446174613A2000000000202044615C
:10BBF00074610000526573706F6E73653A0A0000DD
:10BC000020205461673A2025750A00006F6E0000FD
:10BC10006F6666004F4B202D207265706561742041
:10BC20006973206E6F77204F4E0000004F4B202D20
:10BC300020726570656174206973206E6F77204F84
:10BC4000464600007265626F6F740000616476653D
:10BC5000727400004F4B202D204164766572742071
:10BC600073656E7400000000636C6561722073740C
:10BC700061747300284F4B202D20737461747320FE
:10BC800072657365742900004A756E203235203262
:10BC90003032360076302E302E31202D2042524E5A
:10BCA0002053797374656D7320524953432D5600A8
:10BCB000257320284275696C643A20257329000099
:10BCC000626F61726400000057434820434833327A
:10BCD0005633303700000000636C6F636B00000068
:10BCE00074696D65200000004F4B202D20636C6F40
:10BCF000636B207365743A20253032643A25303204
:10BD0000643A25303264202D2025642F25642F25A8
:10BD10006420555443000000284552523A20636C79
:10BD20006F636B2063616E6E6F7420676F2062615A
:10BD3000636B77617264732900000000636C6F634A
:10BD40006B2073796E6300004552523A20636C6F2A
:10BD5000636B2063616E6E6F7420676F2062616336
:10BD60006B7761726473000070617373776F7264D4
:10BD70002000000070617373776F7264206E6F77BC
:10BD80003A20257300000000676574200000000061
:10BD900067756573742E70617373776F72640000DA
:10BDA0003E202573000000006E616D6500000000FC
:10BDB00072657065617400006C6174003E202564DA
:10BDC000000000006C6F6E007075626C69632E6B12
:10BDD000657900003E200000726F6C650000000075
:10BDE0006164632E6D756C7469706C6965720000B6
:10BDF0003E2025642E2564003F3F3A202573000035
:10BE00007365742000000000616C6C6F772E7265A2
:10BE100061642E6F6E6C7920000000004F4B0000B3
:10BE200067756573742E70617373776F7264200029
:10BE30006E616D65200000007265706561742000A0
:10BE40006C617420000000006C6F6E200000000028
:10BE5000756E6B6E6F776E20636F6E6669673A20E2
:10BE60002573000073746174732D7061636B657466
:10BE7000730000007B2272656376223A25752C22BE
:10BE800073656E74223A25752C22666C6F6F645F41
:10BE90007478223A25752C226469726563745F7424
:10BEA00078223A25752C22666C6F6F645F72782257
:10BEB0003A25752C226469726563745F7278223A40
:10BEC00025757D0073746174732D726164696F00F0
:10BED0007B226E6F6973655F666C6F6F72223A25A5
:10BEE000642C226C6173745F72737369223A2564E7
:10BEF0002C226C6173745F736E72223A25642E304B
:10BF0000302C2274785F6169725F73656373223AC3
:10BF100025752C2272785F6169725F736563732285
:10BF20003A25757D0000000073746174732D636F92
:10BF3000726500007B22626174746572795F6D7650
:10BF4000223A25752C22757074696D655F7365637F
:10BF500073223A25752C226572726F7273223A250C
:10BF6000752C2271756575655F6C656E223A257555
:10BF70007D000000556E6B6E6F776E20636F6D6D88
:10BF8000616E6400456E637279707465644D6573AB
:10BF900073616765000000005B25735D2025733ABF
:10BFA00020506C61696E206C656E3A2025642C20EF
:10BFB000656E63206C656E3A2025640D0A000000F2
:10BFC000456E63727970746564206672616D650098
:10BFD0005B25735D2025733A20456E63727970741A
:10BFE0006564206672616D652074782066696E698B
:10BFF00073680A0D0A0000005B25735D2025733A03
:10C00000204E6F6465206973206E756C6C0D0A009C
:10C010005B25735D2025733A204E6F64652069733C
:10C02000206E6F7420706F70756C617465640D0A9A
:10C030000000000047726F75704D6573736167652E
:10C04000000000005B25735D2025733A204E6F745D
:10C0500020612067726F757020746578740D0A0016
:10C060005B25735D2025733A204368616E6E656CB5
:10C070002068617368202564206E6F7420666F7578
:10C080006E640D0A000000005B25735D2025733A85
:10C0900020484D4143206661696C6564206F6E20C5
:10C0A00067726F757068617368206B6579202564AD
:10C0B0000D0A00004D6573736167652066726F6DD0
:10C0C000206368616E6E656C2025733A2025730AC3
:10C0D00000000000547844756D70446563000000F2
:10C0E0004D657368436F7265000000005B25735DEA
:10C0F0002025733A204672616D6520746F6F206E43
:10C1000065772C20676F742076657273696F6E2077
:10C11000256420696E7374656164206F6620300D3C
:10C120000A00000020205479706578643A20307845
:10C13000253032580A0000005B25735D2025733AD4
:10C140002050726F636573736564206672616D65FC
:10C150000D0A0000CE2100001E2200003422000043
:10C160004C2200006222000080260000942600007D
:10C17000AA260000B6260000CC2600004D65736894
:10C180006672616D696E6700450000005B25735D36
:10C190002025733A20256420697320746F6F206214
:10C1A000696720666F72207378313236320D0A006B
:10C1B000737461727420577269746542756666653E
:10C1C00072000000656E642057726974654275667E
:10C1D000666572005B25735D2025733A20545820F4
:10C1E0007061796C6F61644C656E3D25752070617E
:10C1F00074684C656E3D257520746F74616C4C6578
:10C200006E3D2575206865616465723D3078253026
:10C2100032580D0A000000005B25735D2025733A3B
:10C22000205374617274696E67207478206D6F6436
:10C23000652C2073656E742025642C2073686F75DF
:10C240006C642025640D0A005B25735D2025733A1C
:10C250002053657454782072756E6E696E670D0A8E
:10C26000000000005B25735D2025733A2069727120
:10C270003A203078253034580D0A00005B25735D74
:10C280002025733A2046696E697368656420747866
:10C290000D0A000073746172742052656164427506
:10C2A0006666657200000000656E64205265616418
:10C2B00042756666657200007472616E73706F72AB
:10C2C0007420666C6F6F6400666C6F6F64000000B2
:10C2D00064697265637400007472616E73706F726A
:10C2E0007420646972656374000000002C20706122
:10C2F000796C6F6164207479706520697320000027
:10C300007265717565737400726573706F6E7365B5
:10C310000000000074657874206D65737361676553
:10C320000000000061636B6E6F776C656467656D1C
:10C33000656E740067726F757020746578740000A4
:10C3400067726F757020646174610000616E6F6E5A
:10C350002072657175657374000000007061746807
:10C360000000000074726163650000006D756C74FC
:10C370006970617274000000636F6E74726F6C009C
:10C38000726177002C207061796C6F616420766532
:10C390007273696F6E20697320257320000000009E
:10C3A0005472616E73706F727420636F6465733A58
:10C3B0002025642025640A00506174682069732078
:10C3C0002564206E6F646573206C6F6E67000000DB
:10C3D0006E6F6465202564202D20253032582C2076
:10C3E000000000001F1C1F1E1F1E1F1F1E1F1E1FE0
:10C3F0004A616E4665624D61724170724D61794A63
:10C40000756E4A756C4175675365704F63744E6FF6
:10C410007644656300000000000303060104060281
:10C42000050003050000000022AE28D7982F8A429D
:10C43000CD65EF23914437712F3B4DECCFFBC0B559
:10C44000BCDB8981A5DBB5E938B548F35BC2563959
:10C4500019D005B6F111F1599B4F19AFA4823F9243
:10C4600018816DDAD55E1CAB420203A398AA07D8E7
:10C47000BE6F7045015B83128CB2E44EBE853124E1
:10C48000E2B4FFD5C37D0C556F897BF2745DBE723B
:10C49000B196163BFEB1DE803512C725A706DC9BA0
:10C4A000942669CF74F19BC1D24AF19EC1699BE485
:10C4B000E3254F388647BEEFB5D58C8BC69DC10F9F
:10C4C000659CAC77CCA10C2475022B596F2CE92DFF
:10C4D00083E4A66EAA84744AD4FB41BDDCA9B05C97
:10C4E000B5531183DA88F976ABDF66EE52513E9888
:10C4F0001032B42D6DC631A83F21FB98C82703B078
:10C50000E40EEFBEC77F59BFC28FA83DF30BE0C654
:10C5100025A70A934791A7D56F8203E05163CA0606
:10C52000706E0E0A67292914FC2FD246850AB72798
:10C5300026C9265C38211B2EED2AC45AFC6D2C4DD1
:10C54000DFB3959D130D3853DE63AF8B54730A65CB
:10C55000A8B2773CBB0A6A76E6AEED472EC9C28127
:10C560003B358214852C72926403F14CA1E8BFA282
:10C57000013042BC4B661AA89197F8D0708B4BC221
:10C5800030BE5406A3516CC71852EFD619E892D1A9
:10C5900010A96555240699D62A20715785350EF4C1
:10C5A000B8D1BB3270A06A10C8D0D2B816C1A419D5
:10C5B00053AB4151086C371E99EB8EDF4C774827FF
:10C5C000A8489BE1B5BCB034635AC9C5B30C1C394B
:10C5D000CB8A41E34AAAD84E73E363774FCA9C5B88
:10C5E000A3B8B2D6F36F2E68FCB2EF5DEE828F7403
:10C5F000602F17436F63A57872ABF0A11478C884DD
:10C60000EC39641A0802C78C281E6323FAFFBE9017
:10C61000E9BD82DEEB6C50A41579C6B2F7A3F9BE72
:10C620002B5372E3F27871C69C6126EACE3E27CA8C
:10C6300007C2C021C7B886D11EEBE0CDD67DDAEAAD
:10C6400078D16EEE7F4F7DF5BA6F1772AA67F0064C
:10C65000A698C8A2C57D630AAE0DF9BE04983F1125
:10C660001B471C13350B711B847D0423F577DB28D6
:10C670009324C7407BABCA32BCBEC9150ABE9E3CE0
:10C680004C0D109CC4671D43B6423ECBBED4C54C76
:10C690002A7E65FC9C297F59ECFAD63AAB6FCB5FBA
:10C6A0001758474A8C19446C08C9BCF367E6096AF5
:10C6B0003BA7CA8485AE67BB2BF894FE72F36E3C31
:10C6C000F1361D5F3AF54FA5D182E6AD7F520E518E
:10C6D0001F6C3E2B8C68059B6BBD41FBABD9831F48
:10C6E00079217E1319CDE05B59F1B2FE0AE5A6FF70
:10C6F0007BDD2AFE1E14D4005280030030D1F300EB
:10C70000777940FF32E39CFF006EC501671B900004
:10C71000EDD3F55C1A631258D69CF7A2DEF9DE144D
:10C7200000000000000000000000000000000010F9
:10C730008F64F8016360BCFFC509F8FFD588650008
:10C7400073840E00A061A0FF144BB1FF9DBE6A0070
:10C750003EA4ADFFF56995FFEE3F3D00374F6A00FF
:10C76000703B49FFC26C3C00C5197A003E484E0040
:10C77000C41EDFFFAE03E3FFC36918FE683409FF80
:10C780008D49F800EC6B73FF9A0C6B015E290B006E
:10C790004B3276FEE4E2C9FF78446A009A40B7FF64
:10C7A000517DA700C55C99008FA626004990BEFF69
:10C7B000C8A68AFEB3FB42FFBDC432FFC8E5DD0058
:10C7C0000D7AC4009FFFD30074EAE500682583005A
:10C7D0001D4C32013BA34EFFCF4C300086CE37FFBD
:10C7E000003EC900F0E74FFF33F25BFF514532FFD7
:10C7F0004A7DC3012F8721004E75EFFF8D89B4005C
:10C80000B5095C008494D6000C0BE100267D83FF03
:10C81000A0CFC3FE542DB30002A6DE01F0D2C800A3
:10C820006C491F000B779DFF7FC8E900107750000F
:10C8300094DB8401AEE60100E47AEAFE59B493FF8A
:10C84000DBE499FF082621FF14A59700C900210009
:10C850000609A2FF70E3E5FF944A41007D59D8FF25
:10C860008018A3FE0C9E92FFA0DB8CFE053CB3005B
:10C8700048C0A5FEFC4826FFAD065B009D2D8F003D
:10C880002DF23701F05359003712AF014DEAEAFF9C
:10C8900072A35AFF3A51D100565E7EFF2AF9F90081
:10C8A00054B49100FD23B4FFDD75BBFF3D75C4FF9B
:10C8B00070555E0021313CFFF14F9601109F9E00A4
:10C8C0001802A10159170EFFB4BB7500860485003C
:10C8D000E26173FFF8B520FFEA3BBA01C281A9FF0C
:10C8E0002C824000E4B10300395D35FF282186FF2A
:10C8F00090A993FF34BC8500AACA5FFE8F402F0029
:10C9000053DBC401CD8374FF959C3B00DAE5AB009B
:10C91000CDDBB500B85AEF00750BF1FE6CD654FFB5
:10C92000D9A25BFEAD0D4A00C56F61FE3FDF670017
:10C930008DDB6800DF95EFFF8E7445FE4362D50006
:10C940007C4E62FE9E98D6FF5FE2AC01E59235FF19
:10C9500076EB5D00927AE60027FF350044598DFFA3
:10C960007632D700796AAB002BF005FE6A998D000C
:10C97000083DD901F2254200A01BE4FF670D4600E7
:10C980008906D5000020C300CE6A1600279900FF53
:10C9900058D3FD0128C0D4008E7B7B00100E7AFF97
:10C9A00077A255FF92F01500D0A657010662D5FF79
:10C9B0008167DE0148A5B6FF3C897DFE4F763C00CD
:10C9C0007E5EBF009D9270FF63845DFE9288790059
:10C9D000936294FEA78D54004B5C77FE094097FF4D
:10C9E00018E86B01A3602E00266C74FFA0E65B00C4
:10C9F0002B945DFEB997A100DB328201DAD1E7FF0B
:10CA000030CAA1FE740A4D004926DB019418FDFFCF
:10CA100051CED5FE7A71F6FF1F2EF5FE4B0C04FFAA
:10CA20000F5AE0FECCDC39FF66386CFF9A06E00056
:10CA30001034D1018BC3750073C05AFF21F39200EB
:10CA40007532CE01584D5FFF2ED257FEA73B2DFF0A
:10CA5000FBEC5800539FF500B1238AFE9B8CB80075
:10CA6000D42071002FABAE00CF1FAC013DA0E4FF7E
:10CA7000EB8129FF90844200EFA89101BCBE230006
:10CA8000CF04B2FE3239E7FF347FA3FFD226200065
:10CA900055B149FEB0E28900D1A5D4FE2BCB38FFB9
:10CAA00050DB3AFE5647E20093DDB9FF39FBD80070
:10CAB000C7E235FE7D192D00948AB8002C0D2FFF9A
:10CAC0003B57A5FF91896B004724CFFFD4EDDB00D6
:10CAD0002C0148FFCB7C05FF792076FFB8C291FF7F
:10CAE000B0448D00C459150090D4CF016642A9FF0F
:10CAF000A7FC97FF4189DCFF4BC5A7FECCE50100F1
:10CB000002E51201E9C47F007C143101E0351E000A
:10CB10005BF3E4FE83A08A0011439D0030270600EA
:10CB20005570E200AAFF9200CE2381005B8380FF54
:10CB300077B625FF2FD4DF00B653910100022B00FA
:10CB4000449AA5FEE803CFFF84F32CFF8C53D3FF58
:10CB50003FE106FF98202AFF6E76C500F1B602007D
:10CB60008BA1B9003B69DBFF6A9644FF0EDA94FFA4
:10CB70009D5F9700DA3DD1FFF57715FEAEAC2C0036
:10CB800074AE5501795E1DFFE7802900C546FA00A5
:10CB90009F9291FF50D4B7FF02FC2800816F9CFF49
:10CBA000EE158EFE8DC50CFFC7CEA0FF27E3D60085
:10CBB000B55099005D96BA009CAC2EFEBF413BFF7C
:10CBC00053B155FFCD013600807C50FF3CA4FB00E3
:10CBD000F2A25FFEFEA61AFF590691FF09DC0CFFC8
:10CBE000EE540D0199E2080004DFF2FF9F22FDFFE1
:10CBF0003CC847FF01FC5CFF8372C9FED064ED00B6
:10CC000073E025FE4B6AB3FF901EA0FF8684DDFF14
:10CC100039ADB8FF3FD3B9FF689AC1FFE8C0BD0086
:10CC200021BB22FE9B2D10002F765F0056EC9F004B
:10CC30004E582CFF3CEB1E001466B1FE9B2AD6FF1B
:10CC4000F846DBFF546585FF7E3C7000FC12F00067
:10CC50006A409BFE6B4672001F086900649B0A00D5
:10CC6000EBF46101AA289300AAE301FE8842AD001B
:10CC700032C5CCFE597A61005FE881FF726C7EFF9D
:10CC8000B2428AFFA96530FFE2C62FFF262EE100DF
:10CC90004183D7FEEC9D1BFFEC129E002A3E57FFFE
:10CCA000654BB1FEAB5DB8009F4954FFF6B60CFF73
:10CCB000404D9900E59E5200430A7B01A7657B0029
:10CCC000AAD899FFB395960084BDF100ED6D08FFD9
:10CCD000E71593008B38B4009EAB91FE8AC971FFB3
:10CCE000E9B43B00419869FF1D330F009DD27AFFE4
:10CCF0006EE777FFA6E428FFE39B6E00D4C5DC0057
:10CD00005CF5800165CC79FF63E8DA0016807D0070
:10CD1000CB7A6100CD6C92FF7AB2620071EE7AFF3D
:10CD20001BB6EC00F794EB00F2087000B20265FF4E
:10CD30002EBD12014F2291FFFF5B2100A0884A0007
:10CD40004733A50025E26C00B24227FF80D5500092
:10CD5000528CA6FF3A5FA4FF5BB5AC0145A340002F
:10CD60004A4627FFECE21D001565FFFEDB8C3A000A
:10CD700002E8ABFF32F036FF09853CFE0949BC00F2
:10CD80003EDAE900D6AF0CFF7F8579FF5C01A90090
:10CD90000ECED4FEE560C6FFA0F4B2005488920027
:10CDA000833BB9FF590FAFFFD98E88FF54942900F8
:10CDB0005FA0DC01914200FFF81691FF9CD3E100D7
:10CDC00050E547FEBCDC4900B62948FF701F75FFDF
:10CDD000A8F1E9FFD1D30500BA5327FE83DF03FF93
:10CDE0002CB11300974AC30063C19F01EE8362FF19
:10CDF000A2B5E100607522FF36E75000588B7AFF3C
:10CE00003A0FCCFF7BAEC0FF231463FE9106A40053
:10CE1000173486016052A0FF33BB15FF38B8F40009
:10CE2000B47D1100C67D000072626601CD439200A0
:10CE30004B1D7901E75BEAFFD9CE2E010C4E0400B1
:10CE4000D5B3F3FE73E8A70053A717FE7D8ED6FF78
:10CE500012285D0061E4E5FF8469BFFE8DC9DA0038
:10CE6000717D7A007EFC7C0035A3E5FE87C543FF1B
:10CE7000F61D8001BF9BA5FF81B0EB00243172003D
:10CE800007842FFE14BA9800535228FFB54DC0FFF7
:10CE9000B9599C00090A20FF9FFCFF01F92D2AFFC8
:10CEA000EE896401531CE600386386FF71EF74005D
:10CEB000853B8C01BDF124FFF825C30160DC370000
:10CEC000B74C3EFFC3423D00324CA401E1A44CFFED
:10CED0004C3DA3FF753E1F00519140FF76410E006F
:10CEE000A273D6FF068A2E007CE6F4FF0A8A8F0022
:10CEF000341AC200B8F44C00818F2901BEF413FF2C
:10CF00007BAA7AFF6281440079D5930056651EFFA3
:10CF1000A1679B008C5943FFEFE5BE01430BB500B1
:10CF2000C6F089FEEE45BCFF4397EE00132A6CFF66
:10CF3000E5557101324487FF116A0900326701FF2C
:10CF40005001A80123981EFF10A8B9013859E8FF25
:10CF500065D2FC0029FA4700CCAA4FFF0E2EEFFF46
:10CF6000504DEF00BDD64BFF118DF90026504CFF00
:10CF7000BE55750056E4AA009CD8D001C3CFA4FFCB
:10CF800096424CFFAFE110FF8D5062014CDBF20086
:10CF9000C6A272002EDA98009B2BF1FE9BA068FFC0
:10CFA00033BBA5000211AF004254A001F73A1E00A6
:10CFB000234135FE45ECBF002D86F501A37BDD0046
:10CFC000206E14FF3417A500BAD64700E9B0600000
:10CFD000F2EF360139598A00530054FF88A06400EB
:10CFE0005C8E78FE687CBE00B5B13EFFFA29550024
:10CFF00098822A0160FCF60097973FFEEF853E007D
:10D0000020389C002DA7BDFF8E85B3018356D30029
:10D01000BBB396FEFAAA0EFFD2A34E0025349700AA
:10D02000634D1A00EE9CD5FFD5C0D101492E5400A6
:10D030001441290136CE4F00C98392FEAA6F18FF12
:10D04000B12132FEAB26CBFF4EF77400D1DD990043
:10D050008580B2013A2C1900C9273B01BD13FC00A1
:10D0600031E5D20175BB7500B5B3B8010072DB00C4
:10D07000305E9300F52938007D0DCCFEF4AD7700CD
:10D080002CDD20FE54EA1400F9A0C601EC7EEAFF74
:10D090002F63A8FEAAE299FF66B3D800E28D7AFF5B
:10D0A0007A4299FEB6F58600E3E41901D639EBFF22
:10D0B000D8AD38FFB5E7D20077809DFF815F88FF4C
:10D0C0006E7E330002A9B7FF078262FE45B05EFFA5
:10D0D0007404E301D9F291FFCAAD1F01690127FF72
:10D0E0002EAF4500E42F3AFFD7E045FECF3845FF8D
:10D0F00010FE8BFF17CFD4FFCA147EFF5FD560FFF1
:10D1000009B02100C805CFFFF12A80FE2321C0FF0E
:10D11000F8E5C40181117800FB6797FF073470FFC1
:10D120008C3842FF28E2F5FFD94625FEACD609FF30
:10D130004843860192C0D6FF2C26700044B84BFFAE
:10D14000CE5AFB0095EB8D00B5AA3A0074F4EF00BF
:10D150005C9D020066AD6200E98960017F31CB0011
:10D16000059B9400179409FFD37A0C0022861AFFBE
:10D17000DBCC8800860829FFE0532BFE5519F70009
:10D180006D7F00FEA9883000EE77DBFFE7ADD500AC
:10D19000CE12FEFE08BA07FF7E0907016F2A48007B
:10D1A0006F34ECFE603F8D0093BF7FFECD4EC0FF1D
:10D1B0000E6AED01BBDB4C00AFF3BBFE6959AD005D
:10D1C00055195901A2F394000276D1FE219E09005F
:10D1D0008BA32EFF5D4628006C2A8EFE6FFC8EFF0F
:10D1E0009BDF900033E5A7FF49FC9BFF5E740CFFBB
:10D1F00098A0DAFF9CEE25FFB3EACFFFC500B3FF8E
:10D200009AA48D00E1C468000A2319FED1D4F2FF6C
:10D2100061FDDEFEB865E500DE127F01A48887FFB0
:10D220001ECF8CFE9261F30081C01AFEC95421FF0B
:10D230006F0A4EFF9351B2FF04041800A1EED7FF0E
:10D24000068D210035D70EFF29B5D0FFE78B9D0055
:10D25000B3CBDDFFFFB97100BDE2ACFF7142D6FF79
:10D26000CA3E2DFF664008FF4EAE10FE857544FF96
:10D27000B67859FF8572D300BD6E15FF0F0A6A009C
:10D2800029C0010098E879FFBC3CA0FF9971CEFF4E
:10D2900000B7E2FEB40D48FF0100000000000000EE
:10D2A000000000000000000000000000000000007E
:10D2B000000000000000000000000000000000006E
:10D2C000F7E97A2E8D31092C6BCE7B51EF7C6F0AFA
:10D2D0000000000000000000000000000000000846
:10D2E0008E4ACC46BA18766BB8E7BE39FAAD77638A
:10D2F000FFFFFFFFFFFFFFFFFFFFFFFFFFFFFF0736
:10D300001B132C0AA3E59CEDA72963085D210621C8
:10D31000EBFFFFFFFFFFFFFFFFFFFFFFFFFFFFFF31
:10D320000F000000B0A00EFED3C986FF9E188F002C
:10D330007F693500600CBD00A7D7FBFF9F4C80FEC6
:10D340006A65E1FF1EFC0400920CAE0001000000C3
:10D3500000000000000000000000000000000000CD
:10D360000000000000000000000000008D01020429
:10D3700008102040801B3600637C777BF26B6FC502
:10D380003001672BFED7AB76CA82C97DFA5947F0C8
:10D39000ADD4A2AF9CA472C0B7FD9326363FF7CCA4
:10D3A00034A5E5F171D8311504C723C31896059A41
:10D3B000071280E2EB27B27509832C1A1B6E5AA064
:10D3C000523BD6B329E32F8453D100ED20FCB15B4F
:10D3D0006ACBBE394A4C58CFD0EFAAFB434D3385B8
:10D3E00045F9027F503C9FA851A3408F929D38F58C
:10D3F000BCB6DA2110FFF3D2CD0C13EC5F974417C3
:10D40000C4A77E3D645D197360814FDC222A908839
:10D4100046EEB814DE5E0BDBE0323A0A4906245CC5
:10D42000C2D3AC629195E479E7C8376D8DD54EA92A
:10D430006C56F4EA657AAE08BA78252E1CA6B4C6F6
:10D44000E8DD741F4BBD8B8A703EB5664803F60E4F
:10D45000613557B986C11D9EE1F8981169D98E943E
:10D460009B1E87E9CE5528DF8CA1890DBFE6426857
:10D4700041992D0FB054BB1652096AD53036A538E4
:10D48000BF40A39E81F3D7FB7CE339829B2FFF87AC
:10D49000348E4344C4DEE9CB547B9432A6C2233D90
:10D4A000EE4C950B42FAC34E082EA16628D924B241
:10D4B000765BA2496D8BD12572F8F6648668981662
:10D4C000D4A45CCC5D65B6926C704850FDEDB9DAC1
:10D4D0005E154657A78D9D8490D8AB008CBCD30AAF
:10D4E000F7E45805B8B34506D02C1E8FCA3F0F028B
:10D4F000C1AFBD0301138A6B3A9111414F67DCEA5A
:10D5000097F2CFCEF0B4E67396AC7422E7AD3585D2
:10D51000E2F937E81C75DF6E47F11A711D29C589DC
:10D520006FB7620EAA18BE1BFC563E4BC6D27920BE
:10D530009ADBC0FE78CD5AF41FDDA8338807C731C7
:10D54000B11210592780EC5F60517FA919B54A0DBF
:10D550002DE57A9F93C99CEFA0E03B4DAE2AF5B034
:10D56000C8EBBB3C83539961172B047EBA77D62650
:10D57000E169146355210C7D982F8A4291443771DB
:10D58000CFFBC0B5A5DBB5E95BC25639F111F15946
:10D59000A4823F92D55E1CAB98AA07D8015B831288
:10D5A000BE853124C37D0C55745DBE72FEB1DE8034
:10D5B000A706DC9B74F19BC1C1699BE48647BEEF63
:10D5C000C69DC10FCCA10C246F2CE92DAA84744AEE
:10D5D000DCA9B05CDA88F97652513E986DC631A864
:10D5E000C82703B0C77F59BFF30BE0C64791A7D543
:10D5F0005163CA0667292914850AB72738211B2ECB
:10D60000FC6D2C4D130D385354730A65BB0A6A76B2
:10D610002EC9C281852C7292A1E8BFA24B661AA8BE
:10D62000708B4BC2A3516CC719E892D1240699D6CE
:10D6300085350EF470A06A1016C1A419086C371E47
:10D640004C774827B5BCB034B30C1C394AAAD84E25
:10D650004FCA9C5BF36F2E68EE828F746F63A57860
:10D660001478C8840802C78CFAFFBE90EB6C50A4F3
:10D67000F7A3F9BEF27871C6200000004000000058
:10D680007C6E0000E46E00000C7000004481DA0E35
:10D690004E03C49E847725D83A93BF8048D90000B2
:10D6A00054D9000060D900006CD900005B25735D7F
:10D6B0002025733A204C6F7261496E69740D0A001F
:10D6C0005B25735D2025733A20446F6573206E6F70
:10D6D00074207265636F676E697A6520746865206F
:10D6E0006D6F64756C650D0A000000005B25735D4D
:10D6F0002025733A20435249544943414C3A204C27
:10D700006F5261206E6F7420666F756E642C206896
:10D71000616C7465640D0A00436F6E666967000092
:10D720005B25735D2025733A204465636964696EE7
:10D7300067206F6E206368616E6E656C20696E6431
:10D7400065782025642062656361757365206F6666
:10D750002074696D657374616D7020302C206E616A
:10D760006D652069732025730D0A00005B25735DCC
:10D770002025733A204465636964696E67206F6E83
:10D78000206368616E6E656C20696E646578202523
:10D79000642062656361757365206F66206E616DDC
:10D7A00065206C656E20302C206E616D652069737C
:10D7B0002025730D0A000000556E6B6E6F776E00AA
:10D7C0007646743046527567534F65716E6B736859
:10D7D000496D4D43566667484D357642787931003C
:10D7E00068657369656C6B6F0000000042524E20E3
:10D7F000574348204D696E69000000005075626C07
:10D800006963000042524E54657374005965730099
:10D810004E6F00004E6F64652064617461626173D5
:10D82000653A00004E6F64652025643A0A000000E6
:10D8300020204E616D653A2025730A005075626B99
:10D8400065790000536563726574000020204750BD
:10D85000533A206C61743D25642C206C6F6E3D251D
:10D86000640A00002020506174683A202E2E2E2079
:10D87000286E6F7420657870616E6465642C206119
:10D880006464206966206E6565646564290A000029
:10D890002020466C6167733A203078253032580A70
:10D8A00000000000202041757468656E7469636132
:10D8B0007465643A2025730A0000000020204C6142
:10D8C0007374205365656E202872656D6F746520D2
:10D8D0007473293A2025640A0000000020204C615E
:10D8E0007374205365656E20286C6F63616C2074BF
:10D8F00073293A2025640A00202053796E6320742E
:10D90000696D657374616D703A2025640A000000CA
:10D910002D2D2D2D2D2D2D2D2D2D2D2D2D2D2D2D37
:10D920002D2D2D2D2D2D2D2D2D2D2D2D2D2D2D2D27
:10D930002D2D2D2D2D2D0A008B3387E9C5CDEA6ABB
:10D94000C9E5EDBAA115CD7243686174206E6F64AC
:10D95000650000005265706561746572000000002A
:10D96000526F6F6D207365727665720053656E73CA
:10D970006F72000068656C6C6F207468657265007A
:10D980005B25735D2025733A2053797374656D436D
:10D990006C6B3A25640D0A0D0A0000005B25735D6F
:10D9A0002025733A204368697049443A2530387815
:10D9B0000D0A0D0A000000005B25735D2025733AF7
:10D9C0002053656E64696E67206D6573736167656A
:10D9D0000A0D0A005379535469636B20697320253B
:10D9E0006C6C75005B25735D2025733A2053656E62
:10D9F00064696E67207A65726F20686F7020616459
:10DA0000766572740A0D0A005B25735D2025733AF2
:10DA10002053656E64696E6720666C6F6F64206169
:10DA200064766572740A0D0A0000000053656E6426
:10DA3000696E67206D65737361676520617420533B
:10DA400079535469636B20697320256C6C750000F1
:10DA500053656E64696E67206120646972656374E2
:10DA6000206D65737361676520746F20746865202D
:10DA70006669727374206E6F64650A004368616E34
:10DA80006E656C20696E6465782025642C206E615B
:10DA90006D65642025732C2074696D657374616DE8
:10DAA000702069732025642C206861736820697375
:10DAB0002025640A0000000057686F6C65206672BC
:10DAC000616D65005B25735D2025733A2072737369
:10DAD000693D25645B64426D5D20736E723D256413
:10DAE0005B64425D20726177736E723D25645B7189
:10DAF0007561727465722064425D0D0A0000000059
:10DB00005B25735D2025733A202564207061636B6B
:10DB1000657473206C6F73740D0A00005B25735D70
:10DB20002025733A2073796E63576F72643D3078A5
:10DB300025780D0A000000005B25735D2025733AEF
:10DB400020535831323678206572726F722C206DF6
:10DB500061796265206E6F2053504920636F6E6E4D
:10DB6000656374696F6E0D0A000000005B25735DCC
:10DB70002025733A2053583132367820696E7374F9
:10DB8000616C6C65640D0A005B25735D2025733A3A
:10DB900020757365526567756C61746F724C444F84
:10DBA0003D25640D0A0000005B25735D2025733A56
:10DBB00020416C6D6F737420646F6E6520736574A3
:10DBC00074696E67204C6F52610D0A0053583132F0
:10DBD000363200005B25735D2025733A204C6F526E
:10DBE000614572726F7244656661756C743D25643F
:10DBF0000D0A0000474F4E452057524F4E470A002E
:10DC000073746172742052656164436F6D6D616EEF
:10DC1000640000005B25735D2025733A2052656126
:10DC200064436F6D6D616E643A20434D443D3078BE
:10DC3000253032780D0A0000656E642052656164FB
:10DC4000436F6D6D616E6400737461727420526510
:10DC50006164526567697374657200005B25735D6A
:10DC60002025733A20526561645265676973746553
:10DC7000723A205245473D3078253032780D0A00FF
:10DC80005B25735D2025733A2052656164696E6778
:10DC90002062797465730D0A000000005B25735DD6
:10DCA0002025733A20726561642061206279746571
:10DCB0000D0A0000656E64205265616452656769F3
:10DCC00073746572000000005B25735D2025733A54
:10DCD0002044617461496E3A25303278200D0A0083
:10DCE0005B25735D2025733A2057616974696E67FF
:10DCF00020666F722069646C650D0A005265736559
:10DD0000740000005B25735D2025733A202D2D2DB6
:10DD10002D2D2053657452782074696D656F75746C
:10DD20003D25640D0A0000005B25735D2025733AD4
:10DD300020536574527820496C6C6567616C205380
:10DD400074617475730D0A005B25735D2025733A49
:10DD50002053657453746F70527854696D65724FB7
:10DD60006E507265616D626C6544657465637420A4
:10DD7000656E61626C653D25640D0A005B25735D0F
:10DD80002025733A202D2D2D2D2D20536574547888
:10DD90002074696D656F7574496E4D733D25640D12
:10DDA0000A0000005B25735D2025733A20536574DB
:10DDB00054782074696D656F7574496E4D733D2597
:10DDC0006420746F75743D25640D0A005B25735DD6
:10DDD0002025733A205772697474656E20636F6DE5
:10DDE0006D616E642C207265747279696E670D0ABC
:10DDF000000000005B25735D2025733A2042726F9E
:10DE00006B65206F75740D0A000000005B25735D63
:10DE10002025733A20536574547820496C6C6567EB
:10DE2000616C205374617475730D0A005B25735D1A
:10DE30002025733A2057616974466F7249646C6596
:10DE40002054696D656F757420746578743D257311
:10DE50002074696D656F75743D256C750D0A000041
:10DE60005B25735D2025733A2057616974466F7294
:10DE700049646C65206661696C2072657472793DD5
:10DE800025640D0A000000005B25735D2025733AB0
:10DE9000207374617475733D253032780D0A00006B
:10DEA0005B25735D2025733A205772697465436F53
:10DEB0006D6D616E6432207374617475733D2530CD
:10DEC00032782072657472793D25640D0A00000075
:10DED0005B25735D2025733A2053504920547261AD
:10DEE0006E73616374696F6E206572726F723A301F
:10DEF00078253032780D0A0073746172742057727D
:10DF0000697465436F6D6D616E6432005B25735D8E
:10DF10002025733A205772697465436F6D6D616E89
:10DF2000643A20434D443D3078253032780D0A0064
:10DF3000656E64205772697465436F6D6D616E64C0
:10DF400032000000737461727420577269746552F4
:10DF50006567697374657200656E642057726974D1
:10DF60006552656769737465720000005B25735DB7
:10DF70002025733A20577269746552656769737416
:10DF800065723A205245473D3078253032780D0A87
:10DF9000000000005B25735D2025733A2044617406
:10DFA000614F75743A25303278200D0A0000000068
:10DFB0000001020203030303040404040404040430
:10DFC0000505050505050505050505050505050501
:10DFD00006060606060606060606060606060606E1
:10DFE00006060606060606060606060606060606D1
:10DFF00007070707070707070707070707070707B1
:10E0000007070707070707070707070707070707A0
:10E010000707070707070707070707070707070790
:10E020000707070707070707070707070707070780
:10E030000808080808080808080808080808080860
:10E040000808080808080808080808080808080850
:10E050000808080808080808080808080808080840
:10E060000808080808080808080808080808080830
:10E070000808080808080808080808080808080820
:10E080000808080808080808080808080808080810
:10E090000808080808080808080808080808080800
:10E0A00008080808080808080808080808080808F0
:10E0B000504F5349580000002E000000002020203F
:10E0C0002020202020202828282828202020202028
:10E0D00020202020202020202020202020881010F8
:10E0E0001010101010101010101010101004040454
:10E0F0000404040404040410101010101010414112
:10E1000041414141010101010101010101010101FF
:10E110000101010101010101101010101010424213
:10E1200042424242020202020202020202020202CF
:10E13000020202020202020210101010200000006F
:10E1400000000000000000000000000000000000CF
:10E1500000000000000000000000000000000000BF
:10E1600000000000000000000000000000000000AF
:10E17000000000000000000000000000000000009F
:10E18000000000000000000000000000000000008F
:10E19000000000000000000000000000000000007F
:10E1A000000000000000000000000000000000006F
:10E1B000000000000000000000000000000000005F
:10E1C000000000000000000000000000000000004F
:10E1D000000000000000000000000000000000003F
:10E1E000000000000000000000000000000000002F
:10E1F000000000000000000000000000000000001F
:10E20000000000000000000000000000000000000E
:10E2100000000000000000000000000000000000FE
:10E22000232D302B20000000686C4C00656667458C
:10E2300046470000303132333435363738394142C1
:10E240004344454600000000303132333435363720
:0CE25000383961626364656600000000FC
:10E25C00000000000000000001020304060708098A
:10E26C000000000001020304010203040607080970
:10E27C00430000000000000000000000000000004F
:10E28C000000000000000000000000000000000082
:10E29C00430000000000000000000000000000002F
:10E2AC000000000000000000000000000000000062
:10E2BC00430000000000000000000000000000000F
:10E2CC000000000000000000000000000000000042
:10E2DC0043000000000000000000000000000000EF
:10E2EC000000000000000000000000000000000022
:10E2FC0043000000000000000000000000000000CF
:10E30C000000000000000000000000000000000001
:10E31C0043000000000000000000000000000000AE
:10E32C0000000000000000000000000000000000E1
:10E33C00430000000000000000000000000000008E
:10E34C0000000000000000000000000000000000C1
:10E35C0090A10000FC98000000000000BCE0000050
:10E36C00B8E00000B4D90000B4D90000B4D9000062
:10E37C00B4D90000B4D90000B4D90000B4D900005D
:10E38C00B4D90000B4D90000FFFFFFFFFFFFFFFF6F
:10E39C00FFFFFFFFFFFF000001004153434949000D
:10E3AC000000000000000000000000000000000061
:10E3BC0000000000000000000000415343494900E8
:10E3CC000000000000000000000000000000000041
:10E3DC000000000000000000000000000000000031
:10E3EC00E0E1000000E20000C0E1000000000000DD
:10E3FC000000000000000000000000000000000011
:10E40C000000000000000000000000000000000000
:10E41C0000000000000000000000000000000000F0
:10E42C0000000000000000000000000000000000E0
:10E43C0000000000000000000000000000000000D0
:10E44C0000D8B80502040608801100208C010020B9
:08E45C008C010020000000000B
:00000001FF
